:020000040800F2
:10000000DC0B00205D380008415200084D5200080A
:10001000555200085D5200086552000800000000BB
:100020000000000000000000000000006D52000809
:100030007952000800000000855200089152000823
:10004000D9380008D9380008D9380008D93800084C
:10005000D9380008D9380008D9380008D93800083C
:10006000D9380008D9380008D9380008D93800082C
:10007000D9380008D9380008D9380008D93800081C
:10008000D9380008D9380008D9380008D93800080C
:10009000D9380008D9380008D9380008D9380008FC
:1000A000D9380008D9380008D9380008D9380008EC
:1000B000D9380008D9380008D9380008D9380008DC
:1000C000D9380008D9380008D9380008D9380008CC
:1000D000D9380008D9380008D9380008D9380008BC
:1000E0009D520008D9380008D9380008D9380008CE
:1000F000D9380008D9380008D9380008D93800089C
:10010000D9380008D9380008D9380008D93800088B
:10011000D9380008D9380008D9380008D93800087B
:10012000D9380008D9380008D9380008D93800086B
:10013000D9380008D9380008D9380008D93800085B
:10014000D9380008D9380008D9380008D93800084B
:10015000D9380008D9380008D9380008D93800083B
:10016000D9380008D9380008D9380008D93800082B
:10017000D9380008D9380008D9380008D93800081B
:10018000D9380008D938000890B484B000AF0246CE
:100190000B46FA71BB714FF00003FB60BB7903F0B3
:1001A00003034FEA83034FF00F0202FA03F3FB60ED
:1001B0004FF46053C4F20103BA794FEA9202D2B20B
:1001C00010464FF46052C4F20102B9794FEA91012E
:1001D000C9B201F1020152F82110FA686FEA020275
:1001E000114000F1020243F822104FF46053C4F2B0
:1001F0000103BA794FEA9202D2B210464FF460522C
:10020000C4F20102B9794FEA9101C9B201F10201C8
:1002100052F82110FC79BA7902F003024FEA820207
:1002200004FA02F2114300F1020243F8221007F12E
:100230001007BD4690BC704780B582B000AF4FF04C
:100240003A004FF0010104F0DBFD4CF233733B60E8
:100250004FF002033B714FF002037B714FF000033C
:10026000BB714FF00003FB713B464FF44060C4F29A
:10027000020019460AF090F84FF44060C4F2020000
:100280004FF000014FF00C020AF062F94FF44060A9
:10029000C4F202004FF001014FF00C020AF058F9CD
:1002A0004FF44060C4F202004FF004014FF00C0222
:1002B0000AF04EF94FF44060C4F202004FF005011D
:1002C0004FF00C020AF044F94FF44060C4F202000F
:1002D0004FF008014FF00C020AF03AF94FF4406079
:1002E000C4F202004FF009014FF00C020AF030F99D
:1002F0004FF44060C4F202004FF00A014FF00C02CC
:100300000AF026F94FF44060C4F202004FF00E01EB
:100310004FF00C020AF01CF94FF44060C4F20200E6
:100320004FF00F014FF00C020AF012F94FF68073F4
:100330003B603B464FF48050C4F2020019460AF07D
:100340002BF84FF48050C4F202004FF007014FF039
:100350000C020AF0FDF84FF48050C4F202004FF096
:1003600008014FF00C020AF0F3F84FF48050C4F289
:1003700002004FF009014FF00C020AF0E9F84FF4C7
:100380008050C4F202004FF00A014FF00C020AF054
:10039000DFF84FF48050C4F202004FF00B014FF031
:1003A0000C020AF0D5F84FF48050C4F202004FF06E
:1003B0000C014FF00C020AF0CBF84FF48050C4F25D
:1003C00002004FF00D014FF00C020AF0C1F84FF49B
:1003D0008050C4F202004FF00E014FF00C020AF000
:1003E000B7F84FF48050C4F202004FF00F014FF005
:1003F0000C020AF0ADF84FF008033B603B464FF4A7
:100400008050C4F20200194609F0C6FF4FF4805034
:10041000C4F202004FF003014FF00C020AF098F80A
:100420004FF080033B603B464FF44060C4F2020053
:10043000194609F0B1FF4FF44060C4F202004FF0DA
:100440000A014FF00C020AF083F84FF008033B60FA
:100450004FF001033B714FF000037B714FF000033D
:10046000BB714FF00003FB713B464FF44060C4F298
:100470000200194609F090FF4FF400533B604FF023
:1004800001033B714FF001037B714FF00003BB711F
:100490004FF00003FB713B464FF44060C4F2020092
:1004A000194609F079FF4FF44060C4F202004FF49E
:1004B00000510AF031F807F10807BD4680BD00BFC2
:1004C00080B596B000AF4FF001004FF0010104F08D
:1004D000C1FC4FF001033B604FF000037B604FF025
:1004E0000903BB604FF00003FB604FF000033B616A
:1004F0004FF000037B614FF00003BB614FF000033E
:10050000FB614FF000033B624FF000037B624FF052
:100510001003BB624FF00003FB624FF000033B632C
:100520004FF000037B634FF00003BB634FF0000309
:10053000FB634FF480533B644FF000037B644FF048
:100540000003BB644FF00003FB643B463B653B4646
:100550007B6507F11C03184609F04CFE4FF00000C4
:100560004FF0010109F0EEFE07F15807BD4680BDCE
:1005700080B582B000AFFFF75FFEFFF7A1FF4FF03D
:10058000050000F0C7FC4FF44060C4F202004FF0D9
:10059000080109F0CFFF4FF00A0000F0BBFC4FF458
:1005A0004060C4F202004FF0080109F0B5FF4FF0BF
:1005B00010004FF0010100F01BF94FF01E004FF04A
:1005C000B20100F015F94FF028004FF0060100F0DD
:1005D0000FF94FF000004FF0010100F009F94FF062
:1005E000010047F2EF0100F003F94FF002004FF471
:1005F000C06100F0FDF84FF010004FF0000100F076
:10060000F7F84FF0050000F085FC4FF0110046F6BA
:10061000200100F0EDF84FF0120040F6991100F0C3
:10062000E7F84FF026004FF4605100F0E1F84FF08A
:1006300007004FF0330100F0DBF84FF00C004FF0F3
:10064000050100F0D5F84FF030004FF0000100F048
:10065000CFF84FF0310040F2033100F0C9F84FF00D
:10066000320040F2074100F0C3F84FF0330040F28F
:10067000013100F0BDF84FF0340040F2013100F0DC
:10068000B7F84FF0350040F2034100F0B1F84FF0F9
:10069000360040F2077100F0ABF84FF037004FF42E
:1006A000806100F0A5F84FF03A004FF4206100F0AF
:1006B0009FF84FF03B004FF4805100F099F84FF055
:1006C0000D004FF00A0100F093F84FF00E004FF4C8
:1006D000385100F08DF84FF044004FF46F4100F0B6
:1006E00087F84FF045004FF0000100F081F84FF01F
:1006F000460040F23F1100F07BF84FF04E004FF003
:10070000000100F075F84FF04F004FF0000100F0CD
:100710006FF84FF022004FF0000100F069F84FF041
:1007200000037B6007E04FF0000000F099F87B6861
:1007300003F101037B607A6842F6FF33C0F20103E4
:100740009A42F0D940F27C00C2F2000000F0B0F80A
:1007500007F10807BD4680BD80B582B000AF0246F4
:100760000B46FA807B71FB884FF04E00194600F073
:100770003FF87B799BB24FF04F00194600F038F8F4
:1007800007F10807BD4680BD80B582B000AFF88094
:1007900079717A803B71FA887B88D31A9BB203F116
:1007A00001039BB24FF04500194600F021F8FB8889
:1007B0004FF04600194600F01BF87B799AB23B795E
:1007C0009BB2D31A9BB203F101039BB29AB27B791D
:1007D0004FEA03239BB213439BB29BB24FF04400FA
:1007E000194600F005F807F10807BD4680BD00BFB7
:1007F00080B483B000AF02460B46FA71BB804FF065
:10080000C043FA7992B21A804FF00003C6F2100387
:10081000BA881A8007F10C07BD4680BC704700BF3C
:1008200080B483B000AF0346FB714FF0C043FA7948
:1008300092B21A804FF00003C6F210031B889BB2DD
:10084000184607F10C07BD4680BC704780B400AF66
:100850004FF0C0434FF022021A80BD4680BC704763
:1008600080B483B000AF0346FB804FF00003C6F2B4
:100870001003FA881A8007F10C07BD4680BC704748
:1008800080B400AF4FF00003C6F210031B889BB288
:100890001846BD4680BC704780B400AFBD4680BCE2
:1008A000704700BF80B400AFBD4680BC704700BF3A
:1008B00080B483B000AF786040F26413C2F20003EA
:1008C0007A681A6007F10C07BD4680BC704700BF0C
:1008D00080B584B000AF0346FB804FF00003FB609F
:1008E0004FF0110046F62001FFF782FF40F23F1063
:1008F0004FF00001FFF730FFFFF7A8FF4FF00003B4
:10090000FB6009E04FF00003C6F21003FA881A807A
:10091000FB6803F10103FB60FA6842F6FF33C0F2A3
:1009200001039A42EED907F11007BD4680BD00BF12
:1009300080B584B000AFF88079717A803B717A79A4
:100940003B79D318DBB203F1FF33D9B2F8887A8848
:100950003B79FFF719FF4FF0110046F62001FFF732
:1009600047FFFA887B7910461946FFF7F5FEFFF737
:100970006DFF4FF00003FB6007E03B8B1846FFF76D
:100980006FFFFB6803F10103FB607B883A7902FB90
:1009900003F31A46FB689A42EFD840F23F104FF03B
:1009A00000014FF4A0724FF0F003FFF7EDFE07F1E6
:1009B0001007BD4680BD00BF80B584B000AFF88091
:1009C00079717A803B714FF00003FB813B79002BFA
:1009D00006D14FF011004FF4D041FFF709FF08E0B6
:1009E0003B79012B05D14FF0110046F62801FFF7A6
:1009F000FFFEFA887B7910461946FFF7ADFEFFF738
:100A000025FF4FF00003FB810BE040F26A13C2F2B6
:100A100000031B881846FFF723FFFB8903F101033E
:100A2000FB81FA897B889A42EFD34FF0110046F69A
:100A30002001FFF7DDFE07F11007BD4680BD00BFB6
:100A400080B588B000AFF88079717A803B717A8880
:100A5000FB88D31A9BB2FB833B799AB27B799BB21A
:100A6000D31A9BB2BB83FA887B7910461946FFF7ED
:100A700073FEFFF7EBFE40F26A13C2F200031B881D
:100A80001846FFF7EDFEB7F91E3083EAE372A2EBDA
:100A9000E372B7F91C30002BB8BF5B429A4203DA0D
:100AA000B7F91E30002B5DD0B7F91C3006EE903A36
:100AB000B8EEE67AB7F91E3006EE903AF8EEE67A2E
:100AC000C7EE277AC7ED047A7B7907EE903AB8EE45
:100AD000E77AFB8807EE903AF8EEE76AD7ED047AFA
:100AE00066EEA77A77EE677AC7ED037AB7F91E301C
:100AF000002B02DA4FF6FF7301E04FF00103FB8396
:100B00002BE0FA8BFB88D318FB80FB8806EE903A2B
:100B1000B8EEE67AD7ED047A27EE277AD7ED037A96
:100B200077EE277A17EE900A0AF082FA02460B4611
:100B300043EC102B0AF0B2FD0346DBB2FA881046F4
:100B40001946FFF709FEFFF781FE40F26A13C2F271
:100B500000031B881846FFF783FEFA887B889A42B9
:100B6000CFD15DE0B7F91E3007EE903AB8EEE77AE4
:100B7000B7F91C3006EE903AF8EEE67AC7EE277A1F
:100B8000C7ED067AFB8807EE903AB8EEE77A7B79F4
:100B900007EE903AF8EEE76AD7ED067A66EEA77AA6
:100BA00077EE677AC7ED057AB7F91C30002B02DAC9
:100BB0004FF6FF7301E04FF00103BB832CE0BB8BCA
:100BC000DAB27B79D3187B717B7906EE903AB8EE76
:100BD000E67AD7ED067A27EE277AD7ED057A77EE13
:100BE000277A17EE900A0AF023FA02460B4643ECE6
:100BF000102B0AF053FD03469AB27B791046194632
:100C0000FFF7AAFDFFF722FE40F26A13C2F20003CB
:100C10001B881846FFF724FE7A793B799A42CED199
:100C200007F12007BD4680BD80B582B000AFF880D7
:100C300079717A803B71F9887A797B880846114608
:100C40001A464FF00003FFF7B7FE7A793B79D318C5
:100C5000DBB203F1FF33DAB2F9887B88084611462C
:100C60001A464FF00003FFF7A7FE3B799BB2F988C5
:100C70007A79084611461A464FF00103FFF79CFEA9
:100C8000FA887B88D31A9BB203F1010399B23B79AE
:100C90009BB27A79084611461A464FF00103FFF7D6
:100CA0008BFE07F10807BD4680BD00BF80B483B04E
:100CB00000AF0346FB8040F20203C2F20003FA8851
:100CC0001A8007F10C07BD4680BC704780B483B022
:100CD00000AF0346FB8040F26A13C2F20003FA88B9
:100CE0001A8007F10C07BD4680BC704780B483B002
:100CF00000AF0346FB8040F26813C2F20003FA889B
:100D00001A8007F10C07BD4680BC704780B586B0DD
:100D100000AF13460246FA800A46BA807B807B8881
:100D20004FEA4303C3F103037B614FF000033B61D0
:100D30007B88FB60E5E03B699AB2FB88D3189AB2E6
:100D4000BB88D9B2FB68DBB2CB18DBB210461946C0
:100D5000FFF702FDFFF77AFD40F26A13C2F20003CB
:100D60001B881846FFF77CFD3B699AB2FB88D318B5
:100D70009AB2BB88D9B2FB68DBB2CB1ADBB21046A1
:100D80001946FFF7E9FCFFF761FD40F26A13C2F272
:100D900000031B881846FFF763FD3B699BB2FA8886
:100DA000D31A9AB2BB88D9B2FB68DBB2CB18DBB2DC
:100DB00010461946FFF7D0FCFFF748FD40F26A13D2
:100DC000C2F200031B881846FFF74AFD3B699BB23D
:100DD000FA88D31A9AB2BB88D9B2FB68DBB2CB1AB5
:100DE000DBB210461946FFF7B7FCFFF72FFD40F2C4
:100DF0006A13C2F200031B881846FFF731FDFB6837
:100E00009AB2FB88D3189AB2BB88D9B23B69DBB2DD
:100E1000CB18DBB210461946FFF79EFCFFF716FD14
:100E200040F26A13C2F200031B881846FFF718FD50
:100E3000FB689AB2FB88D3189AB2BB88D9B23B69D7
:100E4000DBB2CB1ADBB210461946FFF785FCFFF781
:100E5000FDFC40F26A13C2F200031B881846FFF73C
:100E6000FFFCFB689BB2FA88D31A9AB2BB88D9B24E
:100E70003B69DBB2CB18DBB210461946FFF76CFCBE
:100E8000FFF7E4FC40F26A13C2F200031B88184625
:100E9000FFF7E6FCFB689BB2FA88D31A9AB2BB88CC
:100EA000D9B23B69DBB2CB1ADBB210461946FFF769
:100EB00053FCFFF7CBFC40F26A13C2F200031B881D
:100EC0001846FFF7CDFC7B69002B08DA3B694FEA37
:100ED00083027B69D31803F106037B610DE03A6955
:100EE000FB68D31A4FEA83027B69D31803F10A0324
:100EF0007B61FB6803F1FF33FB603B6903F1010396
:100F00003B613A69FB689A427FF615AF07F1180713
:100F1000BD4680BD80B485B000AF78604FF000035F
:100F2000FB607B6842F2107202FB03F3FB6003E09C
:100F3000FB6803F1FF33FB60FB68002BF8D107F17E
:100F40001407BD4680BC70472DE9B04F2DED028BD4
:100F5000EAB000AF4FF00003C7F8A4314FF0000330
:100F6000C7F8A0314FF00003C7F89C314FF00003E1
:100F7000C7F898314FF00003C7F894314FF00003E1
:100F8000C7F890314FF00003C7F88C314FF00003E1
:100F9000C7F888314FF00003C7F884314FF00003E1
:100FA000C7F880314FF00003C7F87C314FF00003E1
:100FB000C7F878314FF00003C7F874314FF00003E1
:100FC000C7F870314FF00003C7F86C314FF00003E1
:100FD000C7F868314FF00003C7F864314FF00003E1
:100FE000C7F860314FF00003C7F85C314FF00003E1
:100FF000C7F858314FF00003C7F854314FF00003E1
:10100000C7F850314FF00003C7F84C314FF00003E0
:10101000C7F848314FF00003C7F844314FF00003E0
:10102000C7F840314FF00003C7F83C314FF00003E0
:10103000C7F838314FF00003C7F834314FF00003E0
:10104000C7F8303140F20803C2F200031B884FEAB0
:101050005303A7F82E3140F20803C2F200031A88A6
:101060004CF6CD43CCF6CC43A3FB02034FEA9303EB
:10107000A7F82C3140F20803C2F200031A884CF69C
:10108000CD43CCF6CC43A3FB02134FEA93039BB2B0
:101090004FEA8303A7F82A3140F20803C2F20003A3
:1010A0001A884CF6CD43CCF6CC43A3FB02034FEA9F
:1010B00093039BB24FEA8303A7F8283140F2080359
:1010C000C2F200031A884CF6CD43CCF6CC43A3FB06
:1010D00002134FEA9303A7F8263140F20603C2F247
:1010E00000031B884FEA5303A7F8243140F206039C
:1010F000C2F200031A884CF6CD43CCF6CC43A3FBD6
:1011000002034FEA9303A7F8223140F20603C2F22A
:1011100000031A884CF6CD43CCF6CC43A3FB021354
:101120004FEA9303A7F8203140F20603C2F200030E
:101130001A884CF6CD43CCF6CC43A3FB02034FEA0E
:1011400093039BB24FEA8303A7F81E3140F20603D4
:10115000C2F200031A884CF6CD43CCF6CC43A3FB75
:1011600002134FEA93039BB24FEA8303A7F81C31A3
:101170004FF000024FF00003C7E944234FF0000294
:101180004FF00003C7E942234FF000024FF0000385
:10119000C7E940234FF000024FF00003C7E93E23A8
:1011A0004FF000024FF00003C7E93C234FF000026C
:1011B0004FF00003C7E93A234FF000024FF000035D
:1011C000C7E938234FF000024FF00003C7E9362388
:1011D0004FF000024FF00003C7E934234FF0000244
:1011E0004FF00003C7E932234FF000024FF0000335
:1011F000C7E930234FF000024FF00003C7E92E2368
:101200004FF000024FF00003C7E92C234FF000031A
:10121000C7F8AC3007F1A8034FF000021A6007F1DD
:10122000A4034FF000021A6007F1A0034FF0000280
:101230001A6007F19C034FF000021A6007F198034F
:101240004FF000021A6007F194034FF000021A6099
:1012500007F190034FF000021A6007F18C034FF082
:1012600000021A6007F188034FF000021A6007F1CC
:1012700084034FF000021A6007F180034FF0000270
:101280001A6007F17C034FF000021A6007F178033F
:101290004FF000021A6007F174034FF000021A6069
:1012A00007F170034FF000021A6007F16C034FF072
:1012B00000021A6007F168034FF000021A6007F19C
:1012C00064034FF000021A6007F160034FF0000260
:1012D0001A6007F15C034FF000021A6007F158032F
:1012E0004FF000021A6007F154034FF000021A6039
:1012F00007F150034FF000021A6007F14C034FF062
:1013000000021A6007F148034FF000021A6007F16B
:1013100044034FF000021A6007F140034FF000024F
:101320001A6007F13C034FF000021A6007F138031E
:101330004FF000021A6007F134034FF000021A6008
:1013400007F130034FF000021A6007F12C034FF051
:1013500000021A6007F128034FF000021A6007F13B
:1013600024034FF000021A6007F120034FF000023F
:101370001A6007F11C034FF000021A6007F118030E
:101380004FF000021A6007F114034FF000021A60D8
:1013900007F110034FF000021A6007F10C034FF041
:1013A00000021A6007F108034FF000021A6007F10B
:1013B00006034FF000021A8007F104034FF0000209
:1013C0001A8007F102034FF000021A803B464FF0EB
:1013D00000021A804FF6FF7002F060F84FF0000034
:1013E00002F0C2F84FF6FF7001F01CFE40F2060357
:1013F000C2F200031A8844F62513C2F29243A3FBFB
:101400000203D21A4FEA52029B184FEA93039BB28F
:101410001A464FEA4202D3189AB240F20803C2F2C7
:1014200000031B88A3F119039BB2104619464DF621
:101430002002C0F600024FF0000301F003FD4FF060
:10144000280008F071FD40F20603C2F200031A887A
:1014500044F62513C2F29243A3FB0213D21A4FEAB9
:1014600052029B184FEA93039BB21A464FEA42027C
:10147000D3189AB240F20803C2F200031B88A3F10A
:1014800019039BB2104619464DF63402C0F600020D
:101490004FF0000301F0D6FC4FF0280008F044FDA7
:1014A00040F20603C2F200031A8844F62513C2F282
:1014B0009243A3FB0203D21A4FEA52029B184FEA4F
:1014C00093039BB21A464FEA4202D3189AB240F2F3
:1014D0000803C2F200031B88A3F119039BB2104654
:1014E00019464DF64802C0F600024FF0000301F025
:1014F000A9FC4FF01E0008F017FD40F2AA13C2F23B
:1015000000034FF000021A704FF6FF7001F08AFDE1
:1015100040F20603C2F200031B884FEA53039AB25B
:1015200040F20803C2F200031B884FEA53039BB248
:101530001046194604F0AAFD01E009F019FB40F23B
:10154000AA13C2F200031B78DBB2002BF5D040F2E5
:10155000BC13C2F200031B68C7F8A43140F2C413E5
:10156000C2F200031B68C7F890314FF0320008F058
:10157000DBFC09F0F7FA40F2AA13C2F200034FF0C5
:1015800000021A704FF6FF7001F04CFD40F20603A6
:10159000C2F200031A884CF6CD43CCF6CC43A3FB31
:1015A00002134FEA93039AB240F20803C2F2000317
:1015B00019884CF6CD43CCF6CC43A3FB01034FEA8C
:1015C00093039BB21046194604F060FD01E009F058
:1015D000CFFA40F2AA13C2F200031B78DBB2002B51
:1015E000F5D040F2BC13C2F200031B68C7F8A0316B
:1015F00040F2C413C2F200031B68C7F88C314FF0ED
:10160000320008F091FC09F0ADFA40F2AA13C2F2E0
:1016100000034FF000021A704FF6FF7001F002FD58
:1016200040F20603C2F200031A884CF6CD43CCF612
:10163000CC43A3FB02134FEA93039AB240F2080390
:10164000C2F2000319884CF6CD43CCF6CC43A3FB81
:1016500001034FEA93039BB24FEA83039BB2104608
:10166000194604F013FD01E009F082FA40F2AA13D2
:10167000C2F200031B78DBB2002BF5D040F2BC13A2
:10168000C2F200031B68C7F89C3140F2C413C2F2D7
:1016900000031B68C7F888314FF0320008F044FCA3
:1016A00009F060FA40F2AA13C2F200034FF0000200
:1016B0001A704FF6FF7001F0B5FC40F20603C2F25B
:1016C00000031A884CF6CD43CCF6CC43A3FB02139F
:1016D0004FEA93039BB24FEA83039AB240F20803A6
:1016E000C2F2000319884CF6CD43CCF6CC43A3FBE1
:1016F00001034FEA93039BB24FEA83039BB2104668
:10170000194604F0C3FC01E009F032FA40F2AA13D2
:10171000C2F200031B78DBB2002BF5D040F2BC1301
:10172000C2F200031B68C7F8983140F2C413C2F23A
:1017300000031B68C7F884314FF0320008F0F4FB57
:1017400009F010FA40F2AA13C2F200034FF00002AF
:101750001A704FF6FF7001F065FC40F20603C2F20A
:1017600000031A884CF6CD43CCF6CC43A3FB0213FE
:101770004FEA93039BB24FEA83039AB240F2080305
:10178000C2F2000319884CF6CD43CCF6CC43A3FB40
:1017900001034FEA93039BB21046194604F076FC0E
:1017A00001E009F0E5F940F2AA13C2F200031B7848
:1017B000DBB2002BF5D040F2BC13C2F200031B6871
:1017C000C7F8943140F2C413C2F200031B68C7F893
:1017D00080314FF0320008F0A7FB09F0C3F940F266
:1017E000AA13C2F200034FF000021A704FF6FF7006
:1017F00001F018FC40F20603C2F200031B884FEA16
:1018000053039AB240F20803C2F200031B884FEA66
:1018100053039BB21046194604F038FC01E009F06E
:10182000A7F940F2AA13C2F200031B78DBB2002B27
:10183000F5D040F2BC13C2F200031B68C7F87C313C
:1018400040F2C413C2F200031B68C7F868314FF0BE
:10185000320008F069FB09F085F940F2AA13C2F2E0
:1018600000034FF000021A704FF6FF7001F0DAFB30
:1018700040F20603C2F200031A884CF6CD43CCF6C0
:10188000CC43A3FB02134FEA93039AB240F208033E
:10189000C2F2000319884CF6CD43CCF6CC43A3FB2F
:1018A00001034FEA93039BB21046194604F0EEFB86
:1018B00001E009F05DF940F2AA13C2F200031B78BF
:1018C000DBB2002BF5D040F2BC13C2F200031B6860
:1018D000C7F8783140F2C413C2F200031B68C7F89E
:1018E00064314FF0320008F01FFB09F03BF940F281
:1018F000AA13C2F200034FF000021A704FF6FF70F5
:1019000001F090FB40F20603C2F200031A884CF685
:10191000CD43CCF6CC43A3FB02134FEA93039AB218
:1019200040F20803C2F2000319884CF6CD43CCF60E
:10193000CC43A3FB01034FEA93039BB24FEA83031B
:101940009BB21046194604F0A1FB01E009F010F922
:1019500040F2AA13C2F200031B78DBB2002BF5D0D1
:1019600040F2BC13C2F200031B68C7F8743140F2A6
:10197000C413C2F200031B68C7F860314FF0320095
:1019800008F0D2FA09F0EEF840F2AA13C2F200030E
:101990004FF000021A704FF6FF7001F043FB40F267
:1019A0000603C2F200031A884CF6CD43CCF6CC43B2
:1019B000A3FB02134FEA93039BB24FEA83039AB24D
:1019C00040F20803C2F2000319884CF6CD43CCF66E
:1019D000CC43A3FB01034FEA93039BB24FEA83037B
:1019E0009BB21046194604F051FB01E009F0C0F823
:1019F00040F2AA13C2F200031B78DBB2002BF5D031
:101A000040F2BC13C2F200031B68C7F8703140F209
:101A1000C413C2F200031B68C7F85C314FF03200F8
:101A200008F082FA09F09EF840F2AA13C2F200030D
:101A30004FF000021A704FF6FF7001F0F3FA40F217
:101A40000603C2F200031A884CF6CD43CCF6CC4311
:101A5000A3FB02134FEA93039BB24FEA83039AB2AC
:101A600040F20803C2F2000319884CF6CD43CCF6CD
:101A7000CC43A3FB01034FEA93039BB210461946E4
:101A800004F004FB01E009F073F840F2AA13C2F27B
:101A900000031B78DBB2002BF5D040F2BC13C2F27E
:101AA00000031B68C7F86C3140F2C413C2F2000394
:101AB0001B68C7F858314FF0320008F035FA09F0CA
:101AC00051F840F2AA13C2F200034FF000021A705C
:101AD000D7F8A421D7F87C31D3184FEA5303C7F8BD
:101AE0005431D7F8A021D7F87831D3184FEA5303EF
:101AF000C7F85031D7F89C21D7F87431D3184FEA82
:101B00005303C7F84C31D7F89821D7F87031D31860
:101B10004FEA5303C7F84831D7F89421D7F86C310E
:101B2000D3184FEA5303C7F84431D7F89021D7F8B8
:101B30006831D3184FEA5303C7F84031D7F88C21E6
:101B4000D7F86431D3184FEA5303C7F83C31D7F8BC
:101B50008821D7F86031D3184FEA5303C7F83831DA
:101B6000D7F88421D7F85C31D3184FEA5303C7F86C
:101B70003431D7F88021D7F85831D3184FEA5303BE
:101B8000C7F83031D7F85431D7F8542102FB03F3AA
:101B9000C7F8AC3007F1A803D7F85021D7F8501197
:101BA00001FB02F21A6007F1A403D7F84C21D7F821
:101BB0004C1101FB02F21A6007F1A003D7F848218B
:101BC000D7F8481101FB02F21A6007F19C03D7F81D
:101BD0004421D7F8441101FB02F21A6007F198037F
:101BE000D7F84021D7F8401101FB02F21A6007F143
:101BF0009403D7F83C21D7F83C1101FB02F21A609C
:101C000007F19003D7F83821D7F8381101FB02F219
:101C10001A6007F18C03D7F83421D7F8341101FB8F
:101C200002F21A6007F18803D7F83021D7F8301193
:101C300001FB02F21A6007F18403D7F85421D7F8A8
:101C4000401101FB02F21A6007F18003D7F850211E
:101C5000D7F83C1101FB02F21A6007F17C03D7F8B8
:101C60004C21D7F8381101FB02F21A6007F1780312
:101C7000D7F84821D7F8341101FB02F21A6007F1B6
:101C80007403D7F84421D7F8301101FB02F21A602F
:101C9000B7F82E2107F17003D7F8541101FB02F2B7
:101CA0001A60B7F82C2107F16C03D7F8501101FB2B
:101CB00002F21A60B7F82A2107F16803D7F84C112D
:101CC00001FB02F21A60B7F8282107F16403D7F884
:101CD000481101FB02F21A60B7F8262107F16003F0
:101CE000D7F8441101FB02F21A60B7F82E2107F170
:101CF0005C03D7F8401101FB02F21A60B7F82C21FF
:101D000007F15803D7F83C1101FB02F21A60B7F84B
:101D10002A2107F15403D7F8381101FB02F21A60A7
:101D2000B7F8282107F15003D7F8341101FB02F26C
:101D30001A60B7F8262107F14C03D7F8301101FBE0
:101D400002F21A60B7F8242107F14803D7F85411BA
:101D500001FB02F21A60B7F8222107F14403D7F819
:101D6000501101FB02F21A60B7F8202107F140037D
:101D7000D7F84C1101FB02F21A60B7F81E2107F1E7
:101D80003C03D7F8481101FB02F21A60B7F81C2196
:101D900007F13803D7F8441101FB02F21A60B7F8D3
:101DA000242107F13403D7F8401101FB02F21A6035
:101DB000B7F8222107F13003D7F83C1101FB02F2FA
:101DC0001A60B7F8202107F12C03D7F8381101FB6E
:101DD00002F21A60B7F81E2107F12803D7F8341170
:101DE00001FB02F21A60B7F81C2107F12403D7F8AF
:101DF000301101FB02F21A6007F1A803D7F8AC20FA
:101E00001B68D21807F1A4031B68D21807F1A003BE
:101E10001B68D11807F1200307F19C0212688A1889
:101E20001A6007F1980207F1940312681B68D21830
:101E300007F190031B68D21807F18C031B68D118B7
:101E400007F11C0307F1880212688A181A6007F16B
:101E5000840207F1800312681B68D21807F17C0323
:101E60001B68D21807F178031B68D11807F1180313
:101E700007F1740212688A181A60D7F854319AB2BE
:101E8000D7F850319BB2D3189AB2D7F84C319BB2E5
:101E9000D3189AB2D7F848319BB2D31899B2D7F871
:101EA00044319AB207F106038A181A80D7F84031F4
:101EB0009AB2D7F83C319BB2D3189AB2D7F83831DE
:101EC0009BB2D3189AB2D7F834319BB2D31899B2D7
:101ED000D7F830319AB207F104038A181A8007F153
:101EE000700207F16C0312681B68D21807F16803CF
:101EF0001B68D21807F164031B68D11807F114039B
:101F000007F1600212688A181A6007F1480207F1A7
:101F1000440312681B68D21807F140031B68D218EB
:101F200007F13C031B68D11807F1100307F13802D1
:101F300012688A181A6007F15C0207F158031268E8
:101F40001B68D21807F154031B68D21807F150031D
:101F50001B68D11807F10C0307F14C0212688A18AC
:101F60001A6007F1340207F1300312681B68D218B7
:101F700007F12C031B68D21807F128031B68D1183E
:101F800007F1080307F1240212688A181A60B7F8EB
:101F90002E21B7F82C31D3189AB2B7F82A31D318BA
:101FA0009AB2B7F82831D31899B207F10203B7F8FB
:101FB00026218A181A80B7F82421B7F82231D318BD
:101FC0009AB2B7F82031D3189AB2B7F81E31D318A5
:101FD00099B23B46B7F81C218A181A8007F12003F2
:101FE000186809F003F804460D4607F11C03186849
:101FF00008F0FCFF02460B462046294609F06CF823
:1020000002460B4614461D4607F11803186808F0EF
:10201000EDFF8046894607F11803186808F0E6FFCF
:1020200002460B464046494609F056F802460B4622
:102030002046294608F09CFE02460B4610461946EB
:102040004FF000024FF00003C4F2140309F044F80B
:1020500002460B4614461D4607F11803186808F09F
:10206000C5FF8046894607F106031B88184608F01D
:10207000CDFF02460B464046494609F02DF8024680
:102080000B469046994607F104031B88184608F052
:10209000BDFF02460B464046494609F01DF8024680
:1020A0000B461046194608F065FE02460B462046D0
:1020B000294608F05FFE02460B4614461D4607F10E
:1020C0002003186808F092FF8046894607F1040350
:1020D0001B88184608F09AFF02460B4640464946C0
:1020E00008F0FAFF02460B469046994607F10403B2
:1020F0001B88184608F08AFF02460B4640464946B0
:1021000008F0EAFF02460B462046294608F030FE5A
:1021100002460B4614461D4607F11C03186808F0DA
:1021200065FF8046894607F106031B88184608F0BC
:102130006DFF02460B464046494608F0CDFF024679
:102140000B469046994607F106031B88184608F08F
:102150005DFF02460B464046494608F0BDFF024679
:102160000B462046294608F003FE02460B46C7E907
:10217000382307F11403186808F038FF04460D46A9
:1021800007F11C03186808F031FF02460B46204691
:10219000294608F0A1FF02460B4614461D4607F1EA
:1021A0000C03186808F022FF8046894607F11803DF
:1021B000186808F01BFF02460B464046494608F0E7
:1021C0008BFF02460B462046294608F0D1FD024609
:1021D0000B46104619464FF000024FF00003C4F2C0
:1021E000140308F079FF02460B4614461D4607F11A
:1021F00004031B88184608F0F9FE8046894607F15B
:102200000C03186808F0F2FE82468B4607F10603BD
:102210001B88184608F0FAFE02460B4650465946FF
:1022200008F05AFF02460B4692469B4607F11403FC
:10223000186808F0DBFE41EC180B07F104031B885B
:10224000184608F0E3FE02460B4651EC180B08F066
:1022500043FF02460B465046594608F089FD0246A8
:102260000B464046494608F037FF02460B462046DB
:10227000294608F07FFD02460B4614461D4607F12D
:1022800002031B88184608F0B1FE8046894607F114
:102290001803186808F0AAFE82468B4607F104036B
:1022A0001B88184608F0B2FE02460B4650465946B7
:1022B00008F012FF02460B4692469B4607F11C03AC
:1022C000186808F093FE41EC180B07F106031B8811
:1022D000184608F09BFE02460B4651EC180B08F01E
:1022E000FBFE02460B465046594608F041FD0246A9
:1022F0000B464046494608F0EFFE02460B46204694
:10230000294608F037FD02460B46C7E9362307F198
:102310000C03186808F06AFE04460D4607F1200316
:10232000186808F063FE02460B462046294608F06E
:10233000D3FE02460B4614461D4607F114031868E7
:1023400008F054FE8046894607F11803186808F023
:102350004DFE02460B464046494608F0BDFE024689
:102360000B462046294608F003FD02460B46104660
:1023700019464FF000024FF00003C4F2140308F0B6
:10238000ABFE02460B4614461D4607F106031B88AA
:10239000184608F02BFE8046894607F1140318689A
:1023A00008F024FE82468B4607F104031B8818467A
:1023B00008F02CFE02460B465046594608F08CFEAB
:1023C00002460B4692469B4607F10C03186808F03C
:1023D0000DFE41EC180B07F106031B88184608F0A8
:1023E00015FE02460B4651EC180B08F075FE02462E
:1023F0000B465046594608F0BBFC02460B46404689
:10240000494608F069FE02460B462046294608F078
:10241000B1FC02460B4614461D4607F102031B8819
:10242000184608F0E3FD8046894607F1180318684E
:1024300008F0DCFD82468B4607F106031B88184630
:1024400008F0E4FD02460B465046594608F044FEAB
:1024500002460B4692469B4607F12003186808F097
:10246000C5FD41EC180B07F104031B88184608F062
:10247000CDFD02460B4651EC180B08F02DFE02462E
:102480000B465046594608F073FC02460B46404640
:10249000494608F021FE02460B462046294608F030
:1024A00069FC02460B46C7E9342307F11403186898
:1024B00008F09CFD04460D4607F11803186808F063
:1024C00095FD8046894607F104031B88184608F0ED
:1024D0009DFD02460B464046494608F0FDFD02467A
:1024E0000B469046994607F11C03186808F07EFDDC
:1024F00082468B4607F106031B88184608F086FDC6
:1025000002460B465046594608F0E6FD02460B4689
:102510004046494608F02CFC02460B462046294618
:1025200008F0DAFD02460B4614461D4607F10C037F
:10253000186808F05BFD8046894607F118031868A3
:1025400008F054FD82468B4607F106031B881846A7
:1025500008F05CFD02460B465046594608F0BCFDAB
:1025600002460B4692469B4607F12003186808F086
:102570003DFD41EC180B07F104031B88184608F0D9
:1025800045FD02460B4651EC180B08F0A5FD02462E
:102590000B465046594608F0EBFB02460B464046B8
:1025A000494608F099FD02460B462046294608F0A8
:1025B000E1FB02460B4614461D4607F102031B8849
:1025C000184608F013FD8046894607F12003186875
:1025D00008F00CFD82468B4607F11C03186808F0D2
:1025E00005FD02460B465046594608F075FD024669
:1025F0000B4692469B4607F11803186808F0F6FC54
:1026000041EC180B07F11803186808F0EFFC0246BC
:102610000B4651EC180B08F05FFD02460B46504686
:10262000594608F0A5FB02460B464046494608F0CD
:1026300053FD02460B462046294608F09BFB024606
:102640000B46C7E9322307F11003186808F0CEFCE7
:1026500004460D4607F11C03186808F0C7FC024643
:102660000B462046294608F037FD02460B46144625
:102670001D4607F10803186808F0B8FC8046894633
:1026800007F11803186808F0B1FC02460B464046F3
:10269000494608F021FD02460B462046294608F02F
:1026A00067FB02460B46104619464FF000024FF0FA
:1026B0000003C4F2140308F00FFD02460B46144653
:1026C0001D4607F104031B88184608F08FFC80465E
:1026D000894607F10803186808F088FC82468B4693
:1026E00007F106031B88184608F090FC02460B46CB
:1026F0005046594608F0F0FC02460B4692469B466F
:1027000007F11003186808F071FC41EC180B07F191
:1027100004031B88184608F079FC02460B4651EC6E
:10272000180B08F0D9FC02460B465046594608F0F3
:102730001FFB02460B464046494608F0CDFC0246C8
:102740000B462046294608F015FB02460B46144668
:102750001D463B461B88184608F048FC80468946C3
:1027600007F11803186808F041FC82468B4607F110
:1027700004031B88184608F049FC02460B465046E5
:10278000594608F0A9FC02460B4692469B4607F1C3
:102790001C03186808F02AFC41EC180B07F106032B
:1027A0001B88184608F032FC02460B4651EC180B09
:1027B00008F092FC02460B465046594608F0D8FAFB
:1027C00002460B464046494608F086FC02460B4648
:1027D0002046294608F0CEFA02460B46C7E93023C8
:1027E00007F10803186808F001FC04460D4607F1DC
:1027F0002003186808F0FAFB02460B4620462946DB
:1028000008F06AFC02460B4614461D4607F1100309
:10281000186808F0EBFB8046894607F11803186832
:1028200008F0E4FB02460B464046494608F054FCDB
:1028300002460B462046294608F09AFA02460B4605
:10284000104619464FF000024FF00003C4F2140383
:1028500008F042FC02460B4614461D4607F10603EB
:102860001B88184608F0C2FB8046894607F1100312
:10287000186808F0BBFB82468B4607F104031B88EF
:10288000184608F0C3FB02460B465046594608F06E
:1028900023FC02460B4692469B4607F10803186844
:1028A00008F0A4FB41EC180B07F106031B8818463F
:1028B00008F0ACFB02460B4651EC180B08F00CFC80
:1028C00002460B465046594608F052FA02460B465D
:1028D0004046494608F000FC02460B462046294681
:1028E00008F048FA02460B4614461D463B461B8834
:1028F000184608F07BFB8046894607F118031868E4
:1029000008F074FB82468B4607F106031B881846C5
:1029100008F07CFB02460B465046594608F0DCFBAB
:1029200002460B4692469B4607F12003186808F0C2
:102930005DFB41EC180B07F104031B88184608F0F7
:1029400065FB02460B4651EC180B08F0C5FB02462E
:102950000B465046594608F00BFA02460B464046D5
:10296000494608F0B9FB02460B462046294608F0C6
:1029700001FA02460B46C7E92E2307F11003186837
:1029800008F034FB04460D4607F11803186808F0F8
:102990002DFB8046894607F104031B88184608F082
:1029A00035FB02460B464046494608F095FB024679
:1029B0000B469046994607F11C03186808F016FB71
:1029C00082468B4607F106031B88184608F01EFB5B
:1029D00002460B465046594608F07EFB02460B461F
:1029E0004046494608F0C4F902460B4620462946AF
:1029F00008F072FB02460B4614461D4607F1080319
:102A0000186808F0F3FA8046894607F11803186839
:102A100008F0ECFA82468B4607F106031B8818463D
:102A200008F0F4FA02460B465046594608F054FBAB
:102A300002460B4692469B4607F12003186808F0B1
:102A4000D5FA41EC180B07F104031B88184608F06F
:102A5000DDFA02460B4651EC180B08F03DFB02462E
:102A60000B465046594608F083F902460B4640464D
:102A7000494608F031FB02460B462046294608F03D
:102A800079F902460B4614461D463B461B881846FC
:102A900008F0ACFA8046894607F12003186808F070
:102AA000A5FA82468B4607F11C03186808F09EFAC7
:102AB00002460B465046594608F00EFB02460B46AE
:102AC00092469B4607F11803186808F08FFA41EC0C
:102AD000180B07F11803186808F088FA02460B462D
:102AE00051EC180B08F0F8FA02460B4650465946CE
:102AF00008F03EF902460B464046494608F0ECFA1B
:102B000002460B462046294608F034F902460B4699
:102B1000C7E92C23D7E93601D7E9382308F006FCAA
:102B200002460B46C7E94423D7E93401D7E93823E5
:102B300008F0FCFB02460B46C7E94223D7E9320105
:102B4000D7E9382308F0F2FB02460B46C7E94023D9
:102B5000D7E93001D7E9382308F0E8FB02460B46F5
:102B6000C7E93E23D7E92E01D7E9382308F0DEFB79
:102B700002460B46C7E93C23D7E92C01D7E93823A5
:102B800008F0D4FB02460B46C7E93A23D7E94401D3
:102B90005FA3D3E9002308F09FFA02460B461046D4
:102BA000194608F033FD024640F26C13C2F20003EE
:102BB0001A60D7E9420156A3D3E9002308F08CFA42
:102BC00002460B461046194608F020FD024640F228
:102BD0007013C2F200031A60D7E940014CA3D3E995
:102BE000002308F079FA02460B461046194608F011
:102BF0000DFD024640F27413C2F200031A60D7E9D9
:102C00003E0143A3D3E9002308F066FA02460B46CF
:102C10001046194608F0FAFC024640F27813C2F258
:102C200000031A60D7E93C0139A3D3E9002308F077
:102C300053FA02460B461046194608F0E7FC0246D6
:102C400040F27C13C2F200031A60D7E93A0130A3C4
:102C5000D3E9002308F040FA02460B461046194615
:102C600008F0D4FC024640F28013C2F200031A605E
:102C70004FF6FF7000F0D6F940F20603C2F20003EF
:102C80001A8844F62513C2F29243A3FB0213D21A08
:102C90004FEA52029B184FEA93039BB21A464FEA3F
:102CA0004202D3189AB240F20803C2F20003198814
:102CB00048F6A333CBF62E23A3FB01034FEAD3033D
:102CC0009BB219464FEA8101CB184FEA43039BB2EE
:102CD000104619464DF65C02C0F600024FF00003A4
:102CE00000F0B0F84FF0190007F01EF94FF6FF7032
:102CF00000F098F940F2AC13C2F200034FF0010269
:102D00001A7007F5D477BD46BDEC028BBDE8B08FD5
:102D10000000000080842E4180B485B000AF0246E0
:102D20000B46FA80BB80FA8840F26C13C2F20003B3
:102D30001B6803FB02F2B98840F27013C2F2000371
:102D40001B6803FB01F3D21840F27413C2F20003B4
:102D50001B68D2184DF68363C4F21B3383FB021346
:102D60004FEAA3414FEAE273CB1A07EE103AF8EEAE
:102D7000C77AC7ED027AD7ED027AFCEEE77A17EE52
:102D8000903AFB81FA894EF660239A4202D94FF0BD
:102D90000003FB81FB89184607F11407BD4680BC80
:102DA000704700BF80B485B000AF02460B46FA8082
:102DB000BB80FA8840F27813C2F200031B6803FB61
:102DC00002F2B98840F27C13C2F200031B6803FBD5
:102DD00001F3D21840F28013C2F200031B68D2182C
:102DE0004DF68363C4F21B3383FB02134FEAA34106
:102DF0004FEAE273CB1A07EE103AF8EEC77AC7ED46
:102E0000027AD7ED027AFCEEE77A17EE903AFB8170
:102E1000FA894EF660239A4202D94FF00003FB81F3
:102E2000FB89184607F11407BD4680BC704700BFF8
:102E300080B400AF40F2D013C2F200031846BD4682
:102E400080BC704780B586B000AFBA600246FA8198
:102E50000A46BA81FB714FF000037B61BA8940F2E8
:102E60000403C2F200031B78DBB203F1FF3392FBD1
:102E7000F3F33B6140E0BB681A78B889F989FB79C4
:102E800000F0C2FABB681B78412B17D0BB681B78D7
:102E9000472B13D0BB681B784D2B0FD0BB681B781A
:102EA0004F2B0BD0BB681B78512B07D0BB681B780E
:102EB000582B03D0BB681B786D2B09D140F204035B
:102EC000C2F200031B78DBB2BA89D31ABB810BE0D4
:102ED00040F20403C2F200031B78DBB2BA89D31AB2
:102EE0009BB203F10103BB81BB6803F10103BB602B
:102EF0007B6903F101037B61BB681B78002B0CBF6E
:102F000000230123DAB279693B6999422CBF00237F
:102F10000123DBB21340DBB2002BACD107F1180761
:102F2000BD4680BD80B582B000AFF88079713A713E
:102F30007B80FA887B88D31A9BB203F101039BB292
:102F40004FF045001946FDF753FCFB884FF0460053
:102F50001946FDF74DFC7B799AB23B799BB2D31AA7
:102F60009BB203F101039BB29AB27B794FEA032330
:102F70009BB213439BB29BB24FF044001946FDF73E
:102F800037FCFA887B7910461946FDF7E5FB07F117
:102F90000807BD4680BD00BF80B582B000AF0346C4
:102FA000FB7140F29913C2F20003FA791A7040F2F1
:102FB0009913C2F200031B78002B06D14FF01100C9
:102FC00046F62001FDF714FC28E040F29913C2F206
:102FD00000031B78012B06D14FF0110046F60801C3
:102FE000FDF706FC1AE040F29913C2F200031B78C9
:102FF000022B06D14FF0110046F61001FDF7F8FB49
:103000000CE040F29913C2F200031B78032B05D1A8
:103010004FF0110046F63801FDF7EAFB07F108070B
:10302000BD4680BD80B582B000AF0346FB80FB8803
:103030001846FDF74DFC07F10807BD4680BD00BFEF
:1030400080B586B000AFBA600246FA810A46BA81FE
:10305000FB714FF00003FB754FF00003BB75FB895C
:10306000BB82BB89FB744FF00003FB7598E0BA8A02
:10307000FB7C10461946FDF76FFBFDF7E7FB4FF0B1
:103080000003BB7548E040F29813C2F200031B78BE
:10309000DBB2002B0DD1FB7D4FEA4303BA68D31896
:1030A0001B881A46BB7D42FA03F303F00103002B91
:1030B00016D040F29813C2F200031B78DBB2012B4A
:1030C0001DD1FB7D4FEA4303BA68D3181B881A460B
:1030D000BB7D4FF0800141FA03F31340002B0ED16A
:1030E000FB79002B08D140F2C813C2F200031B8801
:1030F0001846FDF7B5FB0BE0FDF7C2FB08E040F218
:10310000CA13C2F200031B889BB21846FDF7A8FB46
:10311000BB7D03F10103BB7540F20403C2F200035F
:103120001B78DBB2BA7D9A42ADD340F29913C2F25A
:1031300000031B78002B06D1FB89BB82FB7C03F1CB
:103140000103FB7428E040F29913C2F200031B78DC
:10315000012B06D1BB8A03F1FF33BB82BB89FB7411
:103160001AE040F29913C2F200031B78022B06D139
:10317000FB89BB82FB7C03F1FF33FB740CE040F264
:103180009913C2F200031B78032B05D1BB8A03F10C
:103190000103BB82BB89FB74FB7D03F10103FB755B
:1031A00040F20503C2F200031B78DBB2FA7D9A42BB
:1031B000FFF45DAF07F11807BD4680BD80B582B052
:1031C00000AF13460246FA800A46BA807B80F9882F
:1031D000BA887B88084611461A46FDF797FD07F125
:1031E0000807BD4680BD00BF90B585B002AFF8802E
:1031F000B9807A803B80BB88D9B23B88DBB2F88843
:103200007A883C8B0094FDF793FB07F10C07BD46D1
:1032100090BD00BF80B582B000AFF880B9807A80E1
:103220007B70BB88D9B2F8887A887B78FDF7C4FBBD
:1032300007F10807BD4680BD80B582B000AFF880B9
:10324000B9807A803B80BB88D9B23B88DBB2F888F2
:103250007A88FDF7F5FB07F10807BD4680BD00BF82
:1032600080B582B000AFF880B9807A803B80BB889F
:10327000D9B23B88DBB2F8887A88FDF7D5FC07F134
:103280000807BD4680BD00BF80B584B000AF3A607E
:103290000246FA800A467A713B71FB88FB817B7992
:1032A0007B7340F29913C2F200031B78012B14D1F7
:1032B000386808F0F1FA0346DAB240F20403C2F2C9
:1032C00000031B78DBB203FB02F3DAB27B79D3187D
:1032D000DBB203F1FF337B738CE040F29913C2F24F
:1032E00000031B78022B20D1386808F0D5FA03467A
:1032F0009AB240F20403C2F200031B78DBB203FB74
:1033000002F39BB2FA88D31A9BB203F10103FB814B
:1033100040F20503C2F200031B78DAB27B79D318BE
:10332000DBB203F1FF337B7364E040F29913C2F226
:1033300000031B78032B5DD140F20503C2F20003AA
:103340001B78DBB2FA88D31A9BB203F10103FB812D
:1033500050E07B7B99B23B681A78F8893B7900F0A2
:1033600053F840F29913C2F200031B78002B09D1E5
:1033700040F20403C2F200031B78DBB2FA89D31ACD
:10338000FB8132E040F29913C2F200031B78012B5B
:1033900009D140F20403C2F200031B78DBB27A7B4E
:1033A000D31A7B7321E040F29913C2F200031B7819
:1033B000022B0AD140F20403C2F200031B78DBB2F5
:1033C0001A46FB89D318FB810FE040F29913C2F231
:1033D00000031B78032B08D140F20403C2F2000360
:1033E0001B78DAB27B7BD3187B733B6803F1010354
:1033F0003B6000E000BF3B681B78002BA9D107F1C0
:103400001007BD4680BD00BF80B582B000AFF88018
:10341000B980FA70BB70FB78A3F12003FB7040F217
:103420009813C2F200031B78DBB2002B02D0012BF1
:1034300017D02DE040F29C03C2F200031A68F9781D
:1034400040F20503C2F200031B78DBB203FB01F379
:103450004FEA4303D218F888B988BB78FFF7F0FD2C
:1034600017E040F2B403C2F200031A68F97840F2A0
:103470000503C2F200031B78DBB203FB01F34FEA42
:103480004303D218F888B988BB78FFF7D9FD00E06C
:1034900000BF07F10807BD4680BD00BF80B582B000
:1034A00000AF0346FB8040F2C813C2F20003FA8863
:1034B0001A8040F2C813C2F200031B881846FDF7B9
:1034C000F5FB07F10807BD4680BD00BF80B483B09F
:1034D00000AF0346FB7140F29813C2F20003FA7981
:1034E0001A70FB79002B02D0012B0FD01DE040F2A7
:1034F0000403C2F200034FF010021A7040F20503F9
:10350000C2F200034FF018021A700FE040F20403F9
:10351000C2F200034FF008021A7040F20503C2F233
:1035200000034FF00C021A7000E000BF07F10C0717
:10353000BD4680BC704700BF80B582B000AF034677
:10354000FB8040F2F813C2F20003FA881A8040F2BE
:10355000F813C2F200031B881846FDF7B7FB07F10A
:103560000807BD4680BD00BF80B582B000AF0346EE
:10357000FB8040F2CA13C2F20003FA881A8040F2BC
:10358000CA13C2F200031B889BB21846FDF7AEFBBC
:1035900007F10807BD4680BD80B586B000AF7860F2
:1035A0004FF000033B614FF00003FB607B6803F1C9
:1035B000020307F10C021046194600F0F1F87B688F
:1035C00003F10A0307F110021046194600F0E8F86B
:1035D0004FF011004FF4D041FDF70AF9FDF736F92D
:1035E00017E03B697A68D3181B781A463B6903F1E8
:1035F00001037968CB181B784FEA03239BB2D318D9
:10360000FB82FB8A1846FDF72BF93B6903F10203A5
:103610003B613A69FB689A42E3D340F2D013C2F2AD
:10362000000393F82430002B0FD140F2D013C2F2E4
:1036300000031A6840F2D013C2F200031B8910463F
:1036400019464FF0010200F0DFF84FF0110046F686
:103650002001FDF7CDF807F11807BD4680BD00BF7A
:1036600080B582B000AF0346FB71FB79002B02D11D
:10367000FDF712F904E0FB79012B01D1FDF712F9F6
:1036800007F10807BD4680BD80B500AFFCF770FFAD
:1036900080BD00BF80B582B000AFF880B9807A806D
:1036A0007B707B7803F00903002B08D0BB88DBB26A
:1036B000FA8810461946FDF74FF8FDF7C7F87B88E2
:1036C0001846FDF7CDF840F2D013C2F2000393F88C
:1036D0002430002B1CD17B7803F00C03002B17D077
:1036E00040F2D013C2F2000393F82430002B0FD124
:1036F00040F2D013C2F200031A6840F2D013C2F2B3
:1037000000031B89104619464FF0010200F07CF8B7
:1037100007F10807BD4680BD80B584B000AF024602
:103720000B46FA80BB804FF00003FB814FF0000393
:10373000BB814FF000037B81BB88DBB2FA88104667
:103740001946FDF709F840F2D013C2F2000393F8CE
:103750002430002B06D14FF03400FDF761F803460A
:10376000FB8103E000F05EF80346FB81FB894FEA32
:10377000C323BB81FB894FEAD3237B81FB8903F4FD
:10378000FC63FB81BA897B8913439AB2FB8913439B
:10379000FB81FB89184607F11007BD4680BD00BFBD
:1037A00080B483B000AF786039607B684FF000026E
:1037B0001A603B681B781A467B681A607B681A6837
:1037C0003B6803F101031B784FEA0323D2187B689F
:1037D0001A607B681A683B6803F102031B784FEAA2
:1037E0000343D2187B681A607B681A683B6803F150
:1037F00003031B784FEA0363D2187B681A6007F152
:103800000C07BD4680BC704780B483B000AF7860C1
:1038100013460A467A807B7007F10C07BD4680BCD0
:10382000704700BF80B582B000AF4FF00003FB804F
:1038300040F2D013C2F2000393F82430002B05D1DC
:103840004FF03400FCF7ECFF0346FB80FB889BB293
:10385000184607F10807BD4680BD00BF80B582B09D
:1038600000AF44F21833C0F601037B6040F200035E
:10387000C2F200033B600BE07B681A683B681A6089
:103880003B6803F104033B607B6803F104037B6046
:103890003A6840F26413C2F200039A42ECD30B4838
:1038A0000B494FF000028842B8BF40F8042BFFF6E6
:1038B000FAAFDFF82000016841F47001016001F007
:1038C00055F907F10807BD4680BD000064010020DE
:1038D000DC03002088ED00E080B400AFFEE700BF0D
:1038E00080B582B000AF07F0FFF878607B684FF4D6
:1038F00000125A607B684FF400721A817A684FF4A4
:103900008063C4F20203D3607B684FF002021A6145
:103910007B684FF009029A827B684FF004029A613B
:103920007B684FF480729A837A684FF48063C4F2A4
:10393000020313627B684FF002025A627B684FF009
:1039400008021A857B684FF00402DA627B684FF444
:1039500000125A607B684FF00D021A877B684FF0A7
:103960000402DA637B684FF002021A707B684FF042
:103970000D025A807B684FF0280283F830207B6864
:103980004FF400525A637A684FF40063C4F20203A2
:1039900013647B684FF40052A3F844207B684FF017
:1039A00082029A647A684FF4A843C4F20003136554
:1039B00007F10807BD4680BD80B582B000AFFFF7B4
:1039C00037FA78607B684FF0010283F824207B6827
:1039D0004FF00102DA6107F10807BD4680BD00BF64
:1039E00080B500AFFFF77CFFFFF7E6FF80BD00BFAB
:1039F00080B588B000AF02460B46FA71BB71FA7908
:103A00004DF68C03C0F6000353F8223018464FF0F1
:103A1000010101F0F5F94FF480404FF0010101F090
:103A20006DFA4FF000033B774FF00003FB77FA7914
:103A30004DF68803C0F6000333F81230BB61FA7903
:103A400040F22003C2F2000353F8222007F11803CA
:103A50001046194606F0A0FCBB79012B3AD1FA7941
:103A60004DF69403C0F600039A5CF9794DF698037D
:103A7000C0F600035B5C10461946FCF785FBFA793B
:103A80004DF69003C0F6000333F812303B614FF05F
:103A900000033B754FF008037B754FF00103BB75C6
:103AA00007F11003184606F0ABFEFA794DF69C03B9
:103AB000C0F600039B5C3B734FF00F037B734FF02A
:103AC0000F03BB734FF00103FB7307F10C031846A0
:103AD00006F082FF07F12007BD4680BD80B582B0A9
:103AE00000AF0346FB71FA7940F22003C2F20003F3
:103AF00053F82220F9794DF68803C0F6000333F815
:103B000011301046194606F0E9FC0346184607F145
:103B10000807BD4680BD00BF80B500AF00F0DCFEE9
:103B200000F036FF4FF0820000F07EF80346002BD5
:103B300002D04FF004030FE04FF0820000F098F83D
:103B40004FF082004FF007014FF0010200F0D6F86D
:103B500000F068F94FF00003184680BD80B582B0D0
:103B600000AF78604FF004004FF0000100F01CFA45
:103B70007B6803F00103002B13D04FF082004FF05D
:103B8000010100F0EFF84FF082004FF003014FF019
:103B9000010200F013F94FF082004FF00D0100F028
:103BA00045FB00F019FF4FF00003184607F1080726
:103BB000BD4680BD80B584B000AF02460B46FA71A9
:103BC000BB714FF00003FB73FB7918464FF00B01FC
:103BD00000F02CFB0346FB73FB7BDAB2BB7913408E
:103BE000DBB2002B02D04FF0010301E04FF00003E5
:103BF000184607F11007BD4680BD00BF80B582B0F2
:103C000000AF02460B46FA71BB71FA79BB791046D8
:103C10004FF00B011A4600F0F3F94FF0000318467D
:103C200007F10807BD4680BD80B582B000AF0346EE
:103C3000FB71FB79184600F03BF803461A4640F644
:103C400011039A420CD040F23C03C2F200031B88DD
:103C5000002B02D14FF0020304E04FF0010301E01A
:103C60004FF00003184607F10807BD4680BD00BFAE
:103C700080B582B000AF0346FB71FB7918464FF068
:103C800003014FF0020200F0BBF94FF0020000F018
:103C9000F1FEFB7918464FF003014FF0000200F0EF
:103CA000AFF94FF00003184607F10807BD4680BD85
:103CB00080B584B000AF0346FB714FF00003FB8179
:103CC000FB7918464FF0000100F0B0FA0346FB8183
:103CD000FB894FEA0323FB81FB7918464FF0010172
:103CE00000F0A4FA03461A46FB891343FB81FB89C3
:103CF000184607F11007BD4680BD00BF80B584B0EF
:103D000000AF13460246FA710A46BA717B714FF052
:103D10000003FB73FB7918464FF0040100F086FAAC
:103D20000346FB737B79002B08D0BB796FEA030352
:103D3000DAB2FB7B1340DBB2FB7303E0FA7BBB79A7
:103D40001343FB73FA79FB7B10464FF004011A46CC
:103D500000F056F94FF00003184607F11007BD4672
:103D600080BD00BF80B584B000AF02460B46FA713B
:103D7000BB714FF00003FB73FB7918464FF009014C
:103D800000F054FABB79002B04D0FB7B43F0010315
:103D9000FB7303E0FB7B23F00103FB73FA79FB7BEE
:103DA00010464FF009011A4600F02AF94FF00003BF
:103DB000184607F11007BD4680BD00BF80B584B02E
:103DC00000AF13460246FA710A46BA717B714FF092
:103DD0000003FB73FB7918464FF00A0100F026FA46
:103DE0000346FB737B79002B04D0FA7BBB7913432A
:103DF000FB7307E0BB796FEA0303DAB2FB7B134086
:103E0000DBB2FB73FA79FB7B10464FF00A011A46CE
:103E100000F0F6F84FF00003184607F11007BD4612
:103E200080BD00BF80B582B000AF4FF00003FB71D2
:103E30004FF082004FF0040100F0F8F90346FB71E7
:103E4000FB7923F00303FB71FB794FF082004FF005
:103E500004011A4600F0D4F84FF082004FF00A0136
:103E600000F0E4F90346FB71FB7943F00303FB71B7
:103E7000FB794FF082004FF00A011A4600F0C0F8BB
:103E80004FF082004FF020014FF0490200F0B8F8E7
:103E90004FF0020000F0EEFD4FF082004FF02101E4
:103EA0004FF0010200F0ACF84FF082004FF0170124
:103EB00000F0BCF90346FB71FB7923F01E03FB7194
:103EC000FB794FF082004FF017011A4600F098F886
:103ED0004FF082004FF041014FF09A0200F090F84D
:103EE0004FF082004FF04A014FF0010200F088F8D5
:103EF0004FF082004FF04B014FF0010200F080F8CC
:103F00004FF082004FF04B014FF0000200F078F8C4
:103F10004FF082004FF056014FF0010200F070F8B0
:103F20004FF082004FF058014FF0010200F068F8A6
:103F30004FF082004FF040014FF0010200F060F8B6
:103F40004FF082004FF00B014FF0FF0200F058F8E5
:103F500040F2FC13C2F200034FF00002DA8040F29C
:103F6000FC13C2F20003DA8840F2FC13C2F2000331
:103F70009A8040F2FC13C2F200039A8840F2FC13CC
:103F8000C2F200035A8040F2FC13C2F200035A88C6
:103F900040F2FC13C2F200031A804FF000031846EF
:103FA00007F10807BD4680BD80B584B000AF02466A
:103FB0000B46FA71BB714FF00003FB734FF08200A8
:103FC0004FF0090100F032F90346FB73FB7B23F04D
:103FD0000603FB73FA79BB791343DAB2FB7B134315
:103FE000FB73FB7B4FF082004FF009011A4600F093
:103FF00007F84FF00003184607F11007BD4680BDD3
:1040000080B483B000AF13460246FA710A46BA7113
:104010007B714FF4A843C4F200034FF4A842C4F2EA
:104020000002128892B242F0010292B21A804FF45A
:10403000A843C4F200034FF4A842C4F2000212885D
:1040400092B242F4807292B21A8040F23C03C2F201
:1040500000034FF440521A8016E040F23C03C2F2D3
:1040600000031B88002B14BF00220122D2B203F1EF
:10407000FF3399B240F23C03C2F200031980002AD8
:1040800002D04FF00203CBE04FF4A843C4F2000388
:104090009B8A9BB203F00103002BDED04FF4A843B0
:1040A000C4F20003FA7992B21A8240F23C03C2F2DF
:1040B00000034FF440521A8016E040F23C03C2F273
:1040C00000031B88002B14BF00220122D2B203F18F
:1040D000FF3399B240F23C03C2F200031980002A78
:1040E00002D04FF002039BE04FF4A843C4F2000358
:1040F0009B8A9BB203F00203002BDED04FF4A8434F
:10410000C4F200039B8A4FF4A843C4F200031B8B44
:104110004FF4A843C4F20003BA7992B21A8240F273
:104120003C03C2F200034FF440521A8016E040F202
:104130003C03C2F200031B88002B14BF00220122A3
:10414000D2B203F1FF3399B240F23C03C2F2000352
:104150001980002A02D04FF0020361E04FF4A84317
:10416000C4F200039B8A9BB203F08003002BDED0D5
:104170004FF4A843C4F200037A7992B21A8240F253
:104180003C03C2F200034FF440521A8016E040F2A2
:104190003C03C2F200031B88002B14BF0022012243
:1041A000D2B203F1FF3399B240F23C03C2F20003F2
:1041B0001980002A02D04FF0020331E04FF4A843E7
:1041C000C4F200039B8A9BB203F08003002BDED075
:1041D0004FF4A843C4F200039B8A9BB203F004038C
:1041E000002BD4D04FF4A843C4F200034FF4A842EC
:1041F000C4F20002128892B242F4007292B21A80A3
:104200004FF4A843C4F200034FF4A842C4F20002E2
:10421000128892B222F0010292B21A804FF000038B
:10422000184607F10C07BD4680BC704780B485B0C6
:1042300000AF02460B46FA71BB714FF4A843C4F2BB
:1042400000034FF4A842C4F20002128892B242F076
:10425000010292B21A804FF4A843C4F200034FF453
:10426000A842C4F20002128892B242F4807292B262
:104270001A8040F23C03C2F200034FF440521A800D
:1042800016E040F23C03C2F200031B88002B14BF6F
:1042900000220122D2B203F1FF3399B240F23C0373
:1042A000C2F200031980002A02D04FF0000341E15E
:1042B0004FF4A843C4F200039B8A9BB203F00103AE
:1042C000002BDED04FF4A843C4F20003FA7992B277
:1042D0001A8240F23C03C2F200034FF440521A80AB
:1042E00016E040F23C03C2F200031B88002B14BF0F
:1042F00000220122D2B203F1FF3399B240F23C0313
:10430000C2F200031980002A02D04FF0000311E12D
:104310004FF4A843C4F200039B8A9BB203F002034C
:10432000002BDED04FF4A843C4F200039B8A4FF465
:10433000A843C4F200031B8B4FF4A843C4F200034C
:10434000BA7992B21A8240F23C03C2F200034FF4EF
:1043500040521A8016E040F23C03C2F200031B8870
:10436000002B14BF00220122D2B203F1FF3399B215
:1043700040F23C03C2F200031980002A02D04FF041
:104380000003D7E04FF4A843C4F200039B8A9BB21A
:1043900003F08003002BDED04FF4A843C4F20003E7
:1043A0004FF4A842C4F20002128892B242F4807222
:1043B00092B21A8040F23C03C2F200034FF4405222
:1043C0001A8016E040F23C03C2F200031B88002B67
:1043D00014BF00220122D2B203F1FF3399B240F29E
:1043E0003C03C2F200031980002A02D04FF0000300
:1043F000A0E04FF4A843C4F200039B8A9BB203F0F1
:104400000103002BDED04FF4A843C4F20003FA7975
:1044100042F00102D2B21A8240F23C03C2F200031F
:104420004FF440521A8016E040F23C03C2F20003FF
:104430001B88002B14BF00220122D2B203F1FF33EC
:1044400099B240F23C03C2F200031980002A02D064
:104450004FF000036EE04FF4A843C4F200039B8AC0
:104460009BB203F00203002BDED04FF4A843C4F24A
:1044700000034FF4A842C4F20002128892B222F460
:10448000806292B21A804FF4A843C4F200039B8A60
:104490004FF4A843C4F200031B8B40F23C03C2F26A
:1044A00000034FF440521A8016E040F23C03C2F27F
:1044B00000031B88002B14BF00220122D2B203F19B
:1044C000FF3399B240F23C03C2F200031980002A84
:1044D00002D04FF000032DE04FF4A843C4F20003D4
:1044E0009B8A9BB203F04003002BDED04FF4A8431D
:1044F000C4F200031B8A9BB2FB734FF4A843C4F2BF
:1045000000034FF4A842C4F20002128892B242F4AF
:10451000007292B21A804FF4A843C4F200034FF421
:10452000A842C4F20002128892B222F0010292B2B2
:104530001A80FB7B184607F11407BD4680BC704704
:1045400080B485B000AF02460B46FA71BB714FF4E0
:10455000A843C4F200034FF4A842C4F20002128838
:1045600092B242F0010292B21A804FF4A843C4F210
:1045700000034FF4A842C4F20002128892B242F43F
:10458000807292B21A8040F23C03C2F200034FF4F0
:1045900040521A8016E040F23C03C2F200031B882E
:1045A000002B14BF00220122D2B203F1FF3399B2D3
:1045B00040F23C03C2F200031980002A02D04FF0FF
:1045C000000383E14FF4A843C4F200039B8A9BB22B
:1045D00003F00103002BDED04FF4A843C4F2000324
:1045E000FA7992B21A8240F23C03C2F200034FF40D
:1045F00040521A8016E040F23C03C2F200031B88CE
:10460000002B14BF00220122D2B203F1FF3399B272
:1046100040F23C03C2F200031980002A02D04FF09E
:10462000000353E14FF4A843C4F200039B8A9BB2FA
:1046300003F00203002BDED04FF4A843C4F20003C2
:104640009B8A4FF4A843C4F200031B8B4FF4A8438A
:10465000C4F20003BA7992B21A8240F23C03C2F269
:1046600000034FF440521A8016E040F23C03C2F2BD
:1046700000031B88002B14BF00220122D2B203F1D9
:10468000FF3399B240F23C03C2F200031980002AC2
:1046900002D04FF0000319E14FF4A843C4F2000325
:1046A0009B8A9BB203F08003002BDED04FF4A8431B
:1046B000C4F200034FF4A842C4F20002128892B27E
:1046C00042F4807292B21A8040F23C03C2F20003BC
:1046D0004FF440521A8016E040F23C03C2F200034D
:1046E0001B88002B14BF00220122D2B203F1FF333A
:1046F00099B240F23C03C2F200031980002A02D0B2
:104700004FF00003E2E04FF4A843C4F200039B8A99
:104710009BB203F00103002BDED04FF4A843C4F298
:104720000003FA7942F00102D2B21A8240F23C034D
:10473000C2F200034FF440521A8016E040F23C03EC
:10474000C2F200031B88002B14BF00220122D2B248
:1047500003F1FF3399B240F23C03C2F20003198027
:10476000002A02D04FF00003B0E04FF4A843C4F297
:1047700000039B8A9BB203F00203002BDED04FF4B0
:10478000A843C4F200034FF4A842C4F20002128806
:1047900092B242F4806292B21A804FF4A843C4F2FB
:1047A00000039B8A4FF4A843C4F200031B8B40F222
:1047B0003C03C2F200034FF440521A8016E040F26C
:1047C0003C03C2F200031B88002B14BF002201220D
:1047D000D2B203F1FF3399B240F23C03C2F20003BC
:1047E0001980002A02D04FF000036FE04FF4A84375
:1047F000C4F200039B8A9BB203F04003002BDED07F
:104800004FF4A843C4F200034FF4A842C4F20002DC
:10481000128892B222F4806292B21A804FF4A843B6
:10482000C4F200031B8A9BB24FEA0323FB8140F2D0
:104830003C03C2F200034FF440521A8016E040F2EB
:104840003C03C2F200031B88002B14BF002201228C
:10485000D2B203F1FF3399B240F23C03C2F200033B
:104860001980002A02D04FF000032FE04FF4A84334
:10487000C4F200039B8A9BB203F04003002BDED0FE
:104880004FF4A843C4F200031B8A9AB2FB89D318E1
:10489000FB814FF4A843C4F200034FF4A842C4F2D2
:1048A0000002128892B242F4007292B21A804FF45F
:1048B000A843C4F200034FF4A842C4F200021288D5
:1048C00092B222F0010292B21A80FB89184607F1D7
:1048D0001407BD4680BC704780B582B000AF4FF46E
:1048E00000104FF0010100F0DFFA4FF002004FF02E
:1048F000010100F085FA4FF480404FF0010100F013
:10490000FDFA4FF400104FF0010100F021FB4FF4CD
:1049100000104FF0000100F01BFB4FF480733B6070
:104920004FF002033B714FF002037B714FF0010324
:10493000BB714FF00003FB713B464FF48060C4F243
:104940000200194605F028FD4FF400733B603B461A
:104950004FF48060C4F20200194605F01DFD4FF4CB
:104960008060C4F202004FF008014FF0040205F02D
:10497000EFFD4FF48060C4F202004FF009014FF0E8
:10498000040205F0E5FD07F10807BD4680BD00BF44
:1049900080B584B000AF4FF00003BB804BF6FF73CF
:1049A000FB804FF000033B814FF480637B814FF429
:1049B0008043BB8148F2A063C0F201033B603B46E9
:1049C0004FF4A840C4F20000194605F043FE07F179
:1049D0001007BD4680BD00BF80B586B000AF4FF068
:1049E00004004FF0010100F00BFA4FF480404FF04B
:1049F000010100F083FA4FF400533B614FF00003D4
:104A00003B754FF00003FB7507F110034FF4006096
:104A1000C4F20200194605F0BFFC4FF002004FF04F
:104A20000D01FBF7B1FB4FF400537B604FF0000327
:104A30003B724FF010037B724FF00103BB7207F122
:104A40000403184605F0DCFE4FF028033B734FF0DB
:104A50000F037B734FF00F03BB734FF00103FB7326
:104A600007F10C03184605F0B7FF07F11807BD461C
:104A700080BD00BF80B485B000AF78604FF0000308
:104A8000FB607A6848F2A063C0F2010303FB02F303
:104A9000FB6003E0FB6803F1FF33FB60FB68002B66
:104AA000F8D107F11407BD4680BC704780B483B0CD
:104AB00000AF03463960FB7197F90730002B10DA1D
:104AC0004FF46D43CEF20003FA7902F00F02A2F127
:104AD00004013A68D2B24FEA0212D2B25B181A76D7
:104AE0000DE04FF46143CEF2000397F907103A68E6
:104AF000D2B24FEA0212D2B25B1883F8002307F158
:104B00000C07BD4680BC704780B582B000AF7860AE
:104B10007A686FF07F439A4202D94FF001031FE099
:104B20004EF21003CEF200037A6822F07F4202F1C7
:104B3000FF325A604FF0FF304FF00F01FFF7B6FF22
:104B40004EF21003CEF200034FF000029A604EF2D4
:104B50001003CEF200034FF007021A604FF000037B
:104B6000184607F10807BD4680BD00BF80B584B078
:104B700000AF4FF000604FF0000105F09FFF4FF4D1
:104B8000A06005F015FF3B46184600F053F83A6860
:104B900048F21F53C5F2EB13A3FB02134FEA531362
:104BA0001846FFF7B1FF0346002B00D0FEE74FF099
:104BB000FF304FF00B01FFF779FFFEF711FFFEF713
:104BC00063FD4FF6FF70FEF72DFA4FF00100FEF780
:104BD0007DFC4FF00000FEF7C7FC4FF496704FF0DD
:104BE00064014DF6D002C0F600024FF00103FEF75B
:104BF0004BFB4FF000004FF00001FEF7F9FE00BF45
:104C00004FF00000FEF76AFF0346002BF8D000F0DB
:104C100005F805F0DFFA04F08FFFFCE780B500AF80
:104C200005F0A0FFFCF790F94FF00100FEF796FFAA
:104C300080BD00BF80B489B000AF78604FF0000342
:104C4000BB614FF000037B614FF00003FB614FF04D
:104C500002033B614FF00003FB604FF00203BB60B7
:104C60004FF46053C4F202039B6803F00C03BB6172
:104C7000BB69042B0AD0082B0FD0002B60D17A68B7
:104C80004FF41053C0F2F403136060E07A684FF4FD
:104C90009053C0F27A03136059E04FF46053C4F2AA
:104CA00002035B6803F480034FEA9353FB604FF405
:104CB0006053C4F202035B6803F03F03BB60FB6810
:104CC000002B14D04FF49053C0F27A03BA68B3FBB0
:104CD000F2F24FF46053C4F20203596847F6C0730E
:104CE0000B404FEA931303FB02F3FB6113E04FF415
:104CF0001053C0F2F403BA68B3FBF2F24FF46053FE
:104D0000C4F20203596847F6C0730B404FEA93138D
:104D100003FB02F3FB614FF46053C4F202035B68D0
:104D200003F440334FEA134303F101034FEA430313
:104D30003B61FA693B69B2FBF3F27B681A6006E0FB
:104D40007A684FF41053C0F2F403136000BF4FF4BD
:104D50006053C4F202039B6803F0F003BB61BB69BC
:104D60004FEA1313BB6140F24003C2F20003BA6979
:104D70009B181B78DBB27B617B681A687B6922FA1F
:104D800003F27B685A604FF46053C4F202039B68DD
:104D900003F4E053BB61BB694FEA9323BB6140F26C
:104DA0004003C2F20003BA699B181B78DBB27B6137
:104DB0007B685A687B6922FA03F27B689A604FF439
:104DC0006053C4F202039B6803F46043BB61BB6998
:104DD0004FEA5333BB6140F24003C2F20003BA69A9
:104DE0009B181B78DBB27B617B685A687B6922FA6F
:104DF00003F27B68DA6007F12407BD4680BC704788
:104E000080B483B000AF78600B46FB70FB78002B5A
:104E10000CD04FF46053C4F202034FF46052C4F25A
:104E20000202116B7A680A431A630DE04FF4605373
:104E3000C4F202034FF46052C4F20202116B7A68AA
:104E40006FEA02020A401A6307F10C07BD4680BCF4
:104E5000704700BF80B483B000AF78600B46FB7032
:104E6000FB78002B0CD04FF46053C4F202034FF4D4
:104E70006052C4F20202916B7A680A439A630DE0B1
:104E80004FF46053C4F202034FF46052C4F20202C2
:104E9000916B7A686FEA02020A409A6307F10C0785
:104EA000BD4680BC704700BF80B483B000AF78605F
:104EB0000B46FB70FB78002B0CD04FF46053C4F210
:104EC00002034FF46052C4F20202116C7A680A4382
:104ED0001A640DE04FF46053C4F202034FF46052C1
:104EE000C4F20202116C7A686FEA02020A401A6484
:104EF00007F10C07BD4680BC704700BF80B483B08B
:104F000000AF78600B46FB70FB78002B0CD04FF4A1
:104F10006053C4F202034FF46052C4F20202516CB7
:104F20007A680A435A640DE04FF46053C4F20203F6
:104F30004FF46052C4F20202516C7A686FEA0202C6
:104F40000A405A6407F10C07BD4680BC704700BF99
:104F500080B483B000AF78600B46FB70FB78002B09
:104F60000CD04FF46053C4F202034FF46052C4F209
:104F70000202116A7A680A431A620DE04FF4605324
:104F8000C4F202034FF46052C4F20202116A7A685A
:104F90006FEA02020A401A6207F10C07BD4680BCA4
:104FA000704700BF80B586B000AF13460246FA8056
:104FB0000A46BA80FB704FF00003BB754FF0000348
:104FC0003B7540F20823C2F200031B681B68BB60FC
:104FD000FB7803F00103002B64D040F20823C2F2F7
:104FE00000031B681B6803F103033B6140F20823C5
:104FF000C2F200031B68DB68FB604FF00003BB7567
:105000004BE04FF000037B754FF00003FB753BE076
:105010007B7D002B09D13B691B783B753B6903F114
:1050200001033B614FF080037B753A7D7B7D13402C
:10503000DBB2002B20D040F20823C2F200031B6831
:105040009A88FB7D9BB2D31899B240F20823C2F232
:1050500000031B68DA88BB7D9BB2D3189AB2FB6849
:105060001B88F86800F10200F860084611461A46ED
:105070004FF00803FEF70EFB7B7D4FEA53037B7571
:10508000FB7D03F10103FB75BB681B78FA7D9A4237
:10509000BED3BB7D03F10103BB75BB685B78BA7DF2
:1050A0009A42AED3FB7803F00203002B59D040F2B2
:1050B0000823C2F200031B681B6803F103033B6172
:1050C00040F20823C2F200031B68DB68FB604FF06C
:1050D0000003BB7540E04FF000037B754FF0000309
:1050E000FB7530E07B7D002B09D13B691B783B755C
:1050F0003B6903F101033B614FF080037B753A7D0F
:105100007B7D1340DBB2002B15D0FB7D9AB2FB8870
:10511000D3189AB2BB7D99B2BB88CB189BB210460C
:105120001946FEF7F9FA03461A46FB681A80FB682F
:1051300003F10203FB607B7D4FEA53037B75FB7D2C
:1051400003F10103FB75BB681B78FA7D9A42C9D352
:10515000BB7D03F10103BB75BB685B78BA7D9A42E6
:10516000B9D3FB7803F00403002B02D1FB78082BA2
:1051700053D140F20823C2F200031B681B6803F1FD
:1051800003033B614FF00003BB7541E04FF00003A8
:105190007B754FF00003FB7531E07B7D002B09D15F
:1051A0003B691B783B753B6903F101033B614FF0A1
:1051B00080037B753A7D7B7D1340DBB2002B16D0DC
:1051C000FB7D9AB2FB88D31899B2BB7D9AB2BB889B
:1051D000D3189AB240F20823C2F200031B681B8A5C
:1051E000084611461A464FF00803FEF753FA7B7D36
:1051F0004FEA53037B75FB7D03F10103FB75BB682D
:105200001B78FA7D9A42C8D3BB7D03F10103BB75BD
:10521000BB685B78BA7D9A42B8D340F20823C2F2E9
:1052200000031B68FA889A8040F20823C2F2000348
:105230001B68BA88DA8007F11807BD4680BD00BF39
:1052400080B400AFBD4680BC704700BF80B400AFE3
:10525000FEE700BF80B400AFFEE700BF80B400AF40
:10526000FEE700BF80B400AFFEE700BF80B400AF30
:10527000BD4680BC704700BF80B400AFBD4680BC57
:10528000704700BF80B400AFBD4680BC704700BF10
:1052900080B500AF04F060FE80BD00BF80B500AFF8
:1052A00005F02CFC80BD00BF80B500AF40F2B423F8
:1052B000C2F200031B6818464FF0000104F050FFD3
:1052C00080BD00BF80B500AF40F2B423C2F200033E
:1052D0001B6818464FF01F0104F042FF80BD00BF5D
:1052E00080B500AF40F2B423C2F200031B68184639
:1052F00004F04AFE80BD00BF80B500AF40F2B42389
:10530000C2F200031B68184647F6FF7104F028FF3D
:1053100080BD00BF80B500AF40F2B423C2F20003ED
:105320001B6818464FF4FC6104F01AFF80BD00BFF3
:1053300080B500AF40F2B423C2F200031B681846E8
:105340004FF61F0104F00CFF80BD00BF80B500AF19
:1053500040F2B423C2F200031B6818464FF47841B0
:1053600004F0FEFE80BD00BF80B500AF40F2B42364
:10537000C2F200031B6818464FF6FF7104F0F0FEFE
:1053800080BD00BF80B500AF40F2B423C2F200037D
:105390001B6818464FF6E07104F0E2FE80BD00BFC6
:1053A00080B58AB000AF4FF49A704DF6F401C0F6A4
:1053B000000145F2E122C0F6000200F08DFE7862A5
:1053C0004FF496704FF0000145F2A922C0F600029A
:1053D00000F0CEFE38624FF498704FF01F0145F296
:1053E000C522C0F6000200F0C3FEF86140F23110A1
:1053F00047F6FF7145F2F922C0F6000200F0B8FE50
:10540000B86140F22F104FF4FC6145F21532C0F63E
:10541000000200F0ADFE78614FF499704FF61F0165
:1054200045F23132C0F6000200F0A2FE38614FF4BE
:1054300097704FF4784145F24D32C0F6000200F00B
:1054400097FEF86040F22D104FF6FF7145F2693279
:10545000C0F6000200F08CFEB86040F233104FF648
:10546000E07145F28532C0F6000200F081FE7860FE
:1054700040F235104FF49F714FF0C8024FF0000317
:1054800004F02CFE024640F2B423C2F200031A607C
:1054900040F21020C2F2000000F08AFD4FF49F702D
:1054A0004FF001013A6A40F21023C2F2000300F00B
:1054B000C7FA4FF490704FF00101BA6840F2102320
:1054C000C2F2000300F0BCFA4FF481704FF001010A
:1054D000FA6840F21023C2F2000300F0B1FA4FF074
:1054E000E4004FF001017A6940F21023C2F2000398
:1054F00000F0A6FA4FF0C6004FF00101FA6940F241
:105500001023C2F2000300F09BFA4FF0A8004FF006
:1055100001013A6940F21023C2F2000300F090FA50
:105520004FF08A004FF00101BA6940F21023C2F235
:10553000000300F085FA4FF06C004FF001017A682B
:1055400040F21023C2F2000300F07AFA4FF04E004E
:105550004FF002017A6A40F21023C2F2000300F019
:105560006FFA40F2B423C2F200031B684FF49F703D
:105570004FF023011A4640F21023C2F2000300F05C
:105580005FFA07F12807BD4680BD00BF80B500AFB8
:1055900040F28033C2F200031B68002B0ED040F2B1
:1055A0008033C2F200031B68DA6940F28033C2F232
:1055B00000031B6818464FF0000190474FF6FF703C
:1055C000FDF730FD4FF00000FDF7CEFF40F2102355
:1055D000C2F20003DB6940F21020C2F200004FF07B
:1055E0000101984740F28033C2F2000340F21022DA
:1055F000C2F200021A6080BD80B584B000AFF880AE
:1056000079717A803B804FF00203FB60FA887B88D7
:10561000D31A99B27B799AB27B88D31A9AB27B88D3
:10562000084611461A46FDF7C9FDFA887B88D31A49
:1056300099B27B799AB27B88D31A9AB27B8803F1AC
:10564000FF339BB2084611461A46FDF7B7FD3B886B
:105650001846FDF771FF16E0FA887B88D31A99B2D5
:105660007B799AB27B88D31A9AB2FB689BB278880E
:10567000C31A9BB2084611461A46FDF79FFDFB6808
:1056800003F10103FB607A88FB689A42E4D807F1D2
:105690001007BD4680BD00BF90B589B002AFF8804D
:1056A000B9807A803B804FF000033B744FF00003D9
:1056B000FB814FF00003FB824FF00003BB824FF0F1
:1056C0000003BB814FF000037B814FF000037B821E
:1056D0004FF000037B74BA883B889A420ED1FA8857
:1056E0007B889A420AD1B988FA883B8D08461146D0
:1056F0001A464FF00803FDF7CDFFF6E0FA887B88E5
:105700009A4235D1BA883B889A4205D93B88FB81B9
:10571000BB883B80FB89BB80B988FA883B8D0846F3
:1057200011461A464FF00103FDF7B4FFBB8803F1A1
:105730000103FB820DE0B988FA883B8D08461146CB
:105740001A464FF00203FDF7A5FFFB8A03F10103A0
:10575000FB82FA8A3B889A42EDD33988FA883B8DDE
:10576000084611461A464FF00403FDF793FFBCE0CC
:10577000BA883B889A421ED1FA887B889A4205D91A
:105780007B88FB81FB887B80FB89FB803A88BB8818
:10579000D31A9BB2A3F102039AB27988FB88CB1A81
:1057A0009BB203F1FF339BB23888F9883C8D00949B
:1057B000FDF71AFD99E0FA887B889A4203D9FA88A6
:1057C0007B88D21A02E07A88FB88D21AB9883B8893
:1057D000994203D9B9883B88CB1A02E03988BB8843
:1057E000CB1A9A42D4BF00230123DBB23B743B7C2B
:1057F000002B0BD0FB88FB81BB88FB80FB89BB8027
:105800007B88FB813B887B80FB893B80BA883B8817
:105810009A420BD9FB88FB817B88FB80FB897B80CC
:105820003B88FB81BB883B80FB89BB803A88BB8877
:10583000D31ABB81FA887B889A4204D9FA887B887C
:10584000D31A9BB203E07A88FB88D31A9BB27B8180
:10585000BB896FEA03034FEAD372D3184FEA63039D
:105860007B82FB88BB82FA887B889A4203D24FF006
:1058700001037B7402E04FF0FF037B74BB88FB8263
:105880002FE03B7C002B0AD0B98AFA8A3B8D084670
:1058900011461A464FF00803FDF7FCFE09E0B98AED
:1058A000FA8A3B8D084611461A464FF00803FDF769
:1058B000F1FE7A8A7B89D3189BB27B82B7F91230CA
:1058C000002B0ADB97F911309AB2BB8AD318BB823E
:1058D0007A8ABB89D31A9BB27B82FB8A03F10103CC
:1058E000FB82FA8A3B889A42CBD907F11C07BD4656
:1058F00090BD00BF80B582B000AFF880B9807A80DB
:105900003B807B88D9B27B88DAB23B88DBB2D31A82
:10591000DAB2F888BB88C31A9BB2F888FDF702FB9D
:105920003869FDF739FE40F20803C2F200031B8814
:1059300003F1FF3398B240F20603C2F200031B8862
:10594000DBB203F1FF33D9B240F20603C2F2000327
:105950001B88DAB240F20803C2F200031B88FDF78D
:10596000E1FA07F10807BD4680BD00BF80B586B0EB
:1059700000AFF860B9607A604FF000037B61FB68AC
:10598000002B03D0FB685B880A2B02D14FF0000389
:1059900050E04FF0140005F0D7FE03467B617B69B1
:1059A000002B45D07B69FA685A60B86805F074FF2F
:1059B0000346184605F0C8FE03463B61B86805F08B
:1059C0006BFF03460C2B0CD93869B9684FF00C02F9
:1059D00005F06AFF3B6903F10C034FF000021A70F7
:1059E00003E03869B96805F04FFF7B693A699A604E
:1059F0007B697A681A61786900F0BCFAFB685B8899
:105A0000FA6803F102034FEA8303D3187A695A60F4
:105A1000FB685B8803F101039AB2FB685A80FB685C
:105A20005B88012B04D1FB68DB684FF001021A731D
:105A30004FF00103184607F11807BD4680BD00BFAF
:105A400080B596B000AFBA607B600346FB810B4621
:105A5000BB817B681B8B1D2B00F22D824FF0000356
:105A60007B654FF000033B6507F1100318464FF0CC
:105A700000014FF0080205F0CAFEFA8940F208035F
:105A8000C2F200031B8803F1FF339A4209DCBA8992
:105A900040F20603C2F200031B8803F1FF339A426F
:105AA00002DD4FF0000308E2FB893B82BB89FB82E9
:105AB000BB681B7C072B50D1FB89A3F115039BB25C
:105AC0007B82BB8903F115039BB2BB82BA6846F6A1
:105AD000FD73C0F600035361BB6803F1080307F1CF
:105AE000100292E8030083E803007B681B8B1A46D0
:105AF0007B6802F10802B96843F822107B681B8BAF
:105B000003F101039AB27B681A83BB685B683B654B
:105B10003B6D1A88BB681A803B6D5B79002B19D1ED
:105B20004FF0000000F062FBF864FB6C5B687B6583
:105B30007B6DBA689A607B6D4FF001025A71FB89E8
:105B4000A3F116039AB2BB8910461946FA6C7B681A
:105B5000FFF776FF4FF00103AFE1BB681B7C012B21
:105B600003D0BB681B7C052B29D1BB681B7C012B98
:105B70000DD1BB685B68FB61BA6846F25523C0F67D
:105B800000035361FB691A88BB681A800CE0BB688C
:105B90005B68BB61BA6846F6C923C0F6000353616F
:105BA000BB691A88BB681A80FB89A3F108039BB202
:105BB0007B82BB8903F11A039BB2BB825FE1BB68A6
:105BC0001B7C0D2B17D1BB685B68BB64BA6846F2BF
:105BD0005133C0F600035361BB6C1A88BB681A804E
:105BE000FB89A3F11C039BB27B82BB8903F11C03DD
:105BF0009BB2BB8243E1BB681B7C032B17D1BB6804
:105C00005B687B64BA6846F2DD33C0F6000353611B
:105C10007B6C1A88BB681A80FB89A3F114039BB2C2
:105C20007B82BB8903F114039BB2BB8227E1BB6873
:105C30001B7C0A2B0DD1BB685B683B64BA6847F6D6
:105C4000F113C0F6000353613B6C1A88BB681A80DD
:105C500015E1BB681B7C092B0DD1BB685B68FB633E
:105C6000BA6847F2C923C0F600035361FB6B1A8878
:105C7000BB681A8003E1BB681B7C042B0DD1BB6899
:105C80005B68BB63BA6846F22153C0F600035361F8
:105C9000BB6B1A88BB681A80F1E0BB681B7C0B2BBE
:105CA0001FD1BB685B687B63BA6846F6F133C0F608
:105CB000000353617B6B1A88BB681A807B6B5B881F
:105CC000FA89D31A9BB203F101039BB27B827B6BEF
:105CD0009A88BB89D3189BB203F1FF339BB2BB8276
:105CE000CDE0BB681B7C022B18D1BB685B683B63B3
:105CF000BA6846F2D953C0F6000353613B6B1B6888
:105D00001A88BB681A80FB89A3F113039BB27B82BC
:105D1000BB8903F113039BB2BB82B0E0BB681B7C61
:105D2000082B46D1BB685B68FB62BA6846F2F56334
:105D3000C0F600035361FB6A1A88BB681A80FB6ACD
:105D40005B7D002B0AD1FB89A3F103039BB27B820D
:105D5000BB8903F111039BB2BB8290E0FB6A5B7DC0
:105D6000012B0AD1FB89A3F111039BB27B82BB8972
:105D700003F173039BB2BB8281E0FB6A5B7D022B64
:105D80007DD1FB89A3F10D039BB23B8240F2050359
:105D9000C2F200031B78DBB2FA89D31A9BB2A3F1DB
:105DA00012039BB27B82BB8903F177039BB2BB8258
:105DB00065E0BB681B7C062B1AD1BB685B68BB62C5
:105DC000BA6847F27923C0F600035361BB6A1A88A8
:105DD000BB681A80BB6A1B89FA89D31A9BB27B8283
:105DE000BB6A9B7A1A46BB89D3189BB2BB8246E03A
:105DF000BB681B7C0C2B1FD1BB685B687B62BA68DD
:105E000048F63D23C0F6000353617B6A1A88BB68DD
:105E10001A807B6A5B88FA89D31A9BB203F101036B
:105E20009BB27B827B6A9A88BB89D3189BB203F1B1
:105E3000FF339BB2BB8222E0BB681B7C0E2B1ED1C2
:105E4000BB685B683B62BA684AF28513C0F6000320
:105E500053613B6A1A88BB681A803B6A5B88FA897F
:105E6000D31A9BB203F101039BB27B823B6A9A88EF
:105E7000BB89D3189BB203F1FF339BB2BB82BB68D3
:105E800003F1080307F1100292E8030083E803001E
:105E90007B681B8B1A467B6802F10802B96843F8DD
:105EA00022107B681B8B03F101039AB27B681A8373
:105EB0004FF0010301E04FF00003184607F15807C7
:105EC000BD4680BD80B483B000AF78607B68002B96
:105ED00002D14FF0000309E07B684FF001021A7213
:105EE0007B684FF000025A724FF00103184607F129
:105EF0000C07BD4680BC704780B483B000AF7860AB
:105F00007B68002B02D14FF0000309E07B684FF063
:105F100001021A717B684FF000025A714FF00103C1
:105F2000184607F10C07BD4680BC704780B483B0AB
:105F300000AF78607B68002B02D14FF0000313E0C4
:105F40007B684FF001021A717B684FF000025A71B2
:105F50007B684FF000025A807A6845F66D13C0F6F0
:105F6000000353634FF00103184607F10C07BD46C9
:105F700080BC704780B483B000AF78607B68002B32
:105F800002D14FF000030DE07B684FF6FF721A80DC
:105F90007B684FF01F025A807B684FF000021A7333
:105FA0004FF00103184607F10C07BD4680BC70474F
:105FB00080B582B000AF78607B68002B02D14FF0D3
:105FC00000035DE07B684FF000029A757B684FF03C
:105FD0000002DA757A6849F26143C0F60003D361C2
:105FE0007A6849F23143C0F60003C2F898307A6803
:105FF00048F67163C0F60003C2F89C307A6848F630
:106000007973C0F60003C2F8A0307B684FF000023D
:106010001A837B6803F1200318464FF000014FF00C
:10602000780205F0F4FB7B68D3F8983078684FF07D
:106030000001984740F29C13C2F200031B88312BE9
:106040001CD840F29C13C2F200031B881A4640F28F
:10605000B823C2F20003796843F8221040F29C137F
:10606000C2F200031B8803F101039AB240F29C13B1
:10607000C2F200031A804FF0010301E04FF0000369
:10608000184607F10807BD4680BD00BF80B582B045
:1060900000AF02460B46FA80BB80BB8803F11E03AB
:1060A0009AB2FB88104619464FF03C024FF00003AD
:1060B000FDF7B0F8FB88A3F11E039BB2BA88104627
:1060C00019464FF03C024FF00103FDF7A3F807F12A
:1060D0000807BD4680BD00BF80B588B000AF03464D
:1060E000B9607A60FB814FF0100005F02DFB03468C
:1060F000BB614FF00003FB614FF000037B61BB69A4
:10610000002B2FD0B86805F0C7FB0346184605F0F2
:106110001BFB03467B617869B96805F0B5FBBB6979
:10612000FA891A80BB697A695A60BB697A68DA6051
:10613000B869FFF7C7FE4FF0180005F005FB0346EE
:10614000FB61FB69002B07D0FB69BA695A60FB69E8
:106150004FF001021A7405E0B86905F0FDFA4FF03E
:106160000003BB61FB69184607F12007BD4680BDEF
:1061700080B584B000AF0B463A600246FA80BB801F
:106180004FF00C0005F0E0FA0346BB604FF000034F
:10619000FB60BB68002B22D0BB68FA881A80BB6802
:1061A000BA885A80BB683A689A60B868FFF7A4FE5C
:1061B0004FF0180005F0C8FA0346FB60FB68002B9F
:1061C00007D0FB68BA685A60FB684FF00D021A747A
:1061D00005E0B86805F0C0FA4FF00003BB60FB684B
:1061E000184607F11007BD4680BD00BF80B584B0DA
:1061F00000AF0346FB804FF0380005F0A5FA0346D8
:10620000BB604FF00003FB60BB68002B1CD0BB6879
:10621000FA881A80B868FFF789FE4FF0180005F079
:1062200093FA0346FB60FB68002B07D0FB68BA6853
:106230005A60FB684FF007021A7405E0B86805F071
:106240008BFA4FF00003BB60FB68184607F110079C
:10625000BD4680BD80B58AB002AFF86007F1040387
:1062600083E80600FB685B68BB61BB88FB827B89B7
:10627000BB824FF00003FB83BB69002B02D14FF0C0
:1062800000035FE0BB695B68184605F005FB034649
:10629000FB74BB694FF001021A72BB695B7A002B79
:1062A00007D14FF6FF70FDF75FF94FF01F03FB8337
:1062B0000AE0BB695B7A012B06D14FF6E070FDF76F
:1062C00053F94CF21863FB83FB7C03F102039BB28E
:1062D0004FEAC3039BB2F98ABA8AF88B009008464A
:1062E00011461A464FF01A03FCF77EFF4FF00100EB
:1062F000FDF7ECF8FB8AA3F1080399B2BB8ADAB286
:1063000040F20503C2F200031B78DBB2C3F11A03AB
:106310004FEAD370C3184FEA6303DBB2D318DBB282
:1063200003F10103DAB2BB695B68084611461A46FD
:106330004FF00103FCF7A8FF4FF00000FDF714F940
:106340004FF00103184607F12007BD4680BD00BF8E
:1063500080B58AB002AFF86007F1040383E8060055
:10636000FB685B68FB61BB887B837B893B834FF069
:106370000003FB82FB69002B02D14FF0000328E0F1
:10638000FB695B88FB82FB694FF001021A714FF0D9
:106390000000FDF7D1F87A8B3B8B104619464FF081
:1063A0001C024FF01C03FCF75BFF7B8B03F1FF33F8
:1063B0009AB23B8B03F101039BB2F98A009110461C
:1063C00019464FF01A024FF01A03FCF70DFF4FF079
:1063D0000103184607F12007BD4680BD80B588B08F
:1063E00002AFF86007F1040383E80600FB685B680E
:1063F0007B61BB887B827B893B827B69002B02D1DE
:106400004FF0000387E07A8A3B8A4FF00001009149
:10641000104619464FF014024FF01403FCF7E4FE47
:106420007B8A03F1FF339AB23B8A03F101039BB2EB
:106430004FF6FF710091104619464FF012024FF0CF
:106440001203FCF7D1FE7B691B7A002B33D04FF08F
:106450000000FDF789F840F20403C2F200031B7844
:10646000DBB2C3F114034FEAD372D3184FEA6303CC
:106470009BB27A8AD31A9AB23B8AD9B240F2050308
:10648000C2F200031B78DBB2C3F114034FEAD370EE
:10649000C3184FEA6303DBB2CB18DBB203F101038D
:1064A000DBB2104619464DF6FC02C0F600024FF072
:1064B0000103FCF7E9FE4FF00100FDF707F84FF08C
:1064C0000000FDF751F87B8AA3F1150399B23B8ACE
:1064D000DAB240F20503C2F200031B78DBB2C3F16B
:1064E00014034FEAD370C3184FEA6303DBB2D31827
:1064F000DBB203F10103DAB27B695B68084611463F
:106500001A464FF00103FCF7BFFE4FF00000FDF705
:106510002BF84FF00103184607F11807BD4680BD60
:1065200080B586B000AFF86007F1040383E8060089
:10653000FB685B687B61BB887B827B893B827B6974
:10654000002B02D14FF0000341E07B694FF00102C4
:106550001A737B695B891846FDF706F87B691B7A1D
:106560001846FCF7B3FF7B695B7B002B04D14FF02F
:106570000000FCF711FD10E07B695B7B012B04D16F
:106580004FF00100FCF708FD07E07B695B7B022B05
:1065900003D14FF00300FCF7FFFC3B8ADAB27B69C2
:1065A0005B68798A084611461A464FF00103FCF7EA
:1065B0006BFE4FF00000FCF7EFFC4FF00100FCF722
:1065C00085FF4FF00000FCF7CFFF4FF001031846A6
:1065D00007F11807BD4680BD80B588B002AFF860EE
:1065E00007F1040383E80600FB685B687B61BB88F6
:1065F0007B827B893B827B69002B02D14FF00003B9
:1066000073E07B694FF001021A727B695B7A012BA0
:1066100020D14FF00000FCF78FFFBA883B89DBB236
:10662000104619464FF009024FF6FF73FEF7E4FFDC
:10663000BB88A3F103039AB23B89DBB2A3F1030346
:10664000DBB2104619464FF006024FF00003FEF78A
:10665000D3FF21E04FF00000FCF76EFFBA883B89C2
:10666000DBB2104619464FF009024FF6FF73FEF7F2
:10667000C3FF7B8AA3F105039AB23B8A03F10603A9
:106680009BB24FF6FF710091104619464FF0090278
:106690004FF00903FCF7A8FD4FF00100FCF716FFCF
:1066A0004FF00000FCF760FF7B8AA3F1160399B25C
:1066B0003B8ADAB240F20503C2F200031B78DBB278
:1066C000C3F114034FEAD370C3184FEA6303DBB27C
:1066D000D318DAB27B695B68084611461A464FF058
:1066E0000103FCF7D1FD4FF00103184607F118072D
:1066F000BD4680BD90B58BB002AFF86007F10403D2
:1067000083E80600FB685B68BB61BB88FB83FB8892
:10671000FB823B89BB827B89BB834FF00003FB7408
:10672000BB69002B02D14FF00003C7E1BB695B6876
:10673000184605F0B1F80346FB74BB694FF001023F
:106740001A75BB695B7D002B1ED1BB8B03F1FF3338
:1067500099B2BB695B7A1A46BB691B7A03F10203E3
:106760009BB2F88B4FF6FF740094FCF73DFDBB69BC
:106770005B7A1A46BB691B7AF88BB98B4FF01F0402
:106780000094FCF731FD42E0BB695B7D012B1DD11C
:10679000FB8B03F1010398B2BB691B7A03F102037F
:1067A0009AB2BB695B7AB98B4FF6FF740094FCF721
:1067B0001BFDBB691B7A1A46BB695B7AF88BB98BE8
:1067C0004FF01F040094FCF70FFD20E0BB695B7DD8
:1067D000022B1CD1BB691B7A03F102039AB2BB697D
:1067E0005B7AF88BB98B4FF6FF740094FCF7FCFCD6
:1067F000FB8B03F1FF3398B2BB691B7A1A46BB6966
:106800005B7AB98B4FF01F040094FCF7EDFCBB6979
:106810005B7D002B35D1BB699B7AFA8BD31A9BB277
:10682000A3F1040399B2BB8B03F1FF339AB2BB69A6
:106830001B7A03F102039BB24FF4FC600090084600
:1068400011464FF00602FCF7CFFC4CF21860FCF743
:1068500073FEBB699B7AFA8BD31A9BB2A3F1040334
:1068600099B2BB8B03F1FF339AB2BB691B7A03F178
:1068700002039BB2084611464FF00602FCF7F0FCFB
:106880007CE0BB695B7D012B41D1FB8B03F10103F4
:1068900099B2BB695B7A1A46BB8BD3189AB2BB69B3
:1068A0009B7AD31A9BB2A3F10A039AB2BB691B7AF3
:1068B00003F102039BB24FF4FC60009008461146BE
:1068C0001A464FF00603FCF78FFC4CF21860FCF7F9
:1068D00033FEFB8B03F1010399B2BB695B7A1A4665
:1068E000BB8BD3189AB2BB699B7AD31A9BB2A3F124
:1068F0000A039AB2BB691B7A03F102039BB20846F2
:1069000011461A464FF00603FCF7AAFC36E0BB69B5
:106910005B7D022B32D1BB699B7A1A46BB8BD318A5
:106920009BB203F104039AB2BB691B7A03F1020321
:106930009BB2F98B4FF4FC600090084611461A4652
:106940004FF00603FCF750FC4CF21860FCF7F4FD26
:10695000BB699B7A1A46BB8BD3189BB203F1040325
:106960009AB2BB691B7A03F102039BB2F98B08460A
:1069700011461A464FF00603FCF772FCBB699A7A7F
:10698000BB69DA72FB7C002B00F08A804FF00000BC
:10699000FCF7EAFD4FF00100FCF798FDBB695B7D59
:1069A000002B1DD1BB695B7A1A46F97C40F20403C7
:1069B000C2F200031B78DBB203FB01F3D31A4FEAE8
:1069C000D372D3184FEA63039BB2FA8BD31A9BB2EC
:1069D00003F10103FB83BB8A03F10203BB8353E092
:1069E000BB695B7D012B21D14FF00100FCF7D4FA8C
:1069F000FB8AA3F10203FB83BB695B7A1A46F97C2D
:106A000040F20403C2F200031B78DBB203FB01F384
:106A1000D31A4FEAD372D3184FEA63039AB2BB8BEF
:106A2000D3189BB203F1FF33BB832DE0BB695B7DC1
:106A3000022B29D14FF00300FCF7AEFA40F2050318
:106A4000C2F200031B78DBB21A46FB8BD3189BB251
:106A500003F10103FB83BB695B7A1A46F97C40F2C0
:106A60000403C2F200031B78DBB203FB01F3D31A69
:106A70004FEAD372D3184FEA63039AB2BB8BD31891
:106A80009BB203F1FF33BB83BB8BDAB2BB695B689C
:106A9000F98B084611461A464FF00103FCF7F4FB48
:106AA0004FF00000FCF778FA4FF00100FCF70EFD04
:106AB0004FF00000FCF758FD4FF00103184607F1B6
:106AC0002407BD4690BD00BF90B58DB002AFF86001
:106AD00007F1040383E80600FB685B68BB61BB88C1
:106AE000FB827B89BB824FF0000387F82730BB69AC
:106AF000002B02D14FF0000374E0BB695B681846BD
:106B000004F0CAFE0446BB699B68184604F0C4FE44
:106B100003469C4208D9BB695B68184604F0BCFE7A
:106B2000034687F8273007E0BB699B68184604F0E6
:106B3000B3FE034687F82730BB695B7B002B0AD185
:106B4000BB695B683B624FF47840FCF70DFD4CF28B
:106B50001863FB8309E0BB699B683B624FF4FC60F0
:106B6000FCF702FD4FF01F03FB8397F8273003F17A
:106B700002039BB24FEAC3039BB2F98ABA8AF88B2D
:106B80000090084611461A464FF01A03FCF72CFBFA
:106B90004FF00100FCF79AFCFB8AA3F108039AB2BC
:106BA000BB8AD9B240F20503C2F200031B78DBB204
:106BB000C3F11A034FEAD370C3184FEA6303DBB281
:106BC000CB18DBB203F10103DBB2104619463A6A77
:106BD0004FF00103FCF758FB4FF00000FCF7C4FC3A
:106BE0004FF00103184607F12C07BD4690BD00BFCA
:106BF00090B58FB002AFF86007F1040383E8060098
:106C0000FB685B687B62BB887B84FB883B843B8939
:106C1000FB837B89BB837B6A002B02D14FF000038F
:106C2000E6E14FF00000FCF787FC7B6A5A887B6A3C
:106C30009B88788CB98B4FF6FF740094FCF7D4FADC
:106C40007B6A5A887B6A9B88788CB98BFCF708FB37
:106C5000BB8B03F102037B833B8C03F10D039AB2E0
:106C60007B8B104619464FF00C024FF00803FCF7DF
:106C7000F7FA3B8C03F1070398B2BB8B03F10403D3
:106C800099B23B8C03F104039AB2BB8B03F1070367
:106C90009BB2FCF7D1FA3B8C03F1080398B2BB8B93
:106CA00003F1040399B23B8C03F10B039AB2BB8B43
:106CB00003F107039BB2FCF7BFFA3B8C03F10B0314
:106CC00098B2BB8B03F1070399B23B8C03F1040329
:106CD0009AB2BB8B03F107039BB2FCF7ADFA7B8B37
:106CE00003F107037B833B8C03F10D0399B27B6AAD
:106CF0009B88A3F112039BB27A8B084611464FF092
:106D00000C02FCF7ADFA7B6A9A88BB8BD3189BB256
:106D1000A3F10A037B833B8C03F10D039AB27B8BB7
:106D2000104619464FF00C024FF00803FCF798FA92
:106D30003B8C03F1070398B2FB8BA3F1040399B2D8
:106D40003B8C03F104039AB2FB8BA3F107039BB2C4
:106D5000FCF772FA3B8C03F1080398B2FB8BA3F1AA
:106D6000040399B23B8C03F10B039AB2FB8BA3F1A2
:106D700007039BB2FCF760FA3B8C03F10B0398B25C
:106D8000FB8BA3F1070399B23B8C03F104039AB286
:106D9000FB8BA3F107039BB2FCF74EFA7B6A9B883F
:106DA000A3F104024AF6AB23C2F6AA2383FB021323
:106DB0004FEA63014FEAE273CB1A3B857B6ADA88BC
:106DC0003B8DD31A9BB27B85B7F92A30002B05DAAD
:106DD0004FF000037B857B6ADB883B857B6A9B8861
:106DE000A3F114033B833B8B06EE103AB8EEC67A50
:106DF000B7F92A3007EE903AF8EEE76A7B6ADB884B
:106E000006EE103AF8EEC67AC6EEA77AF7EE006AFA
:106E100076EEE77A67EE277AFCEEE77A17EE903A9D
:106E2000FB827B6A1B8907EE903AB8EEE77A3B8BD0
:106E300006EE103AF8EE466A7B6ADB8806EE103AF8
:106E4000F8EEC67AC6EEA77A67EE277AFCEEE77A06
:106E500017EE903A9AB2BB8BD3189BB203F10A0398
:106E60007B833B8C03F10C0399B2BB8B03F10A03C8
:106E70009AB27B6A9B88A3F114039BB24FF6FF7012
:106E80000090084611464FF00A02FCF7ADF9B7F939
:106E90002A30002B0EDD3B8C03F10C0399B27A8B68
:106EA000FB8A4FF01F000090084611464FF00A027F
:106EB000FCF79AF97B6ADB88002B00F093804FF097
:106EC0000100FCF703FB04E07B6A1B691A687B6A1C
:106ED0001A617B6A1B691B68002BF5D14FF0000318
:106EE000BB850DE07B6A1B695B68002B04D07B6A65
:106EF0001B695A687B6A1A61BB8D03F10103BB856C
:106F00007B6A1B89BA8D9A42ECD34FF00003BB8594
:106F100061E07B6A1B691B7A012B07D14FF01F03CD
:106F2000FB854FF6FF70FCF71FFB06E04FF6FF7383
:106F3000FB854FF00000FCF717FB7B8CA3F10203ED
:106F400099B2BB8D1A464FEA4202D3184FEA830327
:106F50009AB2BB8BD3189BB203F102039AB27B6A3D
:106F60005B88A3F111039BB2F88D0090084611468F
:106F70001A464FF00C03FCF737F97B8CA3F103039F
:106F800099B2BB8BDAB2BB8DDBB218464FEA400038
:106F9000C3184FEA8303DBB2D318DBB203F1020359
:106FA000DAB27B6A1B69DB68084611461A464FF065
:106FB0000103FCF769F9BA8DB7F9283003F1FF3303
:106FC0009A420EDA7B6A1B695A687B6A1A61BB8D2A
:106FD00003F10103BB85BA8DB7F928309A4298DBDB
:106FE00000E000BF4FF00000FCF7BEFA4FF00103D5
:106FF000184607F13407BD4690BD00BF80B58CB080
:1070000002AFF86007F1040383E80600FB685B68E1
:107010003B62BB88FB83FB88BB837B897B833B6AAA
:10702000002B02D14FF0000321E14FF000037B62FF
:107030003B6A4FF001021A714FF00100FCF746FA6B
:107040004FF6FF70FCF72AFA4FF00000FCF78CFABD
:10705000FA8B7B8B4CF218610091104619464FF069
:1070600016024FF01603FCF7BFF84FF00000FCF7D4
:107070007BFA4FF00000FCF75FFA3B6A5B79002B6C
:1070800040F083804FF00000FCF720FA7B89DBB2F0
:1070900003F1FF33DBB21A46BB8803F1FF339BB227
:1070A000104619464DF60012C0F600024FF00103DB
:1070B000FBF7C8FE7B89DBB203F1FF33DBB21A4674
:1070C000BB88A3F104039BB2104619464DF600128B
:1070D000C0F600024FF00103FBF7B4FE03E07B6A49
:1070E00003F101037B623B6A5B881A467B6A9A4222
:1070F0000AD93A6A7B6A03F102034FEA8303D31881
:107100005B681B7B002BEAD0BB8BA3F117039AB201
:107110007B8B4FF6FF710091104619464FF06002CD
:107120004FF01603FCF760F8BB8BA3F117039AB27C
:107130007B8B104619464FF060024FF01603FCF7A8
:107140008FF84FF00100FCF7C1F93B6A5B88002B18
:1071500000F08B803B89DBB2A3F11003DBB2194650
:10716000BB88A3F130039AB2386A7B6A03F1020349
:107170004FEA8303C3185B689B68084611461A46AA
:107180004FF00103FBF75EFE6FE04FF00000FCF7ED
:107190009DF97B89DBB21A46BB88A3F103039BB23E
:1071A000104619464DF60412C0F600024FF00103D6
:1071B000FBF748FE3B6A9B685B687B6103E07B6A88
:1071C00003F101037B627B695B8803F1FF331A469D
:1071D0007B6A9A420AD97A697B6A03F102034FEA11
:1071E0008303D3185B681B7B002BE8D0BB8B03F1B8
:1071F000FF339AB27B8B4FF6FF7100911046194610
:107200004FF060024FF01603FBF7EEFFBB8B03F16C
:10721000FF339AB27B8B104619464FF060024FF055
:107220001603FCF71DF84FF00100FCF74FF97B69DE
:107230005B88002B19D03B89DBB2A3F11003DBB2D2
:107240001946BB88A3F11A039AB278697B6A03F1E5
:1072500002034FEA8303C3185B689B680846114624
:107260001A464FF00103FBF7EDFD4FF001031846FE
:1072700007F12807BD4680BD90B589B002AFF86020
:1072800007F1040383E80600FB685B687B617B69A8
:10729000002B02D14FF0000311E07B694FF0010297
:1072A000DA72B888F9883B89DBB21A467B89DBB28F
:1072B0007C6964680094FEF71DFB4FF001031846DB
:1072C00007F11C07BD4690BDB0B598B002AFF8609D
:1072D00007F1040383E80600FB685B687B644FF0FA
:1072E00000037B654FF0000387F843304FF0000246
:1072F0004FF00003C7E912234FF000024FF00003E4
:10730000C7E90E237B6C002B02D14FF000036AE328
:107310007B6C4FF0010283F8722040F20803C2F246
:1073200000031B88A3F13203A7F8523040F2060392
:10733000C2F200031B88A3F14803184603F066FE5F
:1073400002460B46C7E90C23B7F8523003F1040399
:10735000FB85D7E90C014FF000024FF00003C4F2A7
:10736000100303F005FD02460B461046194604F0D3
:1073700075F90346BB8540F20803C2F200031B887F
:10738000A3F13C037B8540F20603C2F200031B8895
:10739000A3F150033B857A8D7B6C1B7B92FBF3F34F
:1073A00087F843303A8D4CF6CD43CCF6CC43A3FB63
:1073B00002134FEAD3039BB2184603F027FE02469E
:1073C0000B46C7E908234FF00000FCF7B5F84FF073
:1073D0000000FCF7C9F84FF00100FCF777F8D7E997
:1073E0000C0104F03BF903469AB2B7F852107B8DBA
:1073F000084611461A464FF00003FBF70BFF3B8D82
:10740000184603F003FE02460B46D7E90C0103F0D1
:10741000AFFC02460B461046194604F01FF903461E
:107420009AB2B7F852103B8D084611461A464FF0F3
:107430000103FBF7EFFED7E90C014FF000024FF01C
:107440000003C4F2180303F095FC02460B461046F5
:10745000194604F003F903469AB2B7F8523003F123
:1074600005039BB2104619464DF60812C0F60002FD
:107470004FF00103FBF7E6FCBB8DA3F105039AB2C5
:10748000FB8D03F10B039BB2104619464DF6081213
:10749000C0F600024FF00103FBF7D4FC4FF00003ED
:1074A0007B652AE07A6C7B6D03F104034FEA4303AA
:1074B000D318DB881BB2184603F0A8FD02460B4622
:1074C00010461946D7E9122304F096F80346002B1C
:1074D0000FD07A6C7B6D03F104034FEA4303D3189A
:1074E000DB881BB2184603F091FD02460B46C7E944
:1074F00012237B6D03F101037B657B6C1B7B1A46BA
:107500007B6D9A42CED83B8D184603F07FFD024634
:107510000B4610461946D7E9082303F029FC02461A
:107520000B46D7E9120103F001FF02460B46C7E9FB
:107530000E234FF000037B6502E14FF00000FBF7E4
:10754000FBFF4FF00000FCF70FF8BB8D184603F06F
:107550005DFD04460D46786D03F048FD02460B467E
:1075600010461946D7E9082303F0B6FD02460B463C
:107570002046294603F0FCFB02460B4610461946FE
:1075800004F06CF803469BB2FA8D104619464FF092
:1075900004024FF00003FBF73DFE7B6D092B40F02A
:1075A000CB80BB8D184603F031FD04460D46786D47
:1075B00003F01CFD02460B4610461946D7E9082386
:1075C00003F08AFD02460B462046294603F0D0FB15
:1075D00002460B46104619464FF000024FF080431A
:1075E00003F0C6FB02460B46104619464FF0000258
:1075F0004FF00003C4F2300303F0BAFB02460B461F
:107600001046194604F02AF8034699B2FB8D03F19F
:1076100028039AB27B6C9B68084611461A464FF0C5
:107620000103FBF70FFC07F1140318464DF60C118C
:10763000C0F60001D7E9122304F002F9D7E91201DC
:107640004FF000024FF48043C4F28F0303F0B6FF03
:107650000346002B38D0BB8D184603F0D7FC0446F8
:107660000D46786D03F0C2FC02460B4610461946E3
:10767000D7E9082303F030FD02460B462046294691
:1076800003F076FB02460B46104619464FF0000207
:107690004FF00003C4F2140303F06AFB02460B46EA
:1076A0001046194603F0DAFF034699B2FB8D03F149
:1076B00028039AB207F11403084611461A464FF000
:1076C0000103FBF7BFFB37E0BB8D184603F09EFCC0
:1076D00004460D46786D03F089FC02460B461046C1
:1076E0001946D7E9082303F0F7FC02460B4620466B
:1076F000294603F03DFB02460B46104619464FF063
:1077000000024FF00003C4F2140303F031FB024601
:107710000B461046194603F0A1FF034699B2FB8DB4
:1077200003F130039AB207F11403084611461A46D2
:107730004FF00103FBF786FB7B6D03F101037B65D3
:107740007B6D092B7FF6F9AE4FF000037B6541E1BD
:107750007A6C7B6D03F104034FEA4303D318DB8893
:107760001BB2184603F052FC02460B46104619465F
:10777000D7E90E2303F0DAFD02460B46D7E90C01E8
:1077800003F0F6FA02460B461046194603F066FF70
:107790000346FB83B7F8523003F1FF339CB2FB8BF7
:1077A000184603F033FC02460B46D7E90C0103F000
:1077B000DFFA02460B461046194603F04FFF034618
:1077C00099B297F843309BB203F1FF339AB2FB8B27
:1077D0004FF01F0000902046FBF706FD97F843305E
:1077E0009BB2B7F85220D31AA7F852304FF00000DE
:1077F000FBF7A2FEB7F8523003F101039CB2D7E9C0
:107800000C0103F02BFF03469BB2204619464FF0B4
:1078100004024FF00103FBF7FDFC7B6C1B7B0F2B7D
:1078200024D87B6D03F1010307F1140210464DF6D5
:107830001411C0F600011A4604F002F8D7E90C0151
:1078400003F00CFF03469BB203F1060399B2B7F8AD
:10785000523003F106039AB207F1140308461146A9
:107860001A464FF00103FBF7EDFA7BE07B6C1B7BC4
:107870000F2B43D97B6C1B7B282B3FD87B6D03F1EF
:1078800001014AF6AB23CAF6AA23A3FB01234FEA60
:10789000530213464FEA43039B18CA1A002A61D1C8
:1078A0007B6D03F1010307F1140210464DF614112C
:1078B000C0F600011A4603F0C3FFD7E90C014FF0F0
:1078C00000024FF00003C4F2180303F053FA02461B
:1078D0000B461046194603F0C1FE034699B2B7F8AD
:1078E000523003F106039AB207F114030846114619
:1078F0001A464FF00103FBF7A5FA33E07B6D03F165
:10790000010303F00303002B2CD17B6D03F1010372
:1079100007F1140210464DF61411C0F600011A4684
:1079200003F08EFFD7E90C014FF000024FF0000387
:10793000C4F2180303F01EFA02460B46104619461D
:1079400003F08CFE034699B2B7F8523003F10603F8
:107950009AB207F11403084611461A464FF0010384
:10796000FBF770FA7B6C1B7B03F1FF331A467B6DD0
:107970009A422BD1D7E90C014FF000024FF00003DF
:10798000C4F2080303F0F6F902460B461046194606
:107990004FF000024FF00003C4F2300303F0EAF9A5
:1079A00002460B461046194603F058FE034699B2AC
:1079B000B7F8523003F118039AB27B6C5B68084643
:1079C00011461A464FF00103FBF73CFA7B6D03F1B9
:1079D00001037B657B6C1B7B1A467B6D9A423FF6ED
:1079E000B7AE4FF00103184607F15807BD46B0BDCA
:1079F000F0B5A3B002AFF86007F1040383E8060016
:107A00004FF00003FB674FF47843FB834FF0000215
:107A10004FF00003C7E91823FB685B68FB65FB6D4B
:107A2000002B03D14FF0000301F003B8FB6D4FF0C2
:107A3000010283F8D6204FF000024FF00003C7E99F
:107A40001C2340F20803C2F200031B88A3F1350394
:107A5000184603F0DBFA02460B46C7E91A2340F248
:107A60000603C2F200031B88A3F13F03184603F08C
:107A7000CDFA02460B46C7E91423D7E91A014FF0A5
:107A800000024FF00003C4F2100303F073F9024642
:107A90000B46C7E91223D7E91423C7E9102340F2A4
:107AA0000803C2F200031B88A3F14803184603F041
:107AB000ADFA02460B46C7E90E2340F20603C2F2B6
:107AC00000031B88A3F15103184603F09FFA0246F6
:107AD0000B46C7E90C23FB6D93F8D430184603F02E
:107AE00095FA02460B46D7E90E0103F01FFC024649
:107AF0000B46C7E90A23D7E90C014FF000024FF00B
:107B00000003C4F2260303F011FC02460B46C7E94A
:107B100008234FF00000FBF727FD4FF00100FBF7B3
:107B2000D5FCD7E91A0103F099FD03469DB2D7E9C8
:107B3000140103F093FD03469CB2D7E90E014FF008
:107B400000024FF0804303F015F902460B46104641
:107B5000194603F083FD03469BB2284621461A4688
:107B60004FF00003FBF756FBD7E91A0103F076FD4F
:107B700003469DB2D7E91401D7E90C2303F0F8F8C6
:107B800002460B461046194603F068FD03469CB2B8
:107B9000D7E90C0103F062FD03469BB2284621465B
:107BA0001A464FF00103FBF735FBD7E914014FF0FC
:107BB00000024FF00003C4F2180303F0DBF80246A2
:107BC0000B461046194603F049FD03469CB2D7E91F
:107BD0001A014FF000024FF00003C4F2140303F047
:107BE000C9F802460B461046194603F037FD034616
:107BF0009BB2204619464DF60812C0F600024FF01F
:107C00000103FBF71FF9D7E910014FF000024FF015
:107C10000003C4F2140303F0ABF802460B4610460F
:107C2000194603F01BFD03469CB2D7E912014FF041
:107C300000024FF00003C4F2320303F09BF8024647
:107C40000B46104619464FF000024FF00003C4F2F5
:107C5000220303F08DF802460B461046194603F046
:107C6000FDFC03469BB2204619464DF60812C0F6AD
:107C700000024FF00103FBF7E5F8FB6D93F8D530F8
:107C8000012B61D1D7E91A0103F0E8FC03469EB24B
:107C9000D7E91401D7E90C2303F06AF802460B4632
:107CA0001046194603F0DAFC03469DB2D7E90E01EF
:107CB0004FF000024FF0804303F05CF802460B46A1
:107CC0001046194603F0CAFC03469CB2D7E90C01E2
:107CD00003F0C4FC03469BB24FF000020092304612
:107CE00029462246FBF780FA4FF6E073FB832BE030
:107CF000FA6DFB6F03F104034FEA4303D3189B882B
:107D00001BB2184603F082F902460B46104619468C
:107D1000D7E91C2303F070FC0346002B0FD0FA6D4B
:107D2000FB6F03F104034FEA4303D3189B881BB294
:107D3000184603F06BF902460B46C7E91C23FB6F9C
:107D400003F10103FB6700E000BFFB6D93F8D43043
:107D50001A46FB6F9A42CBD8D7E90C01D7E9082322
:107D600003F006F802460B46D7E91C0103F0DEFAE1
:107D700002460B46C7E918234FF00003FB676EE18C
:107D8000FB6F002B70D04FF00000FBF7D5FBD7E95D
:107D9000120103F063FC03469CB2F86F03F026F96E
:107DA00002460B4610461946D7E9082303F094F91A
:107DB00002460B46D7E9100102F0DAFF02460B46F5
:107DC0001046194603F04AFC03469BB2204619466A
:107DD0004FF004024FF00003FBF71CFA4CF218605E
:107DE000FBF7AAFBD7E912014FF000024FF00003A6
:107DF000C4F2100302F0BCFF02460B4610461946BF
:107E000003F02CFC03469DB2F86F03F0EFF8024636
:107E10000B4610461946D7E9082303F05DF90246E0
:107E20000B46D7E9100102F0A3FF02460B461046AD
:107E3000194603F013FC03469CB2D7E90E014FF03C
:107E400000024FF0804302F095FF02460B461046B9
:107E5000194603F003FC03469BB2284621461A4606
:107E60004FF00003FBF7D6F9FB6F0A2B40F0F380CD
:107E70004FF00000FBF778FBF86F03F0B7F802460D
:107E80000B4610461946D7E9082303F025F90246A8
:107E90000B46D7E9100102F06BFF02460B46104675
:107EA00019464FF000024FF0804302F061FF024696
:107EB0000B46104619464FF000024FF00003C4F283
:107EC000300302F055FF02460B461046194603F0F8
:107ED000C5FB03469CB2D7E912014FF000024FF0F8
:107EE0000003C4F2420302F045FF02460B4610466F
:107EF000194603F0B3FB03469AB2FB6D9B6820461C
:107F000011461A464FF00103FAF79CFF07F11403DC
:107F100018464DF60C11C0F60001D7E91C2303F0FA
:107F20008FFCD7E91C014FF000024FF48043C4F2EC
:107F30008F0303F043FB0346002B40D0F86F03F0A0
:107F400055F802460B4610461946D7E9082303F0B8
:107F5000C3F802460B46D7E9100102F009FF0246BA
:107F60000B46104619464FF000024FF00003C4F2D2
:107F7000140302F0FDFE02460B461046194603F0BC
:107F80006DFB03469CB2D7E912014FF000024FF09F
:107F90000003C4F2420302F0EDFE02460B46104617
:107FA000194603F05BFB03469AB207F1140320461F
:107FB00011461A464FF00103FAF744FF4BE0F86F01
:107FC00003F014F802460B4610461946D7E9082379
:107FD00003F082F802460B46D7E9100102F0C8FE12
:107FE00002460B46104619464FF000024FF00003C0
:107FF000C4F2140302F0BCFE02460B4610461946BA
:1080000003F02CFB03469CB2D7E912014FF00002AB
:108010004FF00003C4F2200302F0ACFE02460B4610
:10802000104619464FF000024FF00003C4F242031D
:1080300002F0A0FE02460B461046194603F00EFB66
:1080400003469AB207F11403204611461A464FF030
:108050000103FAF7F7FEFB6F03F10103FB67FB6F08
:108060000A2B7FF68DAE4FF00003FB6700F0D3BC08
:10807000D7E91A01D7E90A2302F07AFE02460B4635
:10808000C7E91A234FF00000FBF756FAD7E91A01A7
:108090004FF000024FF00003C3F6F07302F06AFEE7
:1080A00002460B461046194603F0D8FA03469CB226
:1080B000D7E9140103F0D2FA03469BB220461946D1
:1080C0004FF004024FF00103FBF7A4F8FB6D93F8A7
:1080D000D4300F2B6BD8FB6F03F1010307F11402AF
:1080E00010464DF61411C0F600011A4603F0A8FB25
:1080F000D7E914014FF000024FF00003C4F2180357
:1081000002F038FE02460B461046194603F0A6FA66
:1081100003469CB2D7E91A014FF000024FF000036A
:10812000C4F2180302F026FE02460B46104619461A
:1081300003F094FA03469AB207F11403204611465D
:108140001A464FF00103FAF77DFE4CF21860FBF778
:10815000F3F9D7E91A014FF000024FF00003C3F61C
:10816000F07302F007FE02460B461046194603F074
:1081700075FA03469DB2D7E91401D7E90C2302F042
:10818000F7FD02460B461046194603F067FA034610
:108190009CB2D7E90C0103F061FA03469BB2284672
:1081A00021461A464FF00103FBF734F886E1FB6DD8
:1081B00093F8D4300F2B40F28480FB6D93F8D430C9
:1081C000282B7ED8FB6F03F101014AF6AB23CAF6D8
:1081D000AA23A3FB01234FEA530213464FEA4303AA
:1081E0009B18CA1A002A40F06981FB6F03F1010352
:1081F00007F1140210464DF61411C0F600011A469C
:1082000003F01EFBD7E914014FF000024FF000030A
:10821000C4F2180302F0AEFD02460B4610461946A2
:1082200003F01CFA03469CB2D7E91A014FF0000292
:108230004FF00003C4F2180302F09CFD02460B4607
:108240001046194603F00AFA03469AB207F11403DE
:10825000204611461A464FF00103FAF7F3FD4CF29F
:108260001860FBF769F9D7E91A014FF000024FF0E7
:108270000003C3F6F07302F07DFD02460B46104684
:10828000194603F0EBF903469DB2D7E91401D7E98B
:108290000C2302F06DFD02460B461046194603F012
:1082A000DDF903469CB2D7E90C0103F0D7F9034688
:1082B0009BB2284621461A464FF00103FAF7AAFF5F
:1082C000FCE0FB6D93F8D430282B78D9FB6D93F844
:1082D000D430462B73D8FB6F03F1010303F0030383
:1082E000002B40F0EB80FB6F03F1010307F1140258
:1082F00010464DF61411C0F600011A4603F0A0FA1C
:10830000D7E914014FF000024FF00003C4F2180344
:1083100002F030FD02460B461046194603F09EF966
:1083200003469CB2D7E91A014FF000024FF0000358
:10833000C4F2180302F01EFD02460B461046194611
:1083400003F08CF903469AB207F114032046114654
:108350001A464FF00103FAF775FD4CF21860FBF76F
:10836000EBF8D7E91A014FF000024FF00003C3F613
:10837000F07302F0FFFC02460B461046194603F06C
:108380006DF903469DB2D7E91401D7E90C2302F039
:10839000EFFC02460B461046194603F05FF9034610
:1083A0009CB2D7E90C0103F059F903469BB2284669
:1083B00021461A464FF00103FAF72CFF7EE0FB6FCF
:1083C00003F101014CF6CD43CCF6CC43A3FB0123D2
:1083D0004FEAD30213464FEA83039B184FEA430345
:1083E000CA1A002A6AD1FB6F03F1010307F11402D4
:1083F00010464DF61411C0F600011A4603F020FA9B
:10840000D7E914014FF000024FF00003C4F2180343
:1084100002F0B0FC02460B461046194603F01EF966
:1084200003469CB2D7E91A014FF000024FF0000357
:10843000C4F2180302F09EFC02460B461046194691
:1084400003F00CF903469AB207F1140320461146D3
:108450001A464FF00103FAF7F5FC4CF21860FBF7EF
:108460006BF8D7E91A014FF000024FF00003C3F692
:10847000F07302F07FFC02460B461046194603F0EB
:10848000EDF803469DB2D7E91401D7E90C2302F0B9
:108490006FFC02460B461046194603F0DFF8034610
:1084A0009CB2D7E90C0103F0D9F803469BB22846E9
:1084B00021461A464FF00103FAF7ACFEFB6F002B82
:1084C00040F0FD80D7E91A01D7E90A2302F052FCF7
:1084D00002460B461046194603F0C0F803469EB20A
:1084E000D7E9140103F0BAF803469DB2D7E91A019F
:1084F00003F0B4F803469CB2FA6DFB6F03F104037A
:108500004FEA4303D3189B881BB2184602F07EFD46
:1085100002460B4610461946D7E9182302F006FF1B
:1085200002460B46D7E9140102F022FC02460B4634
:108530001046194603F092F803469BB2FA8B92B2AA
:108540000092304629462246FDF7A6F8D7E91A01DF
:10855000D7E90A2302F00EFC02460B4610461946E4
:1085600003F07CF803469EB2D7E914014FF00002F5
:108570004FF00003C3F6F07302F0FAFB02460B461D
:108580001046194603F06AF803469DB2D7E91A016E
:1085900003F064F803469CB2FA6DFB6F03F1040329
:1085A0004FEA4303D3189B881BB2184602F02EFDF6
:1085B00002460B4610461946D7E9182302F0B6FECC
:1085C00002460B46D7E9140102F0D2FB02460B46E5
:1085D000104619464FF000024FF00003C3F6F07347
:1085E00002F0C6FB02460B461046194603F036F869
:1085F00003469BB2FA8B92B200923046294622463D
:10860000FDF74AF8D7E91A01D7E90A2302F0B2FBCD
:1086100002460B46104619464FF000024FF0000389
:10862000C3F6F07302F0A4FB02460B46104619464F
:1086300003F014F803469EB2D7E9140103F00EF8D4
:1086400003469DB2D7E91A014FF000024FF0000334
:10865000C3F6F07302F08CFB02460B461046194637
:1086600002F0FCFF03469CB2FA6DFB6F03F10403BA
:108670004FEA4303D3189B881BB2184602F0C6FC8E
:1086800002460B4610461946D7E9182302F04EFE63
:1086900002460B46D7E9140102F06AFB02460B467C
:1086A0001046194602F0DAFF03469BB2FA8B92B2EB
:1086B0000092304629462246FCF7EEFF61E1D7E9F9
:1086C0001A01D7E90A2302F055FB02460B46104671
:1086D000194602F0C3FF03469EB2FB6F03F1FF335E
:1086E000FA6D03F104034FEA4303D3189B881BB2CE
:1086F000184602F08BFC02460B4610461946D7E995
:10870000182302F013FE02460B46D7E9140102F0CB
:108710002FFB02460B461046194602F09FFF034608
:108720009DB2D7E91A0102F099FF03469CB2FA6D97
:10873000FB6F03F104034FEA4303D3189B881BB27A
:10874000184602F063FC02460B4610461946D7E96C
:10875000182302F0EBFD02460B46D7E9140102F0A4
:1087600007FB02460B461046194602F077FF034608
:108770009BB2FA8B92B20092304629462246FCF711
:108780008BFFD7E91A01D7E90A2302F0F3FA024670
:108790000B461046194602F061FF03469EB2FB6F7E
:1087A00003F1FF33FA6D03F104034FEA4303D318D7
:1087B0009B881BB2184602F029FC02460B46104665
:1087C0001946D7E9182302F0B1FD02460B46D7E956
:1087D000140102F0CDFA02460B46104619464FF03E
:1087E00000024FF00003C3F6F07302F0C1FA024634
:1087F0000B461046194602F031FF03469DB2D7E9F9
:108800001A014FF000024FF00003C3F6F07302F0BC
:10881000AFFA02460B461046194602F01FFF034608
:108820009CB2FA6DFB6F03F104034FEA4303D318C4
:108830009B881BB2184602F0E9FB02460B46104625
:108840001946D7E9182302F071FD02460B46D7E915
:10885000140102F08DFA02460B46104619464FF0FD
:1088600000024FF00003C3F6F07302F081FA0246F3
:108870000B461046194602F0F1FE03469BB2FA8BF6
:1088800092B20092304629462246FCF705FFD7E90E
:108890001A01D7E90A2302F06DFA02460B46104688
:1088A00019464FF000024FF00003C3F6F07302F0D8
:1088B0005FFA02460B461046194602F0CFFE034609
:1088C0009EB2FB6F03F1FF33FA6D03F104034FEA2D
:1088D0004303D3189B881BB2184602F097FB02464D
:1088E0000B4610461946D7E9182302F01FFD024631
:1088F0000B46D7E9140102F03BFA02460B4610463C
:10890000194602F0ABFE03469DB2D7E91A014FF0BB
:1089100000024FF00003C3F6F07302F029FA02469A
:108920000B461046194602F099FE03469CB2FA6DBA
:10893000FB6F03F104034FEA4303D3189B881BB278
:10894000184602F063FB02460B4610461946D7E96B
:10895000182302F0EBFC02460B46D7E9140102F0A3
:1089600007FA02460B461046194602F077FE034608
:108970009BB2FA8B92B20092304629462246FCF70F
:108980008BFEFB6D93F8D43003F1FF331A46FB6F77
:108990009A423CD14FF00000FAF7E6FDD7E9140106
:1089A0004FF000024FF00003C4F2080302F0E2F9B6
:1089B00002460B46104619464FF000024FF00003E6
:1089C000C4F2300302F0D6F902460B4610461946AF
:1089D00002F044FE03469CB2D7E91A014FF00002B0
:1089E0004FF00003C4F2380302F0C4F902460B460C
:1089F0001046194602F032FE03469AB2FB6D5B68E0
:108A0000204611461A464FF00103FAF71BFAFB6F96
:108A100003F10103FB67FB6D93F8D4301A46FB6F3B
:108A20009A423FF625AB4FF00000FAF74FFD4FF0AA
:108A30000103184607F18407BD46F0BD2DE9F04358
:108A40008FB002AFF86007F1040383E806006B46BD
:108A50001E46FB685B68BB6240F20803C2F200037B
:108A60001B884FEAD3039BB203F1010101F1FF33ED
:108A70007B62084602464FF000034FEA52704FEA0D
:108A8000C30940EA09094FEAC208084602464FF006
:108A900000034FEA52704FEAC30505434FEAC20490
:108AA0000B4603F107034FEAD3034FEAC303ADEBD1
:108AB000030D02AB03F100033B62BB88FB837B89A0
:108AC000BB83BB6A002B02D14FF00003C7E04FF01D
:108AD0000000FAF731FDBB6A5A88BB6A9B88F88BA5
:108AE000B98B4FF6FF740094FAF77EFBBB6A5A8885
:108AF000BB6A9B88F88BB98BFAF7B2FBBB6A9B68A1
:108B0000002B00F0AA80BB6A5B88A3F10603002B50
:108B100001DA03F107034FEAE3037B83BB6A9B8817
:108B2000A3F104024AF6AB23C2F6AA2383FB021385
:108B30004FEA63014FEAE273CB1A3B83BB6A9B683F
:108B4000184602F0A9FE0346FB824FF00100FAF737
:108B5000BDFC4FF00000FAF707FDFA8A7B8B9A42C2
:108B600069D94FF00003FB8559E0396ABB6A9A68FE
:108B7000FB8D788B00FB03F3D2187B8B03F1010391
:108B8000084611461A4602F08FFEFA8D3B8B03F120
:108B9000FF339A4216D17B8B03F1FF333A6AD35CE1
:108BA000002B0FD0FA8AFB8D798B01FB03F3D21ACD
:108BB0007B8B9A4206DD7B8B03F1FF333A6A4FF0E1
:108BC0007E01D1547B8B3A6A4FF00001D154FB8B6C
:108BD000A3F1030399B2BB8BDAB2FB8DDBB218466B
:108BE0004FEA4000C3184FEA8303DBB2D318DAB26E
:108BF000FB8D002B0CBF00230123DBB2D31ADBB2A9
:108C000003F10203DAB23B6A084611461A464FF0F6
:108C10000103FAF739FBFB8D03F10103FB85FA8AA7
:108C2000FB8D798B01FB03F39A4216DD3A8BFB8DAA
:108C30009A429AD811E0FB8BA3F1030399B2BB8B44
:108C4000DBB203F10203DAB2BB6A9B680846114645
:108C50001A464FF00103FAF717FB4FF00103B54630
:108C6000184607F13407BD46BDE8F08380B48BB0E9
:108C700000AFF860B9607A60FB685B683B62FB68D4
:108C80005B89FB83FB689B89BB83FB68DB897B83F8
:108C90003B6A002B02D14FF00003E2E0FB8B03F1B3
:108CA00012031A46BB689A4280F084807B8B7A68F4
:108CB000D31AA3F102024AF6AB23CAF6AA23A3FBF6
:108CC00002134FEAD3039AB23B6A1B89D3183B8342
:108CD0003B6ADB883A8B9A4206D33B6A4FF6FF72B7
:108CE0005A814FF00103BCE03A8B3B6A5A8104E0A1
:108CF0003B6A1B691A683B6A1A613B6A1B691B68FD
:108D0000002BF5D13B6A1B7B002B31D14FF00003C8
:108D1000FB8427E0FA8C3B8B9A4210D13B6A1B699B
:108D20001B7A012B05D13B6A1B694FF000021A72B6
:108D30000AE03B6A1B694FF001021A7204E03B6AC9
:108D40001B694FF000021A723B6A1B695B68002BBB
:108D500004D03B6A1B695A683B6A1A61FB8C03F1B9
:108D60000103FB843B6ADB88FA8C9A42D2D376E01B
:108D70004FF00003FB8408E03B6A1B695A683B6ABA
:108D80001A61FB8C03F10103FB84FA8C3B8B9A4242
:108D9000F2D33B6A1B691B7A012B05D13B6A1B6925
:108DA0004FF000021A725AE03B6A1B694FF0010251
:108DB0001A7254E07A8B7B689A422CBF00230123FD
:108DC000DAB27B8B03F10C0319467B68994294BF9E
:108DD00000230123DBB21340DBB2002B0BD03B6A34
:108DE0001B89002B3BD03B6A1B8903F1FF339AB2EE
:108DF0003B6A1A8133E0BB8BA3F10C031A467B68F4
:108E00009A422CBF00230123DAB2B98B7B689942C6
:108E100094BF00230123DBB21340DBB2002B1ED032
:108E20003B6A9B88A3F102024AF6AB23C2F6AA234F
:108E300083FB02134FEA63014FEAE273CB1AFB8212
:108E4000FA8A3B6A1B89D2183B6ADB889A4206DAA7
:108E50003B6A1B8903F101039AB23B6A1A814FF006
:108E60000103184607F12C07BD4680BC704700BFC0
:108E700080B489B000AF78600B467B804FF0000370
:108E8000FB617B68002B6ED067E07B68FA6902F1BA
:108E9000080253F822301B7C012B0FD17B68FA6942
:108EA00002F1080253F822305B68BB61BB691B8882
:108EB0007A889A424DD1BB695B7A56E07B68FA6941
:108EC00002F1080253F822301B7C052B0FD17B687E
:108ED000FA6902F1080253F822305B687B617B6912
:108EE0001B887A889A4234D17B695B7B3DE07B6842
:108EF000FA6902F1080253F822301B7C032B0FD1D0
:108F00007B68FA6902F1080253F822305B683B6122
:108F10003B691B887A889A421BD13B691B7A24E003
:108F20007B68FA6902F1080253F822301B7C062B99
:108F30000FD17B68FA6902F1080253F822305B68AE
:108F4000FB60FB681B887A889A4202D1FB681B7B16
:108F50000BE0FB6903F10103FB617B681B8B1A4685
:108F6000FB699A4291D84FF00003184607F1240795
:108F7000BD4680BC704700BF80B590B000AFF860C0
:108F8000B9601346FB804FF00003FB6307F1100349
:108F900018464FF000014FF0080202F038FCBB68A1
:108FA000002B40F06881FB681A4607F1100303CBE1
:108FB000106051606EE1BB68FA6B02F1080253F871
:108FC00022301B7C042B1DD1BB68FA6B02F1080216
:108FD00053F822305B68BB63BB6B1B88FA889A42EC
:108FE0000CD1BB68FA6B02F1080253F82230FA6820
:108FF00003F1080303CB106051604BE1FB6B03F1FD
:109000000103FB63BB68FA6B02F1080253F82230DC
:109010001B7C012B1DD1BB68FA6B02F1080253F8CF
:1090200022305B687B637B6B1B88FA889A420CD189
:10903000BB68FA6B02F1080253F82230FA6803F1B8
:10904000080303CB1060516024E1FB6B03F10103C3
:10905000FB63BB68FA6B02F1080253F822301B7CF9
:109060000D2B1DD1BB68FA6B02F1080253F82230B8
:109070005B683B633B6B1B88FA889A420CD1BB68E8
:10908000FA6B02F1080253F82230FA6803F1080380
:1090900003CB10605160FDE0FB6B03F10103FB6348
:1090A000BB68FA6B02F1080253F822301B7C052BD7
:1090B0001DD1BB68FA6B02F1080253F822305B68DD
:1090C000FB62FB6A1B88FA889A420CD1BB68FA6B78
:1090D00002F1080253F82230FA6803F1080303CBC7
:1090E00010605160D6E0FB6B03F10103FB63BB68CA
:1090F000FA6B02F1080253F822301B7C032B1DD1BE
:10910000BB68FA6B02F1080253F822305B68BB625D
:10911000BB6A1B88FA889A420CD1BB68FA6B02F1D1
:10912000080253F82230FA6803F1080303CB1060F9
:109130005160AFE0FB6B03F10103FB63BB68FA6BAB
:1091400002F1080253F822301B7C022B1DD1BB68B0
:10915000FA6B02F1080253F822305B687B627B6A8B
:109160001B88FA889A420CD1BB68FA6B02F108029C
:1091700053F82230FA6803F1080303CB1060516002
:1091800088E0FB6B03F10103FB63BB68FA6B02F140
:10919000080253F822301B7C072B1DD1BB68FA6BE9
:1091A00002F1080253F822305B683B623B6A1B887D
:1091B000FA889A420CD1BB68FA6B02F1080253F8A4
:1091C0002230FA6803F1080303CB1060516061E0BC
:1091D000FB6B03F10103FB63BB68FA6B02F108024E
:1091E00053F822301B7C062B1DD1BB68FA6B02F1B1
:1091F000080253F822305B68FB61FB691B88FA8820
:109200009A420CD1BB68FA6B02F1080253F8223083
:10921000FA6803F1080303CB106051603AE0FB6B7E
:1092200003F10103FB63BB68FA6B02F1080253F818
:1092300022301B7C082B1FD1BB68FA6B02F108029D
:1092400053F822305B68BB61BB691B88FA889A427D
:109250000CD1BB68FA6B02F1080253F82230FA68AD
:1092600003F1080303CB1060516013E0FB6B03F1C3
:109270000103FB6300E000BFBB681B8B1A46FB6B5E
:109280009A423FF698AEFB681A4607F1100303CBEB
:1092900010605160F86807F14007BD4680BD00BF0F
:1092A00090B58BB000AF786007F10C0318464FF013
:1092B00000014FF0040202F0AAFA7B681B7C012B2C
:1092C00013D17B685B687B627B6A5B68184602F03F
:1092D000E3FA034603F101039BB24FEAC3039BB2D7
:1092E000FB814FF01A03BB8193E07B681B7C0D2B45
:1092F00006D14FF01C03FB814FF01C03BB8188E0BB
:109300007B681B7C052B2FD17B685B683B623B6ACB
:109310005B68184602F0C0FA04463B6A9B68184630
:1093200002F0BAFA03469C420DD93B6A5B681846C4
:1093300002F0B2FA034603F101039BB24FEAC30302
:109340009BB2FB810CE03B6A9B68184602F0A4FAD2
:10935000034603F101039BB24FEAC3039BB2FB81B7
:109360004FF01A03BB8154E07B681B7C032B06D1B2
:109370004FF01403FB814FF01403BB8149E07B687D
:109380001B7C022B06D14FF01403FB814FF014031A
:10939000BB813EE07B681B7C072B06D14FF0160398
:1093A000FB814FF01603BB8133E07B681B7C082BED
:1093B00014D17B685B68FB61FB695B7D002B06D188
:1093C000FB695B7AFB81FB691B7ABB8121E0FB694E
:1093D0005B7ABB81FB691B7AFB811AE07B681B7C93
:1093E0000B2B09D17B685B68BB61BB695B88FB8128
:1093F000BB699B88BB810CE07B681B7C0E2B08D172
:109400007B685B687B617B695B88FB817B699B8890
:10941000BB81FB683B614FF000033A8A62F30F03A4
:109420007A8A62F31F43184607F12C07BD4690BDA8
:1094300080B483B000AF78600B46FB707B68002B74
:1094400002D14FF0000304E07B68FA789A754FF080
:109450000103184607F10C07BD4680BC704700BFEA
:1094600080B584B000AF78600B46FB704FF000030E
:10947000FB607B68002B02D14FF000033DE07B686E
:10948000FA78DA757B68D3F89830FA7878681146FC
:109490009847FB78012B23D11BE07B68FA6802F127
:1094A000080253F822305B697A68F96801F1080113
:1094B00052F821107A68F86800F1080052F820206C
:1094C000084602F1080206CA9847FB6803F1010347
:1094D000FB607B681B8B1A46FB689A42DDD803E071
:1094E0004FF6FF70F9F79EFD7B68D3F89830FA7855
:1094F0007868114698474FF00103184607F11007A6
:10950000BD4680BD80B58CB002AF78604FF00003DF
:109510007B624FF000033B624FF00003FB614FF0B2
:109520000003BB617B681B7C03F1FF330D2B00F252
:10953000F98201A252F823F07195000825960008DF
:10954000C1950008259B0008F3950008259B00089D
:10955000B1960008E1980008259B0008259B0008AB
:10956000CB9A0008259B0008259B0008019B00085A
:109570007B685B687B617B694FF001025A727B6894
:109580005B697A68786802F1080206CA984703E0C6
:109590007B6A03F101037B627A6A48F29F63C0F23F
:1095A00001039A42F4D97B694FF000025A727B683A
:1095B0005B697A68786802F1080206CA9847B6E2E1
:1095C0007B685B687B617B691B7A012B04D17B69BB
:1095D0004FF000021A7203E07B694FF001021A7229
:1095E0007B685B697A68786802F1080206CA984766
:1095F0009DE27B685B687B617B695B7B012B04D1AF
:109600007B694FF000025A7303E07B694FF001025F
:109610005A737B685B697A68786802F1080206CA47
:10962000984784E27B685B681B68FB617B685B68CA
:109630007B617B695B7A002B40F076824FF0000300
:109640007B620DE0FA697B6A4FEA8303D3185B689B
:109650005B684FF000025A727B6A03F101037B6280
:10966000FB695B881A467B6A9A42EBD87B694FF0AC
:1096700001025A724FF000037B6212E0FA697B6AC2
:109680004FEA8303D3185B687B607B685B697A6809
:10969000786802F1080206CA98477B6A03F1010361
:1096A0007B62FB695B881A467B6A9A42E6D83BE29A
:1096B0007B685B68BB617B681A897B68DB8947F6DE
:1096C000FF710091104619464FF016024FF0160335
:1096D000F9F78AFD4FF00000F9F7F8FEBB695B79F6
:1096E000002B40F081804CF21860F9F73DFF7B6859
:1096F000DB89DBB203F1FF33DBB21A467B681B89DF
:1097000003F1FF339BB2104619464DF60012C0F626
:1097100000024FF00103F9F795FB7B68DB89DBB2B0
:1097200003F1FF33DBB21A467B681B89A3F1040304
:109730009BB2104619464DF60012C0F600024FF0DB
:109740000103F9F77FFB4FF0140000F0EDFB4FF041
:1097500000037B621BE0BA697B6A03F102034FEAF4
:109760008303D3185B681B7B012B01D17B6A3B62AF
:10977000BA697B6A03F102034FEA8303D3185B687B
:109780004FF000021A737B6A03F101037B62BB692D
:109790005B881A467B6A9A42DDD83B6A002B0AD165
:1097A000BA693B6A03F102034FEA8303D3185B688B
:1097B0004FF001021A733B6A002B0CD03B6A03F195
:1097C000FF33BA6903F102034FEA8303D3185B68DE
:1097D0004FF001021A737B685B697A68786802F15E
:1097E000080206CA984776E04CF21860F9F7BCFE0A
:1097F0007B68DB89DBB21A467B681B89A3F1030314
:109800009BB2104619464DF60412C0F600024FF006
:109810000103F9F717FB4FF0140000F085FB7B689C
:109820005B689B685B683B614FF000037B621BE0F9
:109830003A697B6A03F102034FEA8303D3185B683A
:109840001B7B012B01D17B6A3B623A697B6A03F186
:1098500002034FEA8303D3185B684FF000021A73C8
:109860007B6A03F101037B623B695B881A467B6A72
:109870009A42DDD83B695B8803F1FF331A463B6AA5
:109880009A420BD13A693B6A03F102034FEA830320
:10989000D3185B684FF001021A7314E03B695B88D0
:1098A00003F1FF331A463B6A9A420CD93B6A03F133
:1098B00001033A6903F102034FEA8303D3185B689B
:1098C0004FF001021A737B685B697A68786802F16D
:1098D000080206CA98474FF00100F9F7F7FD26E1A4
:1098E0007B685B687B617A6807F1080302F1080214
:1098F00092E8030083E803007B695B7D002B3FD186
:109900003B891A467B699B7AD31AA3F104031A4652
:1099100040F20423C2F200031B689A420FD87B690D
:109920009B7A002B0BD07B699A7A7B69DA727B6910
:109930009B7AA3F10503DAB27B699A72AAE07B896C
:109940001A467B699B7AD31AA3F10A031A4640F29E
:109950000423C2F200031B689A42C0F096807B6920
:109960009B7A632B00F291807B699A7A7B69DA7229
:109970007B699B7A03F10503DAB27B699A7284E012
:109980007B695B7D012B3DD1BB891A467B699B7A44
:10999000D31AA3F104031A4640F20C23C2F20003C7
:1099A0001B689A420FD27B699B7A002B0BD07B6994
:1099B0009A7A7B69DA727B699B7AA3F10503DAB242
:1099C0007B699A7266E0BB891A467B699B7AD31AD7
:1099D000A3F110031A4640F20C23C2F200031B68E5
:1099E0009A4254D97B699B7A632B50D87B699A7AC7
:1099F0007B69DA727B699B7A03F10503DAB27B69D2
:109A00009A7244E07B695B7D022B40F08F80FB897A
:109A10001A467B699B7AD31803F10A031A4640F26F
:109A20000C23C2F200031B689A420FD87B699B7A11
:109A3000632B0BD87B699A7A7B69DA727B699B7A94
:109A400003F10503DAB27B699A7223E0FB891A46B7
:109A50007B699B7AD318A3F104031A4640F20C23C6
:109A6000C2F200031B689A4213D37B699B7A002BD6
:109A70000FD07B699A7A7B69DA727B699B7AA3F152
:109A80000503DAB27B699A7203E000BF02E000BF0F
:109A900000E000BF40F20823C2F200031B689A886E
:109AA00040F20823C2F200031B68DB881046194607
:109AB0004FF00202FBF776FA7B685B697A68786898
:109AC00002F1080206CA984731E040F20423C2F2CC
:109AD00000031A6840F20C23C2F200031B68786886
:109AE00011461A46FFF7C2F87B685B687B617B68AA
:109AF0005B697A68786802F1080206CA984716E03E
:109B000040F20423C2F200031B689AB240F20C2315
:109B1000C2F200031B689BB2786811461A4600F037
:109B200065FA04E000BF02E000BF00E000BF07F1FB
:109B30002807BD4680BD00BF90B587B000AF40F29A
:109B4000AA13C2F200031B78DBB2002B00F0D38013
:109B500040F2A813C2F200031B78DBB2012B0BD139
:109B60004FF00100F9F77CFD40F2A813C2F20003A8
:109B70004FF000021A70B7E040F27803C2F200031F
:109B80001B78DBB2012B40F0AF8040F2A813C2F289
:109B900000031B78DBB2002B40F0A68040F2A41338
:109BA000C2F200034FF000021A604FF00003FB8284
:109BB00091E0FA8A40F2B823C2F2000353F822304F
:109BC0009B7D012B40F083804FF00003BB8273E04C
:109BD000FA8A40F2B823C2F2000353F82230BA8A5C
:109BE00002F1080253F8222007F10C0302F10802E7
:109BF00092E8030083E80300FA8A40F2B823C2F235
:109C0000000353F82230BA8A02F1080253F82230D6
:109C10001846FFF745FB3880C0F30F437B803B6855
:109C2000BB6040F2AA13C2F200031B78DBB2002B28
:109C30003ED0B889BA897B89D31A9BB203F101035C
:109C400099B23A8A3C8A3B89E31A9BB200F01EF92A
:109C50000346002B2CD0FA8A40F2B823C2F200034C
:109C600053F82230BA8A02F1080253F8223018461B
:109C7000FFF748FCFA8A40F2B823C2F2000353F817
:109C80002230BA8A02F1080253F82230184600F056
:109C900037F840F20C23C2F200034FF000021A60C2
:109CA00040F2AA13C2F200034FF000021A700EE055
:109CB000BB8A03F10103BB82FA8A40F2B823C2F2E5
:109CC000000353F822301B8BBA8A9A4280D3FB8A56
:109CD00003F10103FB8240F29C13C2F200031B88D4
:109CE000FA8A9A42FFF465AF40F2AA13C2F2000367
:109CF0004FF000021A7007F11C07BD4690BD00BF6F
:109D000080B586B000AF78604FF000037B617B6860
:109D10001B7C03F1FF330C2B00F2B08001A252F840
:109D200023F000BF599D00089F9D0008759D000805
:109D30007D9E0008839D0008919D0008AD9D000850
:109D40004F9E00087D9E00087D9E00085D9E0008D5
:109D50007D9E0008679D00087B685B683B613B69EE
:109D6000DB6898478DE07B685B683B613B699B687B
:109D7000984786E07B685B683B613B69DB68984796
:109D80007FE07B685B683B613B691B69984778E0D3
:109D90007B685B683B613B691B69984771E07B6846
:109DA0005B683B613B69DB6898476AE07B685B689E
:109DB0003B613B695B79002B22D103E07B6903F1B6
:109DC00001037B613B695B8803F1FF331A467B69C2
:109DD0009A420AD93A697B6903F102034FEA830385
:109DE000D3185B681B7B002BE8D03A697B6903F1D1
:109DF00002034FEA8303D3185B681B69984740E06E
:109E00003B699B685B68FB6003E07B6903F10103CE
:109E10007B61FB685B8803F1FF331A467B699A42DA
:109E20000AD9FA687B6903F102034FEA8303D31866
:109E30005B681B7B002BE8D0FA687B6903F10203A7
:109E40004FEA8303D3185B681B69984719E07B6866
:109E50005B683B613B699B69984712E07B685B6884
:109E60003B613B695B891BB2002B09DB3B695B698A
:109E70003A69528992B21046984701E000BF00E06B
:109E800000BF07F11807BD4680BD00BF80B483B096
:109E900000AFF880B9807A803B80BA8840F2042312
:109EA000C2F200031B689A420AD2FB88A3F10503A1
:109EB0001A4640F20423C2F200031B689A4209D8F2
:109EC00040F2A913C2F200034FF000021A704FF0E3
:109ED000000322E03A8840F20C23C2F200031B6820
:109EE0009A4207D87A8840F20C23C2F200031B681A
:109EF0009A4209D240F2A913C2F200034FF00002C5
:109F00001A704FF0000308E040F2A913C2F20003F8
:109F10004FF001021A704FF00103184607F10C07C9
:109F2000BD4680BC704700BF80B483B000AF78608E
:109F300040F2A013C2F200037A681A6000BF40F238
:109F4000A013C2F200031B68002BF8D107F10C0725
:109F5000BD4680BC704700BF80B400AF40F2A01384
:109F6000C2F200031B68002B0BD040F2A013C2F218
:109F700000031B6803F1FF3240F2A013C2F200039A
:109F80001A60BD4680BC704790B587B002AF78605C
:109F90007B685B68FB607B681B897B817B68DB89F6
:109FA0003B81FB68002B02D14FF0000318E04FF01B
:109FB0000000F9F7C1FAFB685A88FB689B8878892A
:109FC00039894FF6FF740094F9F70EF9FB685A8847
:109FD000FB689B8878893989F9F742F94FF00103CA
:109FE000184607F11407BD4690BD00BF80B582B08A
:109FF00000AF786013460A467A803B807B681B89F5
:10A00000A3F102027B889A4263DD7B685B8903F1DE
:10A0100002027B889A425CDA7B689B89A3F1020288
:10A020003B889A4255DD7B68DB8903F102023B885D
:10A030009A424EDA40F2B013C2F200031B8818466F
:10A04000F9F77AFA7B8803F102039AB23B8810464B
:10A0500019464FF001024FF00103F9F7DBF87B8856
:10A0600003F101039AB23B8803F1FF339BB2104620
:10A0700019464FF003024FF00103F9F7CBF83B8884
:10A08000A3F102039BB27A88104619464FF00502ED
:10A090004FF00103F9F7BEF87B8803F1FF339AB262
:10A0A0003B8803F1FF339BB2104619464FF0030281
:10A0B0004FF00103F9F7AEF87B88A3F102039AB2DF
:10A0C0003B88104619464FF001024FF00103F9F7A3
:10A0D000A1F807F10807BD4680BD00BF80B586B076
:10A0E00000AF7B600346FB810B46BB8113467B813F
:10A0F0004FF000033B614FF000037B614FF00C0019
:10A1000001F022FB03463B613B69002B22D03B69F7
:10A11000FA891A803B69BA895A803B697A899A80A0
:10A120003B697A689A604FF0180001F00DFB034616
:10A130007B617B69002B07D07B693A695A607B6938
:10A140004FF00E021A7405E0386901F005FB4FF07C
:10A1500000033B617B69184607F11807BD4680BDC7
:10A1600080B483B000AF78600B467B8040F2B013C0
:10A17000C2F200037A881A8007F10C07BD4680BC42
:10A18000704700BF80B586B000AFF86007F10403E8
:10A1900083E80600FB685B687B61BB887B827B8908
:10A1A0003B827B69002B02D14FF000030DE04FF0A2
:10A1B0000000F9F7C1F97B695A887B699B88788A26
:10A1C000398AF9F74DF84FF00103184607F11807DF
:10A1D000BD4680BD80B500AFFBF7E2F840F28033AA
:10A1E000C2F2000340F21022C2F200021A60FBF732
:10A1F000CDF980BD80B483B000AF78604FF02043CC
:10A200007A68126879684868796889680843796863
:10A21000C968084379680969084379684969084346
:10A220007968896908437968C96908437968096A5E
:10A2300008437968496A08437968896A08437968F4
:10A24000C96A08437968096B014343F822107B68A7
:10A250009B68082B0DD14FF020437A6812684FF0AD
:10A2600020417868006851F8201041F0400143F81F
:10A2700022104FF020437A68126802F101027968D7
:10A28000496B08687968496B49684FEA01110843CE
:10A290007968496B89684FEA012108437968496BFD
:10A2A000C9684FEA014108437968496B09694FEA77
:10A2B000015108437968496B49694FEA01610843D4
:10A2C0007968496B8969014343F822107B68DB6A2E
:10A2D000B3F5804F27D14FF48273CAF200037A6836
:10A2E00012687968896B08687968896B49684FEAF0
:10A2F000011108437968896B89684FEA0121084395
:10A300007968896B09694FEA015108437968896B5B
:10A3100049694FEA016108437968896B896901439A
:10A3200043F8221009E04FF48273CAF200037A68FE
:10A3300012686FF0704143F8221007F10C07BD4618
:10A3400080BC704780B483B000AF78600B46FB7070
:10A35000FB78002B0CD04FF020434FF0204279685F
:10A3600052F8212042F001017A6843F822100EE0F1
:10A370004FF020424FF02043796853F821104FF6F8
:10A38000FE73C0F20F030B40796842F8213007F1E9
:10A390000C07BD4680BC704780B487B000AF7860C2
:10A3A00039604FF000037B614FF000033B614FF0D9
:10A3B0000003FB604FF000037B6186E07B694FF098
:10A3C000010202FA03F33B613B681A683B691340E0
:10A3D000FB60FA683B699A4273D17B681A687B69B3
:10A3E0004FEA43034FF0030101FA03F36FEA03035B
:10A3F0001A407B681A607B681A683B681B791946AB
:10A400007B694FEA430301FA03F31A437B681A603E
:10A410003B681B79012B03D03B681B79022B34D19D
:10A420007B689A687B694FEA43034FF0030101FAA6
:10A4300003F36FEA03031A407B689A607B689A68AB
:10A440003B685B7919467B694FEA430301FA03F3E2
:10A450001A437B689A607B685A687B699BB24FF0AD
:10A46000010101FA03F36FEA03031A407B685A60A3
:10A470007B685A683B689B7919467B699BB201FAF5
:10A4800003F39BB21A437B685A607B68DA687B6986
:10A490009BB24FEA43034FF0030101FA03F36FEA63
:10A4A00003031A407B68DA607B68DA683B68DB7913
:10A4B00019467B694FEA430301FA03F31A437B68A9
:10A4C000DA607B6903F101037B617B690F2B7FF607
:10A4D00075AF07F11C07BD4680BC704780B485B0DE
:10A4E00000AF78600B467B804FF00003FB737B6806
:10A4F0001A697B881340002B03D04FF00103FB73D4
:10A5000002E04FF00003FB73FB7B184607F11407D2
:10A51000BD4680BC704700BF80B483B000AF786098
:10A520000B467B807B687A881A8307F10C07BD464F
:10A5300080BC704780B483B000AF78600B467B80EE
:10A540007B687A885A8307F10C07BD4680BC704748
:10A5500080B485B000AF786013460A467A807B707D
:10A560004FF00003FB604FF00003BB607A787B88FC
:10A5700003F007034FEA830302FA03F3FB607B88CF
:10A580004FEAD3039BB21A467B884FEAD3039BB2B0
:10A5900019467B6801F1080153F821107B8803F00C
:10A5A00007034FEA83034FF00F0000FA03F36FEA4B
:10A5B000030319407B6802F1080243F822107B88EC
:10A5C0004FEAD3039BB21A467B6802F1080253F8A4
:10A5D0002220FB681343BB607B884FEAD3039BB206
:10A5E0001A467B6802F10802B96843F8221007F1A5
:10A5F0001407BD4680BC704780B485B000AF78605A
:10A6000040F2B413C2F200031B68002B08D140F2E1
:10A61000B413C2F2000340F6E032C2F200021A6044
:10A6200040F2B413C2F200031B68FB6040F2B413A3
:10A63000C2F200031A687B68D21840F2B413C2F267
:10A6400000031A60FB68184607F11407BD4680BC7A
:10A65000704700BF80B58AB000AF786039604FF0B6
:10A660000003FB844FF000037B844FF00403BB84A2
:10A670004FF49053C0F27A03FB617B689B88FB84A4
:10A68000FB8C23F03F03FB8407F10C031846FAF719
:10A69000D1FA7B69FB61FA694DF68363C4F21B331F
:10A6A000A3FB02134FEA93437B84FA8C7B8C134306
:10A6B000FB847B68FA8C9A807B681B889BB223F0B2
:10A6C00001039AB27B681A804FF00003FB843B6859
:10A6D0001A6848F2A063C0F201039A4218D83B6896
:10A6E0001B684FEA4303FA69B2FBF3F3BB84BB8CEC
:10A6F000032B02D84FF00403BB84FA8CBB8C1343AA
:10A70000FB847B8C03F101039AB27B681A844BE0D3
:10A710003B68DA884BF6FF739A420AD13B681A68A5
:10A7200013464FEA43039B18FA69B2FBF3F3BB8469
:10A7300010E03B681A6813464FEA83039B184FEA00
:10A7400083029B18FA69B2FBF3F3BB84BB8C43F41E
:10A750008043BB84BB8C4FEA03534FEA1353002B57
:10A7600003D1BB8C43F00103BB84BA8CFB8C134335
:10A770009BB26FEA43436FEA5343FB847B8C4FF4F5
:10A78000967202FB03F244F6D353C1F2620383FBD9
:10A7900002134FEAA3114FEAE273CB1A9BB203F103
:10A7A00001039AB27B681A847B68FA8C9A837B686F
:10A7B0001B889BB243F001039AB27B681A807B68C6
:10A7C0001B88FB84FB8C23F4816323F00203FB844E
:10A7D0003B689A883B685B8913439AB2FB8C1343AE
:10A7E000FB847B68FA8C1A803B689A893B681B89DA
:10A7F00013439AB27B681A8107F12807BD4680BDD2
:10A8000080B485B000AF78604FF00003FB604FF478
:10A810007053C4F20103FB607B689B79002B78D0F6
:10A820004FF47053C4F201034FF47052C4F20102AA
:10A8300011687A6812686FEA02020A401A604FF4DF
:10A840007053C4F201034FF47052C4F20102516814
:10A850007A6812686FEA02020A405A607B681B79C4
:10A86000FA68D318FB60FB68FA6811687A681268A6
:10A870000A431A604FF47053C4F201034FF470524C
:10A88000C4F2010291687A6812686FEA02020A4013
:10A890009A604FF47053C4F201034FF47052C4F243
:10A8A0000102D1687A6812686FEA02020A40DA602F
:10A8B0007B685B79102B1AD14FF47053C4F20103FB
:10A8C0004FF47052C4F2010291687A6812680A4328
:10A8D0009A604FF47053C4F201034FF47052C4F203
:10A8E0000102D1687A6812680A43DA601FE04FF407
:10A8F0007053C4F20103FB607B685B79FA68D3187C
:10A90000FB60FB68FA6811687A6812680A431A608B
:10A910000DE07B681B79FA68D318FB60FB68FA6866
:10A9200011687A6812686FEA02020A401A6007F139
:10A930001407BD4680BC704780B485B000AF786016
:10A940004FF00003FB734FF00003BB604FF47053F4
:10A95000C4F201031A687B681340BB604FF4705364
:10A96000C4F201035A697B681340002B06D0BB6810
:10A97000002B03D04FF00103FB7302E04FF0000304
:10A98000FB73FB7B184607F11407BD4680BC70477C
:10A9900080B483B000AF78604FF47053C4F2010309
:10A9A0007A685A6107F10C07BD4680BC704700BF4A
:10A9B00080B483B000AF78604FF46D43CEF20003F3
:10A9C0007A6842F0BF6242F40032DA6007F10C07A5
:10A9D000BD4680BC704700BF80B485B000AF7860D2
:10A9E0004FF00003FB734FF00003BB734FF00F03F6
:10A9F0007B737B68DB78002B45D04FF46D43CEF240
:10AA00000003DB686FEA030303F4E0634FEA1323F8
:10AA1000FB73FB7BC3F10403BB737A7BFB7B42FAC2
:10AA200003F37B737B685B781A46BB7B02FA03F304
:10AA3000FB737B689A787B7B1340DAB2FB7B134312
:10AA4000FB73FB7B4FEA0313FB734FF46143CEF2BE
:10AA500000037A6812789B18FA7B83F800234FF47E
:10AA60006143CEF200037A6812784FEA5212D2B2F2
:10AA70007968097801F01F014FF0010000FA01F137
:10AA800043F8221014E04FF46143CEF200037A68D9
:10AA900012784FEA5212D2B27968097801F01F0198
:10AAA0004FF0010000FA01F102F1200243F82210F8
:10AAB00007F11407BD4680BC704700BF80B483B067
:10AAC00000AF786039604FF46D43CEF200033A680E
:10AAD00022F0604222F07F0279680A439A6007F10F
:10AAE0000C07BD4680BC704780B400AF40F2843391
:10AAF000C2F200031846BD4680BC704780B500AF67
:10AB000040F28433C2F200035B6B1846FFF714FF78
:10AB10000346002B24D040F28433C2F200039B6C26
:10AB2000DBB218464FF00701F9F744F8034603F08B
:10AB30000703002B0CD000F01BF840F28433C2F264
:10AB400000039B6CDBB218464FF00701F9F756F88B
:10AB500040F28433C2F200035B6B1846FFF718FF24
:10AB600080BD00BF80B500AFF8F7D6FF80BD00BF45
:10AB700080B500AF40F2BC13C2F200034FF00002F8
:10AB80001A6040F2C413C2F200034FF000021A60D0
:10AB900040F28433C2F200039B6CDBB218464FF0E4
:10ABA0004001F9F743FB0346DBB25BB2002B80F2B6
:10ABB000D9804FF00200FFF7B7F940F28433C2F2B8
:10ABC00000039B6CDBB218464FF040014FF00002CF
:10ABD000F9F716FA40F28433C2F200039B6CDBB241
:10ABE00018464FF04F01F9F7ABFC03461A4640F206
:10ABF000BC13C2F200031A6040F28433C2F20003B5
:10AC00009B6CDBB218464FF04D01F9F799FC0346F7
:10AC10001A4640F2C413C2F200031A6040F28433B1
:10AC2000C2F200039B6CDBB218464FF05101F9F7FA
:10AC300087FC40F2BC13C2F200031B689AB240F2D8
:10AC4000C413C2F200031B689BB210461946F8F702
:10AC500063F803461A4640F20423C2F200031A6066
:10AC600040F2BC13C2F200031B689AB240F2C41354
:10AC7000C2F200031B689BB210461946F8F792F81F
:10AC800003461A4640F20C23C2F200031A6040F257
:10AC9000AA13C2F200034FF001021A7040F284338B
:10ACA000C2F200039B6CDBB218464FF04B014FF031
:10ACB0000102F9F7A5F940F28433C2F200039B6C5C
:10ACC000DBB218464FF00B014FF00702F9F798F985
:10ACD00040F28433C2F200039B6CDBB218464FF0A3
:10ACE0004B014FF00002F9F78BF94FF00200FFF72C
:10ACF0001BF940F28433C2F200039B6CDBB21846AE
:10AD00004FF040014FF00102F9F77AF94FF00200DD
:10AD1000FFF70AF940F28433C2F200039B6CDBB206
:10AD200018464FF04B01F9F781FA0346202B19D052
:10AD300040F28433C2F200039B6CDBB218464FF042
:10AD40004B014FF00102F9F75BF940F28433C2F294
:10AD500000039B6CDBB218464FF04B014FF0000232
:10AD6000F9F74EF980BD00BF81F0004102E000BF5D
:10AD700083F0004330B54FEA41044FEA430594EABB
:10AD8000050F08BF90EA020F1FBF54EA000C55EAF6
:10AD9000020C7FEA645C7FEA655C00F0E2804FEAC7
:10ADA0005454D4EB5555B8BF6D420CDD2C4480EAA9
:10ADB000020281EA030382EA000083EA010180EAD9
:10ADC000020281EA0303362D88BF30BD11F0004F27
:10ADD0004FEA01314FF4801C4CEA113102D040425D
:10ADE00061EB410113F0004F4FEA03334CEA133398
:10ADF00002D0524263EB430394EA050F00F0A780B0
:10AE0000A4F10104D5F1200E0DDB02FA0EFC22FAAA
:10AE100005F2801841F1000103FA0EF2801843FA9E
:10AE200005F359410EE0A5F120050EF1200E012A8F
:10AE300003FA0EFC28BF4CF0020C43FA05F3C018CD
:10AE400051EBE37101F0004507D54FF0000EDCF146
:10AE5000000C7EEB00006EEB0101B1F5801F1BD3EF
:10AE6000B1F5001F0CD349085FEA30004FEA3C0CF3
:10AE700004F101044FEA445212F5800F80F09A80E9
:10AE8000BCF1004F08BF5FEA500C50F1000041EBED
:10AE9000045141EA050130BD5FEA4C0C404141EBF1
:10AEA000010111F4801FA4F10104E9D191F0000F18
:10AEB00004BF01460020B1FA81F308BF2033A3F19B
:10AEC0000B03B3F120020CDA0C3208DD02F1140C92
:10AED000C2F10C0201FA0CF021FA02F10CE002F1CD
:10AEE0001402D8BFC2F1200C01FA02F120FA0CFCC6
:10AEF000DCBF41EA0C019040E41AA2BF01EB04510F
:10AF0000294330BD6FEA04041F3C1CDA0C340EDC0C
:10AF100004F11404C4F1200220FA04F001FA02F34F
:10AF200040EA030021FA04F345EA030130BDC4F10D
:10AF30000C04C4F1200220FA02F001FA04F340EA02
:10AF40000300294630BD21FA04F0294630BD94F0B3
:10AF5000000F83F4801306BF81F480110134013D9A
:10AF60004EE77FEA645C18BF7FEA655C29D094EA0B
:10AF7000050F08BF90EA020F05D054EA000C04BF89
:10AF80001946104630BD91EA030F1EBF0021002074
:10AF900030BD5FEA545C05D14000494128BF41F013
:10AFA000004130BD14F580043CBF01F5801130BD77
:10AFB00001F0004545F0FE4141F470014FF0000002
:10AFC00030BD7FEA645C1ABF194610467FEA655CB3
:10AFD0001CBF0B46024650EA013406BF52EA033555
:10AFE00091EA030F41F4002130BD00BF90F0000F43
:10AFF00004BF0021704730B54FF4806404F132047F
:10B000004FF000054FF0000150E700BF90F0000F37
:10B0100004BF0021704730B54FF4806404F132045E
:10B0200010F0004548BF40424FF000013EE700BF2E
:10B0300042004FEAE2014FEA31014FEA02701FBFBE
:10B0400012F07F4393F07F4F81F06051704792F090
:10B05000000F14BF93F07F4F704730B54FF460740A
:10B0600001F0004521F0004120E700BF50EA010255
:10B0700008BF704730B54FF000050AE050EA010202
:10B0800008BF704730B511F0004502D5404261EB72
:10B0900041014FF4806404F132045FEA915C3FF4B3
:10B0A000DCAE4FF003025FEADC0C18BF03325FEA4C
:10B0B000DC0C18BF033202EBDC02C2F1200300FA01
:10B0C00003FC20FA02F001FA03FE40EA0E0021FA26
:10B0D00002F11444C1E600BF70B54FF0FF0C4CF410
:10B0E000E06C1CEA11541DBF1CEA135594EA0C0FC6
:10B0F00095EA0C0F00F0DEF82C4481EA030621EA01
:10B100004C5123EA4C5350EA013518BF52EA03353B
:10B1100041F4801143F4801338D0A0FB02CE4FF0ED
:10B120000005E1FB02E506F00042E0FB03E54FF01D
:10B130000006E1FB03569CF0000F18BF4EF0010E15
:10B14000A4F1FF04B6F5007F64F5407404D25FEA11
:10B150004E0E6D4146EB060642EAC62141EA5551C4
:10B160004FEAC52040EA5E504FEACE2EB4F1FD0C06
:10B1700088BFBCF5E06F1ED8BEF1004F08BF5FEA84
:10B18000500E50F1000041EB045170BD06F0004636
:10B1900046EA010140EA020081EA0301B4EB5C04E3
:10B1A000C2BFD4EB0C0541EA045170BD41F48011DB
:10B1B0004FF0000E013C00F3AB8014F1360FDEBF00
:10B1C000002001F0004170BDC4F10004203C35DADC
:10B1D0000C341BDC04F11404C4F1200500FA05F35F
:10B1E00020FA04F001FA05F240EA020001F0004200
:10B1F00021F0004110EBD37021FA04F642EB060176
:10B200005EEA430E08BF20EAD37070BDC4F10C049F
:10B21000C4F1200500FA04F320FA05F001FA04F263
:10B2200040EA020001F0004110EBD37041F100014F
:10B230005EEA430E08BF20EAD37070BDC4F120055A
:10B2400000FA05F24EEA020E20FA04F301FA05F2C2
:10B2500043EA020321FA04F001F0004121FA04F26A
:10B2600020EA020000EBD3705EEA430E08BF20EA3A
:10B27000D37070BD94F0000F0FD101F00046400074
:10B2800041EB010111F4801F08BF013CF7D041EAF6
:10B29000060195F0000F18BF704703F000465200FA
:10B2A00043EB030313F4801F08BF013DF7D043EACB
:10B2B0000603704794EA0C0F0CEA135518BF95EA81
:10B2C0000C0F0CD050EA410618BF52EA4306D1D108
:10B2D00081EA030101F000414FF0000070BD50EA27
:10B2E000410606BF1046194652EA430619D094EAB1
:10B2F0000C0F02D150EA013613D195EA0C0F05D19B
:10B3000052EA03361CBF104619460AD181EA0301EE
:10B3100001F0004141F0FE4141F470014FF00000A6
:10B3200070BD41F0FE4141F4780170BD70B54FF041
:10B33000FF0C4CF4E06C1CEA11541DBF1CEA1355C1
:10B3400094EA0C0F95EA0C0F00F0A7F8A4EB0504A3
:10B3500081EA030E52EA03354FEA013100F088809A
:10B360004FEA03334FF0805545EA131343EA126363
:10B370004FEA022245EA111545EA10654FEA002618
:10B380000EF000419D4208BF964244F1FD0404F5D1
:10B39000407402D25B084FEA3202B61A65EB03052D
:10B3A0005B084FEA32024FF480104FF4002CB6EBEA
:10B3B000020E75EB030E22BFB61A754640EA0C006A
:10B3C0005B084FEA3202B6EB020E75EB030E22BFAA
:10B3D000B61A754640EA5C005B084FEA3202B6EBEB
:10B3E000020E75EB030E22BFB61A754640EA9C00AA
:10B3F0005B084FEA3202B6EB020E75EB030E22BF7A
:10B40000B61A754640EADC0055EA060E18D04FEA37
:10B41000051545EA16754FEA06164FEAC30343EAD7
:10B4200052734FEAC2025FEA1C1CC0D111F4801FA4
:10B430000BD141EA00014FF000004FF0004CB6E79D
:10B4400011F4801F04BF01430020B4F1FD0C88BF3C
:10B45000BCF5E06F3FF6AFAEB5EB030C04BFB6EB47
:10B46000020C5FEA500C50F1000041EB045170BD3A
:10B470000EF0004E4EEA113114EB5C04C2BFD4EB67
:10B480000C0541EA045170BD41F480114FF0000EEB
:10B49000013C90E645EA060E8DE60CEA135594EA67
:10B4A0000C0F08BF95EA0C0F3FF43BAF94EA0C0F6A
:10B4B0000AD150EA01347FF434AF95EA0C0F7FF4DF
:10B4C00025AF104619462CE795EA0C0F06D152EA33
:10B4D00003353FF4FDAE1046194622E750EA410617
:10B4E00018BF52EA43067FF4C5AE50EA41047FF428
:10B4F0000DAF52EA43057FF4EBAE12E74FF0FF3C8D
:10B5000006E000BF4FF0010C02E000BF4FF0010C5D
:10B510004DF804CD4FEA410C7FEA6C5C4FEA430CD6
:10B5200018BF7FEA6C5C1BD001B050EA410C0CBF25
:10B5300052EA430C91EA030F02BF90EA020F002087
:10B54000704710F1000F91EA030F58BF994208BFEE
:10B5500090422CBFD8176FEAE37040F001007047AB
:10B560004FEA410C7FEA6C5C02D150EA013C07D102
:10B570004FEA430C7FEA6C5CD6D152EA033CD3D04D
:10B580005DF8040B704700BF8446104662468C4647
:10B590001946634600E000BF01B5FFF7B7FF00287A
:10B5A00048BF10F1000F01BD4DF808EDFFF7F4FFA3
:10B5B0000CBF012000205DF808FB00BF4DF808ED2E
:10B5C000FFF7EAFF34BF012000205DF808FB00BF51
:10B5D0004DF808EDFFF7E0FF94BF012000205DF873
:10B5E00008FB00BF4DF808EDFFF7CEFF94BF012028
:10B5F00000205DF808FB00BF4DF808EDFFF7C4FF21
:10B6000034BF012000205DF808FB00BF4FEA410273
:10B6100012F5001215D211D56FF47873B3EB6252A4
:10B6200012D94FEAC12343F0004343EA505311F0CB
:10B63000004F23FA02F018BF404270474FF000005D
:10B64000704750EA013005D111F0004008BF6FF09B
:10B65000004070474FF00000704700BF4A0011D211
:10B6600012F5001211D20DD56FF47873B3EB62525C
:10B670000ED44FEAC12343F0004343EA505323FA68
:10B6800002F070474FF00000704750EA013002D1DD
:10B690004FF0FF3070474FF00000704753EC102B15
:10B6A00070B5C3F30A5423F07F45A4F2FF3125F4AB
:10B6B0007005002BACBF01234FF0FF33132945F475
:10B6C00080150DDC002938DB4FF4002242FA01F22C
:10B6D0005519C1F1140125FA01F000FB03F070BD0A
:10B6E0001E290ED8332911DDA4F21340A4F23344ED
:10B6F00005FA00F502FA04F245EA020000FB03F045
:10B7000070BD51EC100BFFF781FF70BDA4F2134424
:10B710004FF0004626FA04F6B218C1F1340128BFF2
:10B720000135202918BF22FA01F005FA04F508BFF7
:10B730000020284300FB03F070BDB1F1FF3F0CBFB8
:10B740001846002070BD00BF024B0146186800F08B
:10B750000BB800BF28010020024B0146186801F019
:10B76000B3BC00BF2801002070B5CD1C25F0030537
:10B7700008350C2D38BF0C25002D06462DDB8D42DB
:10B780002BD31D4B1B681C469CB12268501B0DD44B
:10B790000B2802D92060241817E0A34203D1606867
:10B7A000154A10601DE0616859601AE0234664681C
:10B7B000EAE72946304600F033F8431C01460CD036
:10B7C000CC1C24F003048C4201D1256009E03046F2
:10B7D000611A00F025F80130F7D10C20306000200C
:10B7E00070BD04F10B01231D21F00700C31A02D024
:10B7F0005A42E25070BD70BDB801002010B5002360
:10B80000934203D0CC5CC4540133F9E710BD8218D5
:10B810000346934202D003F8011BFAE77047000089
:10B8200038B5064C0023054608462360FEF7E4FEC3
:10B83000431C02D1216801B1296038BDD803002022
:10B840000EB400B59CB01DAB029006906FF00040A6
:10B85000049007904FF402710A4853F8042BADF896
:10B8600014104FF6FF71ADF816100068019302A98D
:10B8700000F086F8029B00221A701CB05DF804EB01
:10B8800003B0704728010020034611F8012B03F88C
:10B89000012B002AF9D17047034613F8012B002A27
:10B8A000FBD1181A0138704730B5013903461C46E0
:10B8B0003AB111F8015F03F8015B013A1C46002D13
:10B8C000F5D199188C4203D0002204F8012BF9E736
:10B8D00030BD2DE9F8439368064689461446002B8F
:10B8E00041D1928912F4906F3DD061692369276834
:10B8F000032502204D43FF1A95FBF0F5791C02F455
:10B900008062A94211B2A8BF3D18304679B12946DC
:10B91000FFF72AFF8046A0B13A462169FFF76EFF84
:10B92000A38923F4906040F08002A28113E01946BD
:10B930002A4601F003FF804668B93046216901F0CC
:10B94000C3FBA0890C2340F0400233604FF0FF306E
:10B95000A281BDE8F88308EB07016561ED1BC4F81F
:10B9600010802160A560A368002B06DD206800F828
:10B97000019BA2682060511EA1600020BDE8F883F1
:10B980002DE9F0479CB00D4603938B8903F08001AD
:10B9900014460AB2064662B12B6953B94021FFF73B
:10B9A000E3FE2860286110B90C213160D3E040200B
:10B9B000686100272021302209978DF829108DF821
:10B9C0002A2023461F4613F8010B28B9B7EB040AB7
:10B9D00016D04FF000090DE02528F3D1F6E73046E8
:10B9E00014F809102A46FFF774FF013000F0AC800C
:10B9F00009F10109D145F2DB099901EB0A0209922B
:10BA00003B78002B00F0A08000244FF0FF3004941E
:10BA10000794059006948DF853401A9407F1010994
:10BA20004C464F4F21783846052201F095FB09F12D
:10BA30000109049B30B1C41B012707FA04F73B43FB
:10BA40000493EDE7D90602D520218DF853101A078B
:10BA500002D52B228DF8532020782A2802D0079B6C
:10BA600027460EE0039A1768101D002F039001DB94
:10BA7000079704E0794243F00203079104930134ED
:10BA80000AE03C46013721783039092903D80A24D5
:10BA900004FB0313F5E7079322782E2A19D1607867
:10BAA0002A2809D103980368021D0234002B03924F
:10BAB000B8BF4FF0FF330BE0671C00233C46013753
:10BAC00021783039092903D80A2404FB0313F5E748
:10BAD0000593244F21783846032201F03DFB38B10D
:10BAE000049BC71B402101FA07F10B430493013467
:10BAF00014F8011B1C488DF82810062201F02CFBBD
:10BB000088B11A4A32B9039FFB1D23F007000830A1
:10BB1000039014E003A90091304604A92A46144B6F
:10BB200000F0C4F807E003A8009004A930462A46B4
:10BB30000F4B00F07BFBB0F1FF3F804604D0099A29
:10BB400002EB080109913CE7AB8903F0400002B227
:10BB50000AB9099801E04FF0FF301CB0BDE8F0874A
:10BB6000B8410108BE410108C2410108ADBC00084E
:10BB7000D3B800082DE9F04F10EE906A85B0002E82
:10BB800010EE108A0F469346DDF83890DDF83CA0A1
:10BB900003DA06F100462D2100E00021BAF1660F1C
:10BBA00019700AD0BAF1460F07D0BAF1650F02D06A
:10BBB000BAF1450F03D1013701E0032100E0022172
:10BBC00003AC02AB019435464446009345EC104B60
:10BBD0003A464B4600F0D8FCBAF1670F044602D053
:10BBE000BAF1470F02D11BF0010F28D0BAF1660F4E
:10BBF00004EB070502D0BAF1460F10D120783028A7
:10BC00000AD14046314600220023FFF7CDFC18B987
:10BC1000C7F10107C9F80070D9F80020AD184046F7
:10BC2000314600220023FFF7BFFC00B103950399C2
:10BC3000A94204D2302301F8013B0391F7E7039BAB
:10BC4000109A181B1060204605B0BDE8F08F03461F
:10BC500073B5002903F8022B02DA49422D2200E0D5
:10BC60002B22092942701A4619DD0DF106040A2615
:10BC700091FBF6F506FB15113031092D234604F82A
:10BC800001192946F3DC303103F8011D0DF10701DC
:10BC90008B4209D213F8011B02F8011BF6E7302290
:10BCA00089181A7059709A1C101A7CBD2DE9F04F32
:10BCB0008DB00C4616461F46DDF85880054601F04B
:10BCC00047FAD0F800A05046FFF7E6FD0790D8F8F5
:10BCD000000094F818B00023C11D0A9321F0070357
:10BCE00003F10802C8F8002093ED007B84ED127B7D
:10BCF00094ED120B01F046FD012819D1D4E912018F
:10BD000000220023FFF75AFC10B12D2284F84320B3
:10BD100099499A48BBF1470F8CBF804688462168F5
:10BD2000032321F00400236120604FF0000984E028
:10BD300094ED120B01F026FD10B991499148E9E705
:10BD40006168481C01D1062007E0BBF1670F02D0F3
:10BD5000BBF1470F02D109B90120606023680020C0
:10BD600043F480620AA909AB8DE8080802910390A8
:10BD7000226094ED120B284661680DF12303FFF752
:10BD8000F9FEBBF1670F804602D0BBF1470F09D126
:10BD9000099BD91C02DB6268934231DDABF1020CD6
:10BDA0005FFA8CFBBBF1650F099912D801395A462D
:10BDB00004F150000991FFF74AFF0A9A8318012AFB
:10BDC0008146236102DC2168CA0730D5581C2061F6
:10BDD0002DE0BBF1660F15D10029636808DD2161F4
:10BDE00013B92268D0071ED50133C91821611AE0A2
:10BDF00013B92068C10701D59A1C13E0012211E094
:10BE00004FF0670B09980A9B984205DB2168206177
:10BE1000CA0708D5421C05E00028D4BFC0F10200C3
:10BE200001201A18226109984FF00009A0659DF8B9
:10BE3000232012B12D2384F8433000972846214651
:10BE40000BAA334600F082F9013002D14FF0FF30E7
:10BE500079E1236813F480620DD191462169894507
:10BE600022DA284618F809103246B8470130EDD0DA
:10BE700009F10109F2E7BBF1650F40F2F180D4E965
:10BE8000120100220023FFF78FFB00282DD0302164
:10BE900028463246B8470130D8D00A9B099A9A42C0
:10BEA00007DB2168C80704D42068830700F14881B4
:10BEB00040E107980AEB000BDA4507D028461AF84C
:10BEC000011B3246B8470130F6D1BFE74FF00008FA
:10BED0000A9B5A1E9045E7DA2846A17E3246B847AB
:10BEE0000130B3D008F10108F2E70999002938DCE4
:10BEF000302128463246B8470130A7D0099A22B9E6
:10BF00000A9911B92068C107CED5079B0AEB030B2C
:10BF1000DA4507D028461AF8011B3246B8470130E7
:10BF2000F6D193E74FF00009099A5142894508DAA2
:10BF30002846A17E3246B847013087D009F1010971
:10BF4000F2E74FF000090A988145ADDA284618F863
:10BF500009103246B84701303FF478AF09F10109C2
:10BF6000F1E7A06D0A9B8342B4BF9C468446BCF1B6
:10BF7000000F09DC002329E0C9410108CD41010877
:10BF8000D1410108D5410108C1460CEB080319F85D
:10BF9000011B0593CDF818C028463246B84701303A
:10BFA000059BDDF818C03FF451AF9945EFD1E1E7AB
:10BFB000CDF818C02846A17E05933246B847013017
:10BFC000DDF818C005983FF441AF431CD4F85890F1
:10BFD0002CEAEC72C2EB09018B42E9DB0A98099B5F
:10BFE00083420FDB2268D2070CD40A98099BC8440D
:10BFF000C21AC9EB00099145A8BF9146B9F1000FDB
:10C000000DDC18E007990AEB010BDA45EDD0284664
:10C010001AF8011B3246B8470130F6D116E708EB93
:10C02000090A284618F8011B3246B84701303FF488
:10C030000DAFD045F5D14FF0000808E02846A17EAD
:10C040003246B84701303FF401AF08F101080999C1
:10C050000A9829EAE972431A991A8845EEDB23E720
:10C060000A99012998F800100ADCDB0708D4284651
:10C070003246B84701303FF4E9AE4FF0000848E0DF
:10C0800028463246B84701303FF4E0AE07980AEB45
:10C09000000BDA4507D028461AF8011B3246B8478C
:10C0A0000130F6D1D2E6D4E9120100220023FFF7D5
:10C0B0007BFA10B14FF000081AE04FF0000A0A991D
:10C0C000481E8245D9DA08EB0A02284651783246E2
:10C0D000B84701303FF4BAAE0AF1010AEFE728464B
:10C0E000A17E3246B84701303FF4B0AE08F10108F6
:10C0F0000A9B5A1E9045F2DBBFE704EB0803284673
:10C1000093F850103246B84701303FF49FAE08F123
:10C110000108C845F1DBC7E62846617E3246B847CC
:10C1200001303FF493AE08F10108E2680B9BD11A8D
:10C130008845F1DBE0680B9A9042B8BF104602E0F8
:10C140004FF00008F1E70DB0BDE8F08F2DE9F047A2
:10C15000154699468A680B69DDF820A09A42A8BF67
:10C1600013462B60804691F843000C4608B1591CD9
:10C1700029602668B20602D52A68931C2B602068C5
:10C1800010F0060618D094F8437020683E1C18BFC3
:10C19000012683061AD5A119302281F8432094F88C
:10C1A0004530023681F8443010E04046617E4A4610
:10C1B000D047013006D00136E1682A688B1A9E42CA
:10C1C000F3DBE0E74FF0FF30BDE8F0870027B74230
:10C1D00009DAE119404691F843104A46D047013048
:10C1E000F0D00137F3E721682868E668236901F099
:10C1F0000602042A08BFC0EB0605A6680CBF25EAA4
:10C20000E57500259E42C4BFC3EB0603ED1800266A
:10C21000AE4207DA4046A17E4A46D0470130D1D02F
:10C220000136F5E70020BDE8F08700002DE9F04376
:10C230000C4685B0257E0C996E2D90460746994692
:10C2400004F1430200F0AA8012D8632D24D009D84B
:10C25000002D00F0BB80582D40F0CB8084F8455075
:10C26000824D57E0642D20D0692D40F0C2801CE043
:10C27000732D00F0AF8009D86F2D2FD0702D40F0B6
:10C28000B880256845F0200626603FE0752D25D052
:10C29000782D40F0AE8039E00868021D0A60016820
:10C2A00004F1420684F84210A7E020680B6810F001
:10C2B000800F02D01E1D0E6008E003F1040510F08F
:10C2C000400F0D6002D0B3F9001000E0196800299A
:10C2D0003CDA2D20494284F8430037E025680E6897
:10C2E00015F0800F02D0331D0B6007E006F104004B
:10C2F00015F0400F086001D0318800E03168267EDB
:10C300005A4D6F2E14BF0A2308231BE07820584D86
:10C3100084F8450020680B6810F0800F03F10406D4
:10C320000E6003D1410601D5198800E01968C607DF
:10C3300044BF40F02000206019B9206820F020039D
:10C3400023601023002084F8430001E0474D0A23B6
:10C350006668002EA66003DB206820F004002060E1
:10C3600001B96EB104F14200B1FBF3FE03FB1E11F3
:10C370000646695C00F8011971460029F4D100E015
:10C380001646921B082B22613CD12368D80739D569
:10C390006068904236DC511C616033E026680B68AF
:10C3A00016F0800F05D01E1D0E60196860690860C8
:10C3B0000CE003F1040016F0400F086003D0186889
:10C3C0006369038002E061691E68316000232361B4
:10C3D000164617E00E68321D0A6036683046FFF7D1
:10C3E0005BFA63682061984288BF236120696060BE
:10C3F00005E004F1420684F8425001232361002144
:10C4000084F84310CDF800903846214603AA4346ED
:10C41000FFF79CFE013002D14FF0FF3022E00025F3
:10C420002269954207DA3846715D4246C8470130B5
:10C43000F2D00135F4E72168890705D4E068039953
:10C440008842B8BF08460DE00025E068039BC21A89
:10C450009542F3DA3846617E4246C8470130DBD068
:10C460000135F2E705B0BDE8F08300BFD94101080E
:10C47000EA4101082DE9F84F02690B699A42054625
:10C480007EDBD81C86008A195C1EAB19506802F14D
:10C4900004095A68461CB2FBF6F601F1140805F1CE
:10C4A0001407002E39D000203A464346824653F8FE
:10C4B00004EB1FFA8EFC06FB0C0C4FEA1E4006FB39
:10C4C00000FB0BEB1C4ED2F800B04FEA1E401AFAEC
:10C4D0008BFA1FFA8EFE1FFA8CFCCCEB0A0CCEEB0B
:10C4E0001B4A0AEB2C4E1FFA8CFC4FEA2E4A4B4596
:10C4F0004CEA0E4E42F804EBD9D9221D05EB82031B
:10C50000586850B9BB421A4601D82C6105E0106842
:10C51000043B0028F9D1013CF4E7284601F03EF83D
:10C5200000282ADB01363B46002058F804CB1A6865
:10C530001FFA8CF11FFA82FAC1EB0A0109184FEABF
:10C540001C40C0EB124202EB214289B2101441EAB6
:10C550000242C84543F8042BE7D9231D05EB8303AA
:10C56000586850B9BB42194601D82C6105E00A68E9
:10C57000043B002AF9D1013CF4E73046BDE8F88FCE
:10C580000020BDE8F88F00002DE9F04F456A99B012
:10C5900083460B910C921493229C8DED020B45B9AE
:10C5A0001020FFF7D1F8CBF82400456085600560C6
:10C5B000C560DBF82430196861B15868012202FABD
:10C5C00000F648608E60584600F009FEDBF8241043
:10C5D00000230B600398002805DA0126266020F06E
:10C5E0000044039401E000222260039C9849984B88
:10C5F000214099421CD11499029B42F20F720A60A9
:10C600003BB9944E9448C4F31304002C18BF304631
:10C6100000E09048239E002E00F04E85C27812B1B3
:10C6200000F1080100E0C11C239E316000F044BD10
:10C63000DDE902890022404649460023FEF7B4FFA7
:10C6400058B1149E01233360239E002E00F03185E3
:10C6500082483060013800F02FBD584649EC108BFD
:10C6600017A916AA01F018F8C4F30A55824665B155
:10C6700029F07F4424F4700242F07F51404641F497
:10C680004011A5F2FF3600221CE01798169A6FF4AD
:10C69000826116188E420ADB7149029A06F2124034
:10C6A0008B1B22FA00F004FA03F4204304E06D4CE3
:10C6B000029DA31B05FA03F0FEF798FC013EA1F1D1
:10C6C000F87101221592684B0022FEF751FB5AA324
:10C6D000D3E90023FEF700FD59A3D3E90023FEF7B9
:10C6E00049FB044630460D46FEF790FC56A3D3E9BD
:10C6F0000023FEF7F1FC02460B4620462946FEF7D2
:10C7000039FB04460D46FEF781FF2946814600228B
:10C7100020460023FEF752FF58B14846FEF776FC4C
:10C7200002460B4620462946FEF73EFF08B909F1AE
:10C73000FF39B9F1160F0ED84C4800EBC903D3E905
:10C740000001DDE90223FEF757FF28B1002209F1BD
:10C75000FF39119201E00120119016998E1B741E71
:10C7600004D5654200200595069002E0002306945A
:10C770000593B9F1000F08DB069DCDF8409005EB5D
:10C78000090000230690099308E0059AC9F1000604
:10C79000C9EB020100240591099610940B9A092A0D
:10C7A00027D8052A03DD111F0B91002500E0012584
:10C7B0000B9EB41E032C21D8DFE804F0060F020400
:10C7C000012302E0012009E000230C9A0A93002AC9
:10C7D0001EDD0892049213461FE000200C9C0A9074
:10C7E00004EB0900431C002B0890049315DC012383
:10C7F00013E0012500220B920A9501E001260A961A
:10C800004FF0FF3100260891049112230C9604E0AA
:10C810000121089104910B460C91DBF82440002083
:10C820006060042101F114029A4221D86068421C20
:10C8300062604900F6E700BF61436F63A787D23F9C
:10C84000B3C8608B288AC63FFB799F501344D33FFF
:10C850000000F07F04420108FB4101080942010881
:10C860000EFCFFFFEEFBFFFF0000F83F184201083F
:10C870006168584600F07EFC2060DBF82440049993
:10C8800023680E29079300F25E81002D00F05B8182
:10C890009DED027BB9F1000F8DED127B33DD9D4BD9
:10C8A00009F00F004FEA291603EBC001F206D1E9A7
:10C8B00000450CD5984F51EC170BD7E90823FEF72C
:10C8C00035FD06F00F06CDE90201032700E002273F
:10C8D000DFF8448276B1F30708D520462946D8E927
:10C8E0000023FEF7F9FB013704460D46761008F1E8
:10C8F0000808EFE7DDE9020122462B46FEF716FDA8
:10C90000CDE9020121E0C9F10007EFB1814E07F046
:10C910000F0506EBC502DDE91201D2E90023FEF79F
:10C92000DBFB7D4D3C1102274CB1E60704D5D5E970
:10C9300000230137FEF7D0FB64100835F4E7024608
:10C940000B46CDE9022300E00227119EE6B1DDE9A6
:10C950000245002220462946704BFEF72FFE98B173
:10C96000049A8AB10898002840F3E98009F1FF335E
:10C970000D93204629460022694BFEF7ADFB013797
:10C98000CDE90201089C02E0049CCDF834903846C1
:10C99000FEF73CFBDDE90223FEF79EFB0022614B24
:10C9A000FEF7E8F9A1F1507506462F46CCB9DDE94E
:10C9B000020100225C4BFEF7DBF932462B46CDE943
:10C9C0000201FEF719FE002840F04682DDE902016F
:10C9D000324605F10043FEF7F1FD002840F03582B4
:10C9E000ADE04C490A98621E01EBC20300284BD00F
:10C9F000D3E9002300204D49FEF798FC32462B4630
:10CA0000FEF7B6F9DDE90267CDE90E01079D39466B
:10CA10003046FEF7FBFD8046FEF7F8FA02460B466D
:10CA200030463946FEF7A4F908F1300305F8013B1A
:10CA3000DDE90E2306460F46A846FEF7BFFD002897
:10CA400040F0258332463B4600203449FEF790F9FA
:10CA5000DDE90E23FEF7B2FD002840F0D2800798F2
:10CA6000291AA1426BDADDE90E0100222C4BFEF7F8
:10CA700033FB0022CDE90E01294B30463946FEF743
:10CA80002BFB06460F46C2E7D3E9000132462B4690
:10CA9000FEF722FB079DCDE90E01DDE902672C19A7
:10CAA000A84639463046FEF7B1FD0546FEF7AEFA18
:10CAB000303502460B4630463946FEF759F908F83C
:10CAC000015BA04506460F4632D10022174BDDE937
:10CAD0000E01FEF74FF902460B4630463946FEF787
:10CAE0008BFD002840F08D80DDE90E2300200F49EA
:10CAF000FEF73EF902460B4630463946FEF75EFD2C
:10CB0000E8B14146884601F1FF3118F8012C302A7E
:10CB1000F8D0BCE218420108F04201080000F03FE2
:10CB20000000244000001C40000014400000E03FD2
:10CB300000229A4BFEF7D0FA06460F46B1E79DED6C
:10CB4000120B8DED020B179C002C7CDBB9F10E0F44
:10CB500079DC934C0C9904EBC9050029D5E9004513
:10CB600014DA049A002A11DC40F06E81204629462E
:10CB700000228C4BFEF7B0FADDE90223FEF732FD0E
:10CB8000049C2546002840F0618168E1079E0498D6
:10CB9000079F33180137059322462B46DDE9020132
:10CBA000FEF7C4FBFEF732FD0490FEF72FFA224693
:10CBB0002B46FEF791FA02460B46DDE90201FEF72D
:10CBC000D7F8049E303607F8016C059EB74202463E
:10CBD0000B46B84629D1FEF7CDF822462B4606462D
:10CBE0000F46FEF709FD70B93046394622462B46FE
:10CBF000FEF7DAFC002800F04C820499C90702D441
:10CC000047E2DDF8349040468046013818F8012CA0
:10CC1000392A06D1079B8342F6D1302609F1010952
:10CC20001E7001784A1C027033E200225B4BFEF753
:10CC300053FA00220023CDE902010137FEF7B4FCCC
:10CC40000028A9D025E20A9F002F30D00B9D012D8E
:10CC50000ADC159E16B104F2334002E0169BC3F1C4
:10CC60003600099C059E16E0049A099E501E8642D5
:10CC700001DB341A06E0099B109F0990C11A7C1849
:10CC800010940024049D002D03DA059A0020561B01
:10CC900001E0059E04980599069D0F182818069036
:10CCA00001215846059700F039FB054602E0099C32
:10CCB000059E0A9D66B1069A002A09DD059B069F1E
:10CCC000B242A8BF3246991AB81A0591B61A069010
:10CCD000099A002A20DD0A9BC3B1002C10DD2946E9
:10CCE0002246584600F0B4FB0546524629465846AF
:10CCF00000F01DFB51460746584600F070FABA4650
:10CD000009990A1B08D05846514602E0099A58462C
:10CD1000514600F09DFB82460121584600F0FEFA84
:10CD200004461098002805DD21465846109A00F068
:10CD30008FFB04460B9A012A10DC029B73B90399FE
:10CD4000C1F3130767B9184F0F4057B10598069BF9
:10CD5000421C591C05920691012702E0002700E0C1
:10CD6000029F109840B1236904EB8301086900F029
:10CD700089FAC0F1200200E001220699501810F053
:10CD80001F0315D0C3F12002042A0FDD059AC3F159
:10CD90001C03D0180590F61810E000BF00002440D6
:10CDA00018420108000014400000F07F08D013462C
:10CDB00005991C33C81806990590F618CB180693E8
:10CDC000059A002A04DD5146584600F093FB82463E
:10CDD000069A002A04DD2146584600F08BFB0446E3
:10CDE0001199E1B15046214600F0D8FB002816DA2F
:10CDF000514658460A22002300F008FA82460A9853
:10CE000009F1FF3948B129460A225846002300F0AB
:10CE1000FDF9089A0546049201E0089B04930498E2
:10CE2000002825DC0B99022922DD78B9214605224C
:10CE3000049B584600F0EAF904462146504600F0AB
:10CE4000ADFB00280BDC01E0002425460C9BDDF83F
:10CE50001C806FEA030909E0DDF834902546DDF80F
:10CE60001C80312008F8010B09F101090026FDE0C2
:10CE70000A9B002B00F0B280002E05DD29465846A3
:10CE8000324600F037FB05469FB16968584600F00E
:10CE900071F92B699A1C074605F10C01920000F10B
:10CEA0000C00FEF7ABFC58463946012200F022FB8D
:10CEB00000E02846079B0499079E5A18771C0692A3
:10CEC0002E46054621465046FFF7D4FA0346303336
:10CED000049031465046009300F060FB21460590D7
:10CEE0002A46584600F077FB8446C068009B07F14D
:10CEF000FF3848B961465046CDF804C000F04EFBFB
:10CF00009DE80810024600E0012258466146019261
:10CF1000009300F064F9019A009B6AB90B9959B922
:10CF2000029800F0010139B9392B2BD0059A002A5B
:10CF30002DDD049B31332AE00598002806DB1DD146
:10CF40000B99D9B9029800F00101B9B9002A1F461E
:10CF50001DDD514601225846009300F0CBFA2146D0
:10CF6000824600F01BFB0028009B02DC0FD1DA0791
:10CF70000DD5049B3133392F09D103E0002A09DD97
:10CF8000392B03D1392308F8013B55E0013308F868
:10CF9000013B6BE0069A07F8013C9742B8463BD04C
:10CFA00051460A220023584600F030F90A22002395
:10CFB000AE4282463146584604D100F027F9064673
:10CFC000054609E000F022F9294606460A2258469D
:10CFD000002300F01BF90546013773E70A9E50460F
:10CFE0002146FFF747FA079A00F13003049893555A
:10CFF0000136864207DA514658460A22002300F0DD
:10D0000005F98246EBE7DDF81C800499002601292A
:10D01000ACBF884408F101085146012258460093EC
:10D0200000F068FA2146824600F0B8FA0028009B1A
:10D0300002DC14D1DB0712D5414611F8010C392866
:10D04000884601F1FF3107D107988842F5D1312395
:10D0500009F10109037009E0421C0A7006E040462C
:10D060008046013818F8011C3029F9D0584621466D
:10D0700000F0B5F86DB12EB1AE4203D0584631463E
:10D0800000F0ADF85846294600F0A9F801E0DDF8B7
:10D09000349051460026584600F0A1F888F8006008
:10D0A000149A239E09F10101116026B1C6F800808F
:10D0B00001E0034800E0079819B0BDE8F08F00BF19
:10D0C00008420108AFF3008030B500293CD051F888
:10D0D000042C0B1F1D49002AB8BF9B180A6812B9FF
:10D0E0005A600B6030BD93420ED2196858189042B6
:10D0F00003D15A5889184268196014485A6003606D
:10D1000030BD994203D80A4651680029F9D1146804
:10D1100015199D420AD118682318D0188842136047
:10D1200012D108681B1813604B680CE002D90C235D
:10D13000036030BD18681C188C4203D10C68496824
:10D14000001918605960536030BD00BFB80100205D
:10D15000004870472C01002010B5C9B20346821860
:10D160009342184604D0047801338C42F8D100E091
:10D17000002010BD70B5456A04460E463DB910202A
:10D18000FEF7E2FA6062456085600560C560656A29
:10D19000EB6843B1626AD36853F8260078B101683E
:10D1A00043F8261017E004212046212200F020FB3E
:10D1B000E860606AC1680029ECD1002070BD0121DF
:10D1C00001FA06F56A1D2046920000F011FB0028C6
:10D1D000F3D04660856000230361C36070BD70B505
:10D1E000446A06460D463CB91020FEF7ADFA70625F
:10D1F000446084600460C4603DB1736A6A68D86842
:10D2000050F82210296040F8225070BD2DE9F041FD
:10D210000C461E460D69074601F1140100230868FB
:10D220001FFA80FC02FB0C6C060C564306EB1C40FC
:10D2300001331FFA8CFC060C0CEB0040AB4241F8AA
:10D24000040BECDBDEB1A268954213DB6168384663
:10D250000131FFF78FFF80462069831C04F10C0128
:10D260009A0008F10C00FEF7C9FA21463846FFF78C
:10D27000B6FF444604EB8502013556612561204620
:10D28000BDE8F081020C0346100410B91B04102005
:10D2900000E0002013F07F4F01D108301B0213F093
:10D2A000704F01D104301B0113F0404F01D1023007
:10D2B0009B00002B04DB5B0001D501307047202070
:10D2C00070470368024613F007000BD0D90721D43A
:10D2D000980703D55908116001207047980810601D
:10D2E0000220704799B209B91B0C102013F0FF0FF0
:10D2F00001D108301B0A190701D104301B09990715
:10D3000001D102309B08D90702D45B0804D0013058
:10D3100013607047002070472020704710B50C46FE
:10D320000121FFF727FF01224461026110BD2DE9B1
:10D33000F04F16460A6933699A4285B00D4601DA04
:10D3400035460E46D5F810803769AA68696808EB3B
:10D3500007049442C8BF0131FFF70CFF00EB8401C2
:10D36000143100F114030191019A934203D2002277
:10D3700043F8042BF8E706EB870705F1140305EBE8
:10D38000880C143702930CF1140E039700F1180364
:10D3900006F11402039DAA4211464CD209880432B8
:10D3A00009B3029F1D1F002657F8049BD5F8008083
:10D3B0001FFA89FB1FFA88FA01FB0BAC0CEB060A7B
:10D3C0004FEA19494FEA184601FB096808EB1A4869
:10D3D0001FFA8AFC4CEA084ABE454FEA184645F84F
:10D3E00004ABE1D82E6032F8021C11B353F8046C80
:10D3F000029F1D464FF0000935F802ACB7F800B0A7
:10D4000001FB0BACE144B6B246EA094645F8046CB0
:10D41000A84657F8046BB8F800A0360C01FB06A626
:10D42000043506EB194677454FEA1649E4D3C8F8A8
:10D4300000600433AEE7019B002C03DC046105B0FF
:10D44000BDE8F08F53F8042D002AF7D1013CF3E733
:10D4500012F003032DE9F04105460E46174607D0AA
:10D460005E1E234A002352F82620FFF7CFFE064611
:10D47000BF1039D06C6A3CB91020FEF765F96862BC
:10D48000446084600460C460D5F82480D8F8084003
:10D490009CB9284640F27121FFF740FF0446C8F8C6
:10D4A00008000020206008E07F101DD0D4F8008024
:10D4B0004046B8F1000F0ED00446F807F4D53146C7
:10D4C00022462846FFF733FF314680462846FFF7BD
:10D4D00086FE4646E8E7284621462246FFF727FF14
:10D4E0002060C0F80080E7E73046BDE8F08100BF6B
:10D4F000E04201082DE9F0470C464FEA6218236923
:10D500004968A56808EB030A814617460AF1010637
:10D51000AE4202DD01316D00FAE74846FFF72AFE10
:10D520000022054600F11400424504DA002140F8CB
:10D5300022100132F8E728EAE870226905EB80033F
:10D54000143304EB820017F01F0704F1140100F1FB
:10D55000140E14D01846C7F1200C00230A6802FAF2
:10D5600007F2134340F8043B51F8043B714523FA9A
:10D570000CF3F3D3036043B10AF1020605E051F85E
:10D58000042B8E4543F8042BF9D8013E48462E6102
:10D590002146FFF724FE2846BDE8F08703460A69C6
:10D5A0000069801A30B515D1151DAA0003F11404C5
:10D5B00089189B1804330A1D53F8045D52F8041DA2
:10D5C0008D4203D005D24FF0FF3030BD9C42F3D3E3
:10D5D00030BD012030BD2DE9F84306460C46084613
:10D5E00011461546FFF7DAFF071E08D139463046C7
:10D5F000FFF7C0FD012101614761BDE8F88301DB50
:10D60000002703E0234601272C461D46616830466B
:10D61000FFF7B0FD2A692369C76005EB820104EBBF
:10D62000830C0CF1140C01F114081434143500F1BE
:10D630001407002254F8046B55F8041B12FA86F202
:10D640001FFA81F9090CC9EB020EC1EB164606EB75
:10D650002E411FFA8EF90A1449EA014147F8041BCA
:10D66000A84526463946E5D866450DD256F8044BFE
:10D6700012FA84F5220C02EB2544ADB2221445EADD
:10D68000044441F8044BEFE751F8042D0AB9013B7B
:10D69000FAE70361BDE8F8832DE9F74389460121E4
:10D6A00055EC104B9046FFF765FDC5F30A5725F082
:10D6B0007F43064623F470000FB140F480100190C0
:10D6C000DCB102AA684642F8084DFFF7FAFD009C5B
:10D6D00050B1019AC0F1200302FA03F10C4322FA7F
:10D6E00000F27461019200E07461019A002A0CBF9B
:10D6F00001240224B261346107E001A8FFF7E1FDD3
:10D70000019901247161346120303FB1A7F23347A0
:10D710003F18C9F80070C0F135010AE006EB840338
:10D72000A0F23240C9F800001869FFF7ABFD6401B0
:10D73000211AC8F800103046BDE8FE83F8B5064649
:10D7400015460C4621B91146BDE8F840FEF70CB865
:10D750001AB9FFF7B9FC2C4612E000F057F8A842BE
:10D760000ED230462946FDF7FFFF074638B1214665
:10D770002A46FEF743F830462146FFF7A5FC3C4613
:10D780002046F8BD53EC102B10EE100A1A4613B1C8
:10D79000B3F1004F00D1E0B1124BA2F580119942D4
:10D7A00019D902F1FF4101F5E001994213D90E4B5D
:10D7B0009A4212D902F1004199420ED90B4B9A427A
:10D7C00002D012F5801F0AD1D0F1010038BF00202D
:10D7D00070470220704704207047032070470020E4
:10D7E000704700BFFFFFDF7FFFFF0F000000F07FEB
:10D7F00038B501FB02F42146FDF7B6FF054618B126
:10D8000000212246FEF703F8284638BD51F8040CE3
:10D81000002802DA04390B58C01804387047000099
:10D8200052756E2043616C6962726174696F6E2E0D
:10D830000000000052756E2043616C696272617471
:10D84000696F6E2E2E00000052756E2043616C6968
:10D8500062726174696F6E2E2E2E000043616C69D6
:10D8600062726174696F6E20646F6E6521000000E2
:10D8700000100020004000800800000008000000A8
:10D880000800000008000000010000000100000086
:10D890000100000000000000000000000600000081
:10D8A000200000000000040004000000040000004C
:10D8B0000400000004000000400000048000000894
:10D8C00006000A0007000B00080007000800070018
:10D8D0005072657373205573657220627574746F2E
:10D8E0006E20746F20636F6E74696E75652E2E2EB8
:10D8F00000000000436C65617200000058000000E9
:10D900002D0000002B0000003000000025342E31D7
:10D910006600000025640000000000000000000018
:10D9200000000000000000000000000000000000F7
:10D9300000000000000000000000000000000000E7
:10D940000000000000000000000080018001800154
:10D9500080018001800180018001800180018001BF
:10D9600080018001000000008001800100000000B3
:10D97000000000000000000000000000CC00CC000F
:10D98000CC00CC00CC00CC00000000000000000067
:10D990000000000000000000000000000000000087
:10D9A0000000000000000000000000000000000077
:10D9B00000000000600C600C600C30063006FE1F9A
:10D9C000FE1F300638071803FE1FFE1F180318033A
:10D9D0008C018C018C01000000008000E003F80F36
:10D9E0009C0E8C1C8C188C009800F801E007800EAF
:10D9F000801C8C188C189C18B80CF00FE003800069
:10DA000080000000000000000000000000000E1870
:10DA10001B0C110C11061106110311039B018E0141
:10DA2000C038C06C60446044304430441844186CC2
:10DA30000C380000000000000000E001F00338078F
:10DA4000180618063003F001F000F8009C310E3380
:10DA5000061E061C061C063FFC73F0210000000099
:10DA60000000000000000000000000000C000C009E
:10DA70000C000C000C000C00000000000000000076
:10DA80000000000000000000000000000000000096
:10DA90000000000000000000000000020003800100
:10DAA000C000C00060006000300030003000300076
:10DAB000300030003000300060006000C000C00066
:10DAC0008001000300020000000020006000C00090
:10DAD0008001800100030003000600060006000626
:10DAE0000006000600060006000300038001800116
:10DAF000C0006000200000000000000000000000E6
:10DB000000000000C000C000D806F807E0013003A4
:10DB100038070000000000000000000000000000C6
:10DB200000000000000000000000000000000000F5
:10DB30000000000080018001800180018001FC3F25
:10DB4000FC3F800180018001800180010000000015
:10DB500000000000000000000000000000000000C5
:10DB600000000000000000000000000000000000B5
:10DB700000000000000000000000800180010001A2
:10DB80000001800000000000000000000000000014
:10DB90000000000000000000000000000000000085
:10DBA000E007E007000000000000000000000000A7
:10DBB0000000000000000000000000000000000065
:10DBC0000000000000000000000000000000000055
:10DBD00000000000000000000000C000C0000000C5
:10DBE00000000000000000000000000C000C000617
:10DBF000000600060003000300038003800180018B
:10DC00008001C000C000C000600060000000000093
:10DC100000000000000000000000E003F007380EE4
:10DC2000180C0C180C180C180C180C180C180C18D4
:10DC30000C180C18180C380EF007E0030000000058
:10DC40000000000000000000000000018001C00191
:10DC5000F00198018801800180018001800180012C
:10DC600080018001800180018001800100000000AE
:10DC700000000000000000000000E003F80F180C96
:10DC80000C180C1800180018000C00060003800186
:10DC9000C000600030001800FC1FFC1F00000000E6
:10DCA00000000000000000000000E001F807180E6E
:10DCB0000C0C0C0C000C0006C003C007000C001874
:10DCC00000180C180C18180CF807E00300000000EE
:10DCD00000000000000000000000000C000E000F1B
:10DCE000000F800DC00C600C600C300C180C0C0C7C
:10DCF000FC3FFC3F000C000C000C000C000000007E
:10DD000000000000000000000000F80FF80F1800ED
:10DD100018000C00EC03FC071C0E001C0018001877
:10DD200000180C181C0C180EF807E0030000000087
:10DD300000000000000000000000C007F00F381CC9
:10DD4000181818000C00CC03EC0F3C0E1C1C0C180F
:10DD50000C180C18181C380EF007E0030000000027
:10DD600000000000000000000000FC1FFC1F000C71
:10DD700000060006000380038001C001C000E0002F
:10DD800060006000700030003000300000000000D3
:10DD900000000000000000000000E003F007380E63
:10DDA000180C180C180C3806F007F007180C0C1893
:10DDB0000C180C180C18380CF80FE00300000000C9
:10DDC00000000000000000000000E003F007380E33
:10DDD0001C0C0C180C180C181C1C381EF81BE01915
:10DDE0000018000C000C1C0EF807F00100000000E9
:10DDF0000000000000000000000000000000000023
:10DE00000000000080018001000000000000000010
:10DE10000000000000000000800180010000000000
:10DE200000000000000000000000000000000000F2
:10DE300000000000800180010000000000000000E0
:10DE400000000000000000008001800100010001CE
:10DE50008000000000000000000000000000000042
:10DE600000000000000000000010001C800FE00314
:10DE7000F8001800F800E003800F001C00100000FC
:10DE80000000000000000000000000000000000092
:10DE90000000000000000000F81F0000000000006B
:10DEA000F81F00000000000000000000000000005B
:10DEB0000000000000000000000000000000000062
:10DEC000000000000000000008003800F001C0075A
:10DED000001F0018001FC007F001380008000000F4
:10DEE00000000000000000000000E003F80F180C24
:10DEF0000C180C180018000C000600038001C0006C
:10DF0000C000C00000000000C000C0000000000011
:10DF1000000000000000000000000000E0071818EA
:10DF20000420C229224A114409440944094409220F
:10DF30001113E20C024004201818E0070000000052
:10DF40000000000000000000000080038003C00605
:10DF5000C006C006600C600C301830183018F83F4E
:10DF6000F83F1C700C600C6006C006C0000000008A
:10DF700000000000000000000000FC03FC0F0C0C7F
:10DF80000C180C180C180C0CFC07FC0F0C180C309F
:10DF90000C300C300C300C18FC1FFC07000000008B
:10DFA00000000000000000000000C007F01F38382B
:10DFB0001C300C7006600600060006000600060015
:10DFC000060006600C701C30F01FE0070000000027
:10DFD00000000000000000000000FE03FE0F060E1F
:10DFE00006180618063006300630063006300630B1
:10DFF000063006180618060EFE0FFE03000000008D
:10E0000000000000000000000000FC3FFC3F0C008E
:10E010000C000C000C000C00FC1FFC1F0C000C0082
:10E020000C000C000C000C00FC3FFC3F000000004A
:10E0300000000000000000000000F83FF83F18005A
:10E040001800180018001800F81FF81F1800180012
:10E050001800180018001800180018000000000030
:10E0600000000000000000000000E00FF83F3C78D6
:10E070000E6006E007C00300030003FE03FE03C0BA
:10E0800007C006C00EC03CF0F83FE00F00000000E3
:10E09000000000000000000000000C300C300C30CC
:10E0A0000C300C300C300C30FC3FFC3F0C300C3092
:10E0B0000C300C300C300C300C300C3000000000F8
:10E0C00000000000000000000000800180018001CD
:10E0D0008001800180018001800180018001800138
:10E0E000800180018001800180018001000000002A
:10E0F000000000000000000000000006000600060E
:10E1000000060006000600060006000600060006DF
:10E110000006180618063807F003E00100000000AA
:10E120000000000000000000000006300618060C89
:10E13000060606038601C60066007600DE008E0134
:10E1400006030606060C06180630066000000000EE
:10E150000000000000000000000018001800180077
:10E1600018001800180018001800180018001800EF
:10E170001800180018001800F81FF81F0000000011
:10E18000000000000000000000000EE01EF01EF085
:10E190001EF036D836D836D836D866CC66CC66CCA3
:10E1A000C6C6C6C6C6C6C6C686C386C300000000AD
:10E1B000000000000000000000000C301C303C306B
:10E1C0003C306C306C30CC30CC308C310C330C3378
:10E1D0000C360C360C3C0C3C0C380C3000000000AB
:10E1E00000000000000000000000E007F81F1C38DD
:10E1F0000E70066003C003C003C003C003C003C0A9
:10E2000003C006600E701C38F81FE0070000000015
:10E2100000000000000000000000FC0FFC1F0C3894
:10E220000C300C300C300C300C18FC1FFC070C00B0
:10E230000C000C000C000C000C000C000000000096
:10E2400000000000000000000000E007F81F1C387C
:10E250000E70066003E003C003C003C003C003C028
:10E2600007E006630E3F1C3CF83FE0F700C00000EB
:10E2700000000000000000000000FE0FFE1F063836
:10E280000630063006300638FE1FFE070603060677
:10E29000060C06180618063006300660000000005E
:10E2A00000000000000000000000E003F80F1C0C5C
:10E2B0000C180C180C001C00F803E00F001E0038AE
:10E2C000063006300E301C1CF80FE007000000007E
:10E2D00000000000000000000000FE7FFE7F8001C3
:10E2E0008001800180018001800180018001800126
:10E2F0008001800180018001800180010000000018
:10E30000000000000000000000000C300C300C3059
:10E310000C300C300C300C300C300C300C300C301D
:10E320000C300C300C301818F81FE007000000000B
:10E33000000000000000000000000360063006300E
:10E3400006300C180C180C18180C180C380E300667
:10E350003006700760036003C001C00100000000C8
:10E36000000000000000000000000360C361C36102
:10E37000C3616633663366336633663366336C1B5C
:10E380006C1B6C1B2C1A3C1E380E380E0000000053
:10E39000000000000000000000000FE00C701830CA
:10E3A0003018700C600EC00780038003C003E006C5
:10E3B000700C301C18180C300E6007E000000000D4
:10E3C0000000000000000000000003C006600C30E8
:10E3D0001C383818300C6006E007C003800180014B
:10E3E0008001800180018001800180010000000027
:10E3F00000000000000000000000FC7FFC7F0060C7
:10E4000000300018000C000600038001C00060000E
:10E41000300018000C000600FE7FFE7F00000000A8
:10E4200000000000000000000000E003E0036000C6
:10E4300060006000600060006000600060006000DC
:10E4400060006000600060006000600060006000CC
:10E450006000E003E00300000000300030006000D6
:10E4600060006000C000C000C000C00180018001E9
:10E470008001000300030003000600060000000006
:10E4800000000000000000000000E003E0030003C3
:10E490000003000300030003000300030003000364
:10E4A0000003000300030003000300030003000354
:10E4B0000003E003E003000000000000C001C00111
:10E4C00060036003600330063006180C180C00006F
:10E4D000000000000000000000000000000000003C
:10E4E000000000000000000000000000000000002C
:10E4F000000000000000000000000000000000001C
:10E5000000000000000000000000FFFFFFFF00000F
:10E51000000000000000000000000C000C000C00D7
:10E520000C000C000C0000000000000000000000C7
:10E5300000000000000000000000000000000000DB
:10E5400000000000000000000000000000000000CB
:10E5500000000000F003F8071C0C0C0C000FF00F7B
:10E56000F80C0C0C0C0C1C0FF80FF018000000003D
:10E570000000000000000000000018001800180053
:10E5800018001800D803F80F380C181818181818A5
:10E59000181818181818380CF80FD80300000000C5
:10E5A000000000000000000000000000000000006B
:10E5B00000000000C003F007300E180C180018000F
:10E5C00018001800180C300EF007C00300000000FF
:10E5D00000000000000000000000001800180018F3
:10E5E00000180018C01BF01F301C18181818181835
:10E5F000181818181818301CF01FC01B0000000055
:10E60000000000000000000000000000000000000A
:10E6100000000000C003F00F300C1818F81FF81F9E
:10E62000180018003818301CF00FC0070000000058
:10E6300000000000000000000000800FC00FC000BC
:10E64000C000C000F007F007C000C000C000C0005C
:10E65000C000C000C000C000C000C000000000003A
:10E6600000000000000000000000000000000000AA
:10E6700000000000E00DF80F180E0C0C0C0C0C0C38
:10E680000C0C0C0C0C0C180EF80FE00D000C0C0C04
:10E690001C06F807F0010000000018001800180020
:10E6A00018001800D807F80F381C18181818181870
:10E6B000181818181818181818181818000000003A
:10E6C00000000000000000000000C000C0000000CA
:10E6D00000000000C000C000C000C000C000C000BA
:10E6E000C000C000C000C000C000C00000000000AA
:10E6F00000000000000000000000C000C00000009A
:10E7000000000000C000C000C000C000C000C00089
:10E71000C000C000C000C000C000C000C000C000F9
:10E72000C000F8007800000000000C000C000C0095
:10E730000C000C000C0C0C060C038C01CC006C00C3
:10E74000FC009C018C030C030C060C0C0000000068
:10E7500000000000000000000000C000C000C00079
:10E76000C000C000C000C000C000C000C000C000A9
:10E77000C000C000C000C000C000C0000000000019
:10E780000000000000000000000000000000000089
:10E79000000000007C3CFF7EC7E383C183C183C1CE
:10E7A00083C183C183C183C183C183C100000000D1
:10E7B0000000000000000000000000000000000059
:10E7C000000000009807F80F381C181818181818BF
:10E7D0001818181818181818181818180000000019
:10E7E0000000000000000000000000000000000029
:10E7F00000000000C003F00F300C1818181818188B
:10E80000181818181818300CF00FC003000000007A
:10E8100000000000000000000000000000000000F8
:10E8200000000000D803F80F380C18181818181832
:10E83000181818181818380CF80FD80318001800F2
:10E840001800180018000000000000000000000080
:10E8500000000000C01BF01F301C181818181818F2
:10E86000181818181818301CF01FC01B00180018B2
:10E870000018001800180000000000000000000050
:10E8800000000000B007F0037000300030003000DE
:10E890003000300030003000300030000000000058
:10E8A0000000000000000000000000000000000068
:10E8B00000000000E003F003380E180C3800F003ED
:10E8C000C007000C180C380EF007E0030000000031
:10E8D0000000000000000000000000008000C000F8
:10E8E000C000C000F007F007C000C000C000C000BA
:10E8F000C000C000C000C000C007800700000000CA
:10E900000000000000000000000000000000000007
:10E9100000000000181818181818181818181818D7
:10E92000181818181818381CF01FE01900000000FB
:10E9300000000000000000000000000000000000D7
:10E94000000000000C18180C180C180C30063006CB
:10E950003006600360036003C001C00100000000D6
:10E9600000000000000000000000000000000000A7
:10E9700000000000C141C141C3616363636363631D
:10E980003636363636361C1C1C1C1C1C000000009B
:10E990000000000000000000000000000000000077
:10E9A000000000001C38381C300C60066003600357
:10E9B000600360036006300C381C1C380000000047
:10E9C0000000000000000000000000000000000047
:10E9D000000000001830301830187018600C600CFF
:10E9E000E00CC006C0068003800380038001800124
:10E9F000C001F000700000000000000000000000F6
:10EA000000000000FC1FFC1F000C0006000380013A
:10EA1000C000600030001800FC1FFC1F0000000058
:10EA20000000000000000000000000038001C000A2
:10EA3000C000C000C000C000C00060006000300026
:10EA400060004000C000C000C000C000C000C000A6
:10EA500080010003000000000000800180018001AF
:10EA6000800180018001800180018001800180019E
:10EA7000800180018001800180018001800180018E
:10EA8000800180018001000000006000C000C00122
:10EA900080018001800180018001000300030006E5
:10EAA000000300018001800180018001800180015C
:10EAB000C000600000000000000000000000000036
:10EAC0000000000000000000F010F81F080F000018
:10EAD0000000000000000000000000000000000036
:10EAE0000000000000000000000000000000000026
:10EAF0000000000000000000000000000000000016
:10EB00000000002000200020002000200020002025
:10EB100000000020000000000000005000500050E5
:10EB200000000000000000000000000000000000E5
:10EB30000000000900090012007F0012007F00128F
:10EB40000024002400000000001000380054005091
:10EB50000050003800140054005400380010000029
:10EB60000000803000490049004AC03220052009D9
:10EB70002009C010000000000000000C001200126C
:10EB800000140018002500230023801D0000000051
:10EB900000000040004000400000000000000000B5
:10EBA000000000000000000000000008001000103D
:10EBB0000020002000200020002000200010001075
:10EBC0000000004000200020001000100010001085
:10EBD0000010001000200020000000200070002025
:10EBE00000500000000000000000000000000000D5
:10EBF00000000000000000080008007F0008000876
:10EC00000000000000000000000000000000000004
:10EC10000000000000000000000000200020004074
:10EC20000000000000000000000000000070000074
:10EC300000000000000000000000000000000000D4
:10EC400000000000000000000000002000000000A4
:10EC50000000001000100010002000200020002004
:10EC600000400040000000000000001000280044A8
:10EC7000004400440044004400280010000000004C
:10EC800000000010003000500010001000100010B4
:10EC90000010001000000000000000300048004498
:10ECA00000040008001000200040007C000000006C
:10ECB0000000003000480004000800100008004474
:10ECC0000048003000000000000000080018001894
:10ECD000002800280048007C000800080000000010
:10ECE0000000003C00200040007000480004004488
:10ECF0000048003000000000000000180024004020
:10ED0000005000680044004400280010000000008B
:10ED10000000007C0004000800100010001000201B
:10ED20000020002000000000000000100028004427
:10ED300000280010002800440028001000000000F7
:10ED400000000010002800440044002C00140004BF
:10ED5000004800300000000000000000000000201B
:10ED60000000000000000000000000200000000083
:10ED70000000000000000020000000000000000073
:10ED800000000020002000400000000000040008F7
:10ED900000300040003000080004000000000000C7
:10EDA000000000000000007C00000000007C00006B
:10EDB00000000000000000000000000000400020F3
:10EDC00000180004001800200040000000000000AF
:10EDD0000000003800640044000400080010001027
:10EDE00000000010000000000000800F4010A02E66
:10EDF000A0512051205120512053C04D20204010BF
:10EE0000000000080014001400140022003E00223C
:10EE100000410041000000000000003C00220022F0
:10EE20000022003C002200220022003C00000000E2
:10EE30000000000E00110021002000200020002111
:10EE40000011000E000000000000003C0022002124
:10EE500000210021002100210022003C00000000D0
:10EE60000000003E002000200020003E0020002086
:10EE70000020003E000000000000003E00200020B6
:10EE80000020003C002000200020002000000000A6
:10EE90000000000E001100210020002700210021A9
:10EEA0000011000E000000000000002100210021E0
:10EEB0000021003F0021002100210021000000006E
:10EEC0000000002000200020002000200020002062
:10EED00000200020000000000000000800080008DA
:10EEE000000800080008004800480030000000004A
:10EEF00000000022002400280028003800280024F8
:10EF0000002400220000000000000020002000205B
:10EF100000200020002000200020003E0000000013
:10EF200000008020803180318031802A802A802A30
:10EF3000802A802400000000000000210031003100
:10EF400000290029002500230023002100000000E3
:10EF50000000000C001200210021002100210021EE
:10EF60000012000C000000000000003C0022002203
:10EF70000022003C002000200020002000000000B3
:10EF80000000000C001200210021002100210021BE
:10EF90000016000D000100000000003E00210021CD
:10EFA0000021003E002400220021802000000000FB
:10EFB0000000001C002200220020001C0002002291
:10EFC0000022001C000000000000003E00080008B5
:10EFD0000008000800080008000800080000000001
:10EFE000000000210021002100210021002100213A
:10EFF0000012000C0000000000000041004100224F
:10F000000022002200140014001400080000000078
:10F0100000004044404A402A802A802A802A802AD0
:10F02000802A0011000000000000004100220014AE
:10F030000014000800140014002200410000000029
:10F04000000000410022002200140008000800080F
:10F0500000080008000000000000007E000200041C
:10F0600000080010001000200040007E000000009A
:10F0700000000030002000200020002000200020A0
:10F080000020002000200020000000400040002060
:10F0900000200020002000200010001000000000D0
:10F0A0000000006000200020002000200020002040
:10F0B0000020002000200020000000100028002870
:10F0C00000280044000000000000000000000000D4
:10F0D0000000000000000000000000000000000030
:10F0E000000000000000007E004000200000000042
:10F0F0000000000000000000000000000000000010
:10F10000000000000000003800440004003C0044FF
:10F110000044003C00000000000000400040005897
:10F1200000640044004400440064005800000000F3
:10F130000000000000000030004800400040004097
:10F14000004800300000000000000004000400340B
:10F15000004C004400440044004C00340000000017
:10F16000000000000000003800440044007C004023
:10F17000004400380000000000000060004000E093
:10F1800000400040004000400040004000000000FF
:10F190000000000000000034004C00440044004423
:10F1A000004C0034000400440000004000400058BF
:10F1B0000064004400440044004400440000000097
:10F1C00000000040000000400040004000400040BF
:10F1D000004000400000000000000040000000402F
:10F1E000004000400040004000400040004000401F
:10F1F00000000040004000480050006000500050F7
:10F2000000480048000000000000004000400040AE
:10F21000004000400040004000400040000000006E
:10F220000000000000000052006D00490049004944
:10F2300000490049000000000000000000000058E4
:10F240000064004400440044004400440000000006
:10F250000000000000000038004400440044004466
:10F2600000440038000000000000000000000058CA
:10F270000064004400440044006400580040004022
:10F280000000000000000034004C00440044004432
:10F29000004C003400040004000000000000005096
:10F2A00000600040004000400040004000000000BE
:10F2B000000000000000003000480040003000085E
:10F2C000004800300000000000000040004000E066
:10F2D000004000400040004000400060000000008E
:10F2E00000000000000000440044004400440044CA
:10F2F000004C00340000000000000000000000444A
:10F300000044002800280028002800100000000009
:10F31000000000000000004900490055005500555C
:10F320000055002200000000000000000000004422
:10F3300000280028001000280028004400000000D9
:10F3400000000000000000440044002800280028BD
:10F3500000100010001000100000000000000078F5
:10F36000000800100020002000400078000000008D
:10F37000000000100020002000200020004000209D
:10F38000002000200020002000000020002000209D
:10F39000002000200020002000200020002000206D
:10F3A000000000400020002000200020001000206D
:10F3B00000200020002000200000000000000000CD
:10F3C0000074005800000000000000000000000071
:10F3D000000000000070005000500050005000502D
:10F3E000005000700000000000000000000000005D
:10F3F000000000000000000000000000000000000D
:10F4000000000000000010001000100010001000AC
:10F4100010000000100000000000000000002800A4
:10F42000280028000000000000000000000000008C
:10F43000000000000000140014003E00140028002A
:10F440007C002800280000000000000010003800A8
:10F45000540050003800140014005400380010000C
:10F460000000000000004400A800A80050001400A4
:10F470001A002A0024000000000000000000200004
:10F48000500050002000E800980098006000000044
:10F4900000000000000080008000800000000000EC
:10F4A000000000000000000000000000000040001C
:10F4B000800080008000800080008000800080004C
:10F4C00000000000000080004000400040004000BC
:10F4D00040004000400040000000000000004000EC
:10F4E000E0004000A000000000000000000000005C
:10F4F0000000000000000000000020002000F800D4
:10F5000020002000000000000000000000000000BB
:10F51000000000000000000000000000400040006B
:10F5200000000000000000000000000000000000DB
:10F53000C00000000000000000000000000000000B
:10F54000000000000000000000000000400000007B
:10F5500000000000000020002000200040004000CB
:10F5600080008000800000000000000000006000BB
:10F5700090009000900090009000900060000000CB
:10F5800000000000000020006000A000200020001B
:10F5900020002000200000000000000000006000AB
:10F5A000900010001000200040008000F0000000DB
:10F5B00000000000000060009000100060001000DB
:10F5C000100090006000000000000000000010002B
:10F5D0003000500050009000F800100010000000B3
:10F5E000000000000000700040008000E0001000FB
:10F5F00010009000600000000000000000006000AB
:10F6000090008000A000D0009000900060000000FA
:10F61000000000000000F00010002000200020008A
:10F6200040004000400000000000000000006000BA
:10F63000900090006000900090009000600000003A
:10F64000000000000000600090009000B00050003A
:10F6500010009000600000000000000000000000AA
:10F66000000040000000000000000000400000001A
:10F67000000000000000000000004000000000004A
:10F6800000000000400040000000000000000000FA
:10F69000000010006000800060001000000000000A
:10F6A000000000000000000000000000F00000006A
:10F6B000F00000000000000000000000000000005A
:10F6C000000080006000100060008000000000006A
:10F6D00000000000000060009000100020004000CA
:10F6E00040000000400000000000000000001C007E
:10F6F00022005B00A500A500A500A5009E0041001A
:10F700000000000000002000500050005000500099
:10F710007000880088000000000000000000F00079
:10F7200088008800F000880088008800F000000051
:10F7300000000000000038004400840080008000C9
:10F740008400440038000000000000000000E000D9
:10F75000900088008800880088009000E000000089
:10F76000000000000000F80080008000F800800029
:10F7700080008000F8000000000000000000780019
:10F780004000400070004000400040004000000089
:10F7900000000000000038004400840080009C004D
:10F7A00084004400380000000000000000008800D1
:10F7B00088008800F8008800880088008800000021
:10F7C00000000000000080008000800080008000B9
:10F7D0008000800080000000000000000000100099
:10F7E0001000100010001000900090006000000059
:10F7F00000000000000088009000A000E000A000D1
:10F8000090009000880000000000000000008000D0
:10F81000800080008000800080008000F0000000F8
:10F820000000000000008200C600C600AA00AA0076
:10F83000AA00AA009200000000000000000084005E
:10F84000C400A400A400940094008C008400000074
:10F8500000000000000030004800840084008400A4
:10F860008400480030000000000000000000F000AC
:10F87000880088008800F000800080008000000080
:10F880000000000000003000480084008400840074
:10F8900084005800340004000000000000007800DC
:10F8A000440044007800500048004400420000003A
:10F8B0000000000000007000880080007000080058
:10F8C0008800880070000000000000000000F800C0
:10F8D0002000200020002000200020002000000048
:10F8E0000000000000008400840084008400840084
:10F8F0008400480030000000000000000000880084
:10F9000088005000500050005000500020000000BF
:10F910000000000000009200AA00AA00AA00AA00AD
:10F92000AA00AA00440000000000000000008400BB
:10F9300048004800300030004800480084000000C3
:10F94000000000000000880050005000200020004F
:10F950002000200020000000000000000000F8004F
:10F96000080010002000200040008000F800000087
:10F97000000000000000C0008000800080008000C7
:10F9800080008000800080000000000000008000F7
:10F9900080004000400040004000200020000000A7
:10F9A000000000000000C000400040004000400097
:10F9B0004000400040004000000000000000400007
:10F9C000A000A000A0000000000000000000000057
:10F9D0000000000000000000000000000000000027
:10F9E000000000000000F80000000000000080009F
:10F9F00040000000000000000000000000000000C7
:10FA000000000000000000000000E0001000700096
:10FA100090009000700000000000000000008000D6
:10FA20008000A000D00090009000D000A000000056
:10FA30000000000000000000000060009000800056
:10FA40008000900060000000000000000000100036
:10FA500010005000B00090009000B0005000000076
:10FA60000000000000000000000060009000F000B6
:10FA70008000900060000000000000000000C00056
:10FA80008000C000800080008000800080000000B6
:10FA9000000000000000000000005000B0009000D6
:10FAA0009000B00050001000000000000000800036
:10FAB0008000A000D0009000900090009000000016
:10FAC0000000000000008000000080008000800036
:10FAD0008000800080000000000000000000800026
:10FAE0000000800080008000800080008000800096
:10FAF000000000000000800080009000A000C00016
:10FB0000A0009000900000000000000000008000B5
:10FB10008000800080008000800080008000000065
:10FB200000000000000000000000A600DA009200C3
:10FB3000920092009200000000000000000000000F
:10FB40000000A000D0009000900090009000000005
:10FB50000000000000000000000060009000900025
:10FB60009000900060000000000000000000000015
:10FB70000000A000D00090009000D000A000800005
:10FB8000000000000000000000005000B0009000E5
:10FB90009000B000500010000000000000000000C5
:10FBA0000000A000C00080008000800080000000F5
:10FBB00000000000000000000000E0009000400095
:10FBC00020009000600000000000000000008000A5
:10FBD0008000C0008000800080008000C000000025
:10FBE0000000000000000000000090009000900065
:10FBF0009000B00050000000000000000000000075
:10FC000000008800880050005000500020000000D4
:10FC1000000000000000000000009200AA00AA00FE
:10FC2000AA00AA004400000000000000000000003C
:10FC300000008800500020002000500088000000D4
:10FC4000000000000000000000008800500050008C
:10FC500050002000200020000000000000000000F4
:10FC60000000F0001000200040008000F0000000C4
:10FC7000000000000000C000800080008000000044
:10FC800080008000800080000000000000008000F4
:10FC90008000800080008000800080008000800064
:10FCA000000000000000C0004000400040002000B4
:10FCB0004000400040004000000000000000000044
:10FCC00000000000E800B00000000000000000009C
:10FCD0000000000000000000E000A000A000A00064
:10FCE000A000A000E00000000000000000000000F4
:10FCF0000000000000000000400040004000400004
:10FD00004000400000004000A000A000A000000053
:10FD10000000000000000000000024002400FE009D
:10FD20004800FC00480048003800540050003800EB
:10FD300014001400540038004400A800A80050002B
:10FD400014001A002A0024001000280028001000C7
:10FD500074004C004C003000100010001000000037
:10FD6000000000000000000008001000100010005B
:10FD70001000100010000800100008000800080023
:10FD8000080008000800100000000000240018000F
:10FD90003C001800240000000000000010001000CB
:10FDA0007C001000100000000000000000000000B7
:10FDB0000000080008001000000000000000000023
:10FDC0003C000000000000000000000000000000F7
:10FDD00000000000180018000800080008001000CB
:10FDE000100020002000200018002400240024001F
:10FDF000240024002400180008001800280008002F
:10FE00000800080008000800380044000000040052
:10FE10000800100020007C001800240004001800D6
:10FE2000040004002400180004000C001400240046
:10FE300044007E00040004003C0020002000380044
:10FE400004000400240018001800240020003800DA
:10FE500024002400240018003C00040008000800CE
:10FE600008001000100010001800240024001800E2
:10FE7000240024002400180018002400240024007A
:10FE80001C00040024001800000000001000000006
:10FE9000000010000000000000000000080000004A
:10FEA000000008001000000000000000040018001E
:10FEB00020001800040000000000000000003C00CA
:10FEC00000003C00000000000000000020001800BE
:10FED000040018002000000018002400040008009E
:10FEE00010001000000010003C0042009900A50026
:10FEF000A5009D0042003800380044004400440042
:10FF00007C00440044004400780044004400780031
:10FF100044004400440078001C00220042004000DD
:10FF20004000420022001C007000480044004400D1
:10FF300044004400480070007C00400040007C0009
:10FF40004000400040007C003C00200020003800C1
:10FF500020002000200020001C0022004200400061
:10FF60004E00420022001C004400440044007C007B
:10FF70004400440044004400100010001000100031
:10FF80001000100010001000040004000400040021
:10FF900004002400240018004400480050007000B1
:10FFA00050004800480044002000200020002000AD
:10FFB0002000200020003C008200C600C600AA00ED
:10FFC000AA00AA00AA009200420062005200520059
:10FFD0004A004A0046004200180024004200420045
:10FFE000420042002400180078004400440044000D
:10FFF0007800400040004000180024004200420009
:020000040801F1
:10000000420042002C001A007800440044007800AE
:1000100050004800440042003800440040003800CE
:1000200004004400440038007C0010001000100060
:100030001000100010001000420042004200420078
:100040004200420024001800440044002800280018
:1000500028002800280010009200AA00AA00AA0088
:10006000AA00AA00AA0044004200240024001800AC
:10007000180024002400420044002800280010003A
:1000800010001000100010007C0004000800100098
:100090001000200040007C001C0010001000100028
:1000A0001000100010001C001000100008000800D4
:1000B00008000800040004001C0004000400040000
:1000C0000400040004001C0010002800440000008C
:1000D0000000000000000000000000000000000020
:1000E00000000000000000002000100010000000D0
:1000F00000000000000000000000000018000400E4
:100100001C00240024001C002000200028003400D3
:1001100024002400340028000000000018002400FF
:1001200020002000240018000400040014002C000B
:10013000240024002C0014000000000018002400FB
:100140003C002000240018000000180010001000DF
:1001500018001000100010000000180024002400F7
:10016000180004002400180020002000280034009B
:1001700024002400240024001000000010001000BF
:100180001000100010001000080000000800080017
:10019000080008002800100020002000240028008B
:1001A000300028002400240010001000100010006F
:1001B000100010001000100000000000A600DA007F
:1001C000920092009200920000000000280034008B
:1001D0002400240024002400000000001800240053
:1001E000240024002400180000002800340024000B
:1001F0003800200020002000000014002C00240003
:100200001C00040004000400000000002C0030006A
:100210002000200020002000000000001800240022
:100220001000080024001800000010003800100022
:10023000100010001000180000000000240024002E
:10024000240024002C00140000000000440044009E
:100250002800280028001000000000009200AA00DA
:10026000AA00AA00AA0044000000000044002800E0
:10027000100010002800440000002800280028007A
:100280001000100010001000000000003C000400EE
:100290000800100020003C000000080010001000C2
:1002A00020001000100008001000100010001000C6
:1002B00010001000100010000000100008000800DE
:1002C00004000800080010000000000000006000AA
:1002D00092000C0000000000FF00FF00FF00FF0084
:1002E000FF00FF00FF00FF00000000000000000012
:1002F00000000000000000000000000000000000FE
:1003000000000000000000000000000000000000ED
:10031000000000000000000000008001800180015A
:1003200080018001800180018001800180018001C5
:1003300080018001000000008001800100000000B9
:10034000000000000000000000000000CC00CC0015
:10035000CC00CC00CC00CC0000000000000000006D
:10036000000000000000000000000000000000008D
:10037000000000000000000000000000000000007D
:1003800000000000600C600C600C30063006FE1FA0
:10039000FE1F300638071803FE1FFE1F1803180340
:1003A0008C018C018C01000000008000E003F80F3C
:1003B0009C0E8C1C8C188C009800F801E007800EB5
:1003C000801C8C188C189C18B80CF00FE00380006F
:1003D00080000000000000000000000000000E1877
:1003E0001B0C110C11061106110311039B018E0148
:1003F000C038C06C60446044304430441844186CC9
:100400000C380000000000000000E001F003380795
:10041000180618063003F001F000F8009C310E3386
:10042000061E061C061C063FFC73F021000000009F
:100430000000000000000000000000000C000C00A4
:100440000C000C000C000C0000000000000000007C
:10045000000000000000000000000000000000009C
:100460000000000000000000000000020003800106
:10047000C000C0006000600030003000300030007C
:10048000300030003000300060006000C000C0006C
:100490008001000300020000000020006000C00096
:1004A000800180010003000300060006000600062C
:1004B000000600060006000600030003800180011C
:1004C000C0006000200000000000000000000000EC
:1004D00000000000C000C000D806F807E0013003AB
:1004E00038070000000000000000000000000000CD
:1004F00000000000000000000000000000000000FC
:100500000000000080018001800180018001FC3F2B
:10051000FC3F80018001800180018001000000001B
:1005200000000000000000000000000000000000CB
:1005300000000000000000000000000000000000BB
:1005400000000000000000000000800180010001A8
:10055000000180000000000000000000000000001A
:10056000000000000000000000000000000000008B
:10057000E007E007000000000000000000000000AD
:10058000000000000000000000000000000000006B
:10059000000000000000000000000000000000005B
:1005A00000000000000000000000C000C0000000CB
:1005B00000000000000000000000000C000C00061D
:1005C0000006000600030003000380038001800191
:1005D0008001C000C000C00060006000000000009A
:1005E00000000000000000000000E003F007380EEB
:1005F000180C0C180C180C180C180C180C180C18DB
:100600000C180C18180C380EF007E003000000005E
:100610000000000000000000000000018001C00197
:10062000F001980188018001800180018001800132
:1006300080018001800180018001800100000000B4
:1006400000000000000000000000E003F80F180C9C
:100650000C180C1800180018000C0006000380018C
:10066000C000600030001800FC1FFC1F00000000EC
:1006700000000000000000000000E001F807180E74
:100680000C0C0C0C000C0006C003C007000C00187A
:1006900000180C180C18180CF807E00300000000F4
:1006A00000000000000000000000000C000E000F21
:1006B000000F800DC00C600C600C300C180C0C0C82
:1006C000FC3FFC3F000C000C000C000C0000000084
:1006D00000000000000000000000F80FF80F1800F4
:1006E00018000C00EC03FC071C0E001C001800187E
:1006F00000180C181C0C180EF807E003000000008E
:1007000000000000000000000000C007F00F381CCF
:10071000181818000C00CC03EC0F3C0E1C1C0C1815
:100720000C180C18181C380EF007E003000000002D
:1007300000000000000000000000FC1FFC1F000C77
:1007400000060006000380038001C001C000E00035
:1007500060006000700030003000300000000000D9
:1007600000000000000000000000E003F007380E69
:10077000180C180C180C3806F007F007180C0C1899
:100780000C180C180C18380CF80FE00300000000CF
:1007900000000000000000000000E003F007380E39
:1007A0001C0C0C180C180C181C1C381EF81BE0191B
:1007B0000018000C000C1C0EF807F00100000000EF
:1007C0000000000000000000000000000000000029
:1007D0000000000080018001000000000000000017
:1007E0000000000000000000800180010000000007
:1007F00000000000000000000000000000000000F9
:1008000000000000800180010000000000000000E6
:1008100000000000000000008001800100010001D4
:100820008000000000000000000000000000000048
:1008300000000000000000000010001C800FE0031A
:10084000F8001800F800E003800F001C0010000002
:100850000000000000000000000000000000000098
:100860000000000000000000F81F00000000000071
:10087000F81F000000000000000000000000000061
:100880000000000000000000000000000000000068
:10089000000000000000000008003800F001C00760
:1008A000001F0018001FC007F001380008000000FA
:1008B00000000000000000000000E003F80F180C2A
:1008C0000C180C180018000C000600038001C00072
:1008D000C000C00000000000C000C0000000000018
:1008E000000000000000000000000000E0071818F1
:1008F0000420C229224A1144094409440944092216
:100900001113E20C024004201818E0070000000058
:100910000000000000000000000080038003C0060B
:10092000C006C006600C600C301830183018F83F54
:10093000F83F1C700C600C6006C006C00000000090
:1009400000000000000000000000FC03FC0F0C0C85
:100950000C180C180C180C0CFC07FC0F0C180C30A5
:100960000C300C300C300C18FC1FFC070000000091
:1009700000000000000000000000C007F01F383831
:100980001C300C700660060006000600060006001B
:10099000060006600C701C30F01FE007000000002D
:1009A00000000000000000000000FE03FE0F060E25
:1009B00006180618063006300630063006300630B7
:1009C000063006180618060EFE0FFE030000000093
:1009D00000000000000000000000FC3FFC3F0C0095
:1009E0000C000C000C000C00FC1FFC1F0C000C0089
:1009F0000C000C000C000C00FC3FFC3F0000000051
:100A000000000000000000000000F83FF83F180060
:100A10001800180018001800F81FF81F1800180018
:100A20001800180018001800180018000000000036
:100A300000000000000000000000E00FF83F3C78DC
:100A40000E6006E007C00300030003FE03FE03C0C0
:100A500007C006C00EC03CF0F83FE00F00000000E9
:100A6000000000000000000000000C300C300C30D2
:100A70000C300C300C300C30FC3FFC3F0C300C3098
:100A80000C300C300C300C300C300C3000000000FE
:100A900000000000000000000000800180018001D3
:100AA000800180018001800180018001800180013E
:100AB0008001800180018001800180010000000030
:100AC0000000000000000000000000060006000614
:100AD00000060006000600060006000600060006E6
:100AE0000006180618063807F003E00100000000B1
:100AF0000000000000000000000006300618060C90
:100B0000060606038601C60066007600DE008E013A
:100B100006030606060C06180630066000000000F4
:100B2000000000000000000000001800180018007D
:100B300018001800180018001800180018001800F5
:100B40001800180018001800F81FF81F0000000017
:100B5000000000000000000000000EE01EF01EF08B
:100B60001EF036D836D836D836D866CC66CC66CCA9
:100B7000C6C6C6C6C6C6C6C686C386C300000000B3
:100B8000000000000000000000000C301C303C3071
:100B90003C306C306C30CC30CC308C310C330C337E
:100BA0000C360C360C3C0C3C0C380C3000000000B1
:100BB00000000000000000000000E007F81F1C38E3
:100BC0000E70066003C003C003C003C003C003C0AF
:100BD00003C006600E701C38F81FE007000000001C
:100BE00000000000000000000000FC0FFC1F0C389B
:100BF0000C300C300C300C300C18FC1FFC070C00B7
:100C00000C000C000C000C000C000C00000000009C
:100C100000000000000000000000E007F81F1C3882
:100C20000E70066003E003C003C003C003C003C02E
:100C300007E006630E3F1C3CF83FE0F700C00000F1
:100C400000000000000000000000FE0FFE1F06383C
:100C50000630063006300638FE1FFE07060306067D
:100C6000060C061806180630063006600000000064
:100C700000000000000000000000E003F80F1C0C62
:100C80000C180C180C001C00F803E00F001E0038B4
:100C9000063006300E301C1CF80FE0070000000084
:100CA00000000000000000000000FE7FFE7F8001C9
:100CB000800180018001800180018001800180012C
:100CC000800180018001800180018001000000001E
:100CD000000000000000000000000C300C300C3060
:100CE0000C300C300C300C300C300C300C300C3024
:100CF0000C300C300C301818F81FE0070000000012
:100D00000000000000000000000003600630063014
:100D100006300C180C180C18180C180C380E30066D
:100D20003006700760036003C001C00100000000CE
:100D3000000000000000000000000360C361C36108
:100D4000C3616633663366336633663366336C1B62
:100D50006C1B6C1B2C1A3C1E380E380E0000000059
:100D6000000000000000000000000FE00C701830D0
:100D70003018700C600EC00780038003C003E006CB
:100D8000700C301C18180C300E6007E000000000DA
:100D90000000000000000000000003C006600C30EE
:100DA0001C383818300C6006E007C0038001800151
:100DB000800180018001800180018001000000002D
:100DC00000000000000000000000FC7FFC7F0060CD
:100DD00000300018000C000600038001C000600015
:100DE000300018000C000600FE7FFE7F00000000AF
:100DF00000000000000000000000E003E0036000CD
:100E000060006000600060006000600060006000E2
:100E100060006000600060006000600060006000D2
:100E20006000E003E00300000000300030006000DC
:100E300060006000C000C000C000C00180018001EF
:100E4000800100030003000300060006000000000C
:100E500000000000000000000000E003E0030003C9
:100E6000000300030003000300030003000300036A
:100E7000000300030003000300030003000300035A
:100E80000003E003E003000000000000C001C00117
:100E900060036003600330063006180C180C000075
:100EA0000000000000000000000000000000000042
:100EB0000000000000000000000000000000000032
:100EC0000000000000000000000000000000000022
:100ED00000000000000000000000FFFFFFFF000016
:100EE000000000000000000000000C000C000C00DE
:100EF0000C000C000C0000000000000000000000CE
:100F000000000000000000000000000000000000E1
:100F100000000000000000000000000000000000D1
:100F200000000000F003F8071C0C0C0C000FF00F81
:100F3000F80C0C0C0C0C1C0FF80FF0180000000043
:100F40000000000000000000000018001800180059
:100F500018001800D803F80F380C181818181818AB
:100F6000181818181818380CF80FD80300000000CB
:100F70000000000000000000000000000000000071
:100F800000000000C003F007300E180C1800180015
:100F900018001800180C300EF007C0030000000005
:100FA00000000000000000000000001800180018F9
:100FB00000180018C01BF01F301C1818181818183B
:100FC000181818181818301CF01FC01B000000005B
:100FD0000000000000000000000000000000000011
:100FE00000000000C003F00F300C1818F81FF81FA5
:100FF000180018003818301CF00FC007000000005F
:1010000000000000000000000000800FC00FC000C2
:10101000C000C000F007F007C000C000C000C00062
:10102000C000C000C000C000C000C0000000000040
:1010300000000000000000000000000000000000B0
:1010400000000000E00DF80F180E0C0C0C0C0C0C3E
:101050000C0C0C0C0C0C180EF80FE00D000C0C0C0A
:101060001C06F807F0010000000018001800180026
:1010700018001800D807F80F381C18181818181876
:101080001818181818181818181818180000000040
:1010900000000000000000000000C000C0000000D0
:1010A00000000000C000C000C000C000C000C000C0
:1010B000C000C000C000C000C000C00000000000B0
:1010C00000000000000000000000C000C0000000A0
:1010D00000000000C000C000C000C000C000C00090
:1010E000C000C000C000C000C000C000C000C00000
:1010F000C000F8007800000000000C000C000C009C
:101100000C000C000C0C0C060C038C01CC006C00C9
:10111000FC009C018C030C030C060C0C000000006E
:1011200000000000000000000000C000C000C0007F
:10113000C000C000C000C000C000C000C000C000AF
:10114000C000C000C000C000C000C000000000001F
:10115000000000000000000000000000000000008F
:10116000000000007C3CFF7EC7E383C183C183C1D4
:1011700083C183C183C183C183C183C100000000D7
:10118000000000000000000000000000000000005F
:10119000000000009807F80F381C181818181818C5
:1011A000181818181818181818181818000000001F
:1011B000000000000000000000000000000000002F
:1011C00000000000C003F00F300C18181818181891
:1011D000181818181818300CF00FC0030000000081
:1011E00000000000000000000000000000000000FF
:1011F00000000000D803F80F380C18181818181839
:10120000181818181818380CF80FD80318001800F8
:101210001800180018000000000000000000000086
:1012200000000000C01BF01F301C181818181818F8
:10123000181818181818301CF01FC01B00180018B8
:101240000018001800180000000000000000000056
:1012500000000000B007F0037000300030003000E4
:10126000300030003000300030003000000000005E
:10127000000000000000000000000000000000006E
:1012800000000000E003F003380E180C3800F003F3
:10129000C007000C180C380EF007E0030000000037
:1012A0000000000000000000000000008000C000FE
:1012B000C000C000F007F007C000C000C000C000C0
:1012C000C000C000C000C000C007800700000000D0
:1012D000000000000000000000000000000000000E
:1012E00000000000181818181818181818181818DE
:1012F000181818181818381CF01FE0190000000002
:1013000000000000000000000000000000000000DD
:10131000000000000C18180C180C180C30063006D1
:101320003006600360036003C001C00100000000DC
:1013300000000000000000000000000000000000AD
:1013400000000000C141C141C36163636363636323
:101350003636363636361C1C1C1C1C1C00000000A1
:10136000000000000000000000000000000000007D
:10137000000000001C38381C300C6006600360035D
:10138000600360036006300C381C1C38000000004D
:10139000000000000000000000000000000000004D
:1013A000000000001830301830187018600C600C05
:1013B000E00CC006C006800380038003800180012A
:1013C000C001F000700000000000000000000000FC
:1013D00000000000FC1FFC1F000C00060003800141
:1013E000C000600030001800FC1FFC1F000000005F
:1013F0000000000000000000000000038001C000A9
:10140000C000C000C000C000C0006000600030002C
:1014100060004000C000C000C000C000C000C000AC
:1014200080010003000000000000800180018001B5
:1014300080018001800180018001800180018001A4
:101440008001800180018001800180018001800194
:10145000800180018001000000006000C000C00128
:1014600080018001800180018001000300030006EB
:101470000003000180018001800180018001800162
:10148000C00060000000000000000000000000003C
:101490000000000000000000F010F81F080F00001E
:1014A000000000000000000000000000000000003C
:1014B000000000000000000000000000000000002C
:1014C000000000000000000000000000000000001C
:1014D000000000200020002000200020002000202C
:1014E00000000020000000000000005000500050EC
:1014F00000000000000000000000000000000000EC
:101500000000000900090012007F0012007F001295
:101510000024002400000000001000380054005097
:10152000005000380014005400540038001000002F
:101530000000803000490049004AC03220052009DF
:101540002009C010000000000000000C0012001272
:1015500000140018002500230023801D0000000057
:1015600000000040004000400000000000000000BB
:101570000000000000000000000000080010001043
:10158000002000200020002000200020001000107B
:10159000000000400020002000100010001000108B
:1015A000001000100020002000000020007000202B
:1015B00000500000000000000000000000000000DB
:1015C00000000000000000080008007F000800087C
:1015D000000000000000000000000000000000000B
:1015E000000000000000000000000020002000407B
:1015F000000000000000000000000000007000007B
:1016000000000000000000000000000000000000DA
:1016100000000000000000000000002000000000AA
:10162000000000100010001000200020002000200A
:1016300000400040000000000000001000280044AE
:101640000044004400440044002800100000000052
:1016500000000010003000500010001000100010BA
:10166000001000100000000000000030004800449E
:1016700000040008001000200040007C0000000072
:10168000000000300048000400080010000800447A
:10169000004800300000000000000008001800189A
:1016A000002800280048007C000800080000000016
:1016B0000000003C0020004000700048000400448E
:1016C0000048003000000000000000180024004026
:1016D0000050006800440044002800100000000092
:1016E0000000007C00040008001000100010002022
:1016F000002000200000000000000010002800442E
:1017000000280010002800440028001000000000FD
:1017100000000010002800440044002C00140004C5
:101720000048003000000000000000000000002021
:101730000000000000000000000000200000000089
:101740000000000000000020000000000000000079
:1017500000000020002000400000000000040008FD
:1017600000300040003000080004000000000000CD
:10177000000000000000007C00000000007C000071
:1017800000000000000000000000000000400020F9
:1017900000180004001800200040000000000000B5
:1017A000000000380064004400040008001000102D
:1017B00000000010000000000000800F4010A02E6C
:1017C000A0512051205120512053C04D20204010C5
:1017D000000000080014001400140022003E002243
:1017E00000410041000000000000003C00220022F7
:1017F0000022003C002200220022003C00000000E9
:101800000000000E00110021002000200020002117
:101810000011000E000000000000003C002200212A
:1018200000210021002100210022003C00000000D6
:101830000000003E002000200020003E002000208C
:101840000020003E000000000000003E00200020BC
:101850000020003C002000200020002000000000AC
:101860000000000E001100210020002700210021AF
:101870000011000E000000000000002100210021E6
:101880000021003F00210021002100210000000074
:101890000000002000200020002000200020002068
:1018A00000200020000000000000000800080008E0
:1018B0000008000800080048004800300000000050
:1018C00000000022002400280028003800280024FE
:1018D0000024002200000000000000200020002062
:1018E00000200020002000200020003E000000001A
:1018F00000008020803180318031802A802A802A37
:10190000802A802400000000000000210031003106
:1019100000290029002500230023002100000000E9
:101920000000000C001200210021002100210021F4
:101930000012000C000000000000003C0022002209
:101940000022003C002000200020002000000000B9
:101950000000000C001200210021002100210021C4
:101960000016000D000100000000003E00210021D3
:101970000021003E00240022002180200000000001
:101980000000001C002200220020001C0002002297
:101990000022001C000000000000003E00080008BB
:1019A0000008000800080008000800080000000007
:1019B0000000002100210021002100210021002140
:1019C0000012000C00000000000000410041002255
:1019D000002200220014001400140008000000007F
:1019E00000004044404A402A802A802A802A802AD7
:1019F000802A0011000000000000004100220014B5
:101A0000001400080014001400220041000000002F
:101A10000000004100220022001400080008000815
:101A200000080008000000000000007E0002000422
:101A300000080010001000200040007E00000000A0
:101A400000000030002000200020002000200020A6
:101A50000020002000200020000000400040002066
:101A600000200020002000200010001000000000D6
:101A70000000006000200020002000200020002046
:101A80000020002000200020000000100028002876
:101A900000280044000000000000000000000000DA
:101AA0000000000000000000000000000000000036
:101AB000000000000000007E004000200000000048
:101AC0000000000000000000000000000000000016
:101AD000000000000000003800440004003C004406
:101AE0000044003C0000000000000040004000589E
:101AF00000640044004400440064005800000000FA
:101B0000000000000000003000480040004000409D
:101B10000048003000000000000000040004003411
:101B2000004C004400440044004C0034000000001D
:101B3000000000000000003800440044007C004029
:101B4000004400380000000000000060004000E099
:101B50000040004000400040004000400000000005
:101B60000000000000000034004C00440044004429
:101B7000004C0034000400440000004000400058C5
:101B8000006400440044004400440044000000009D
:101B900000000040000000400040004000400040C5
:101BA0000040004000000000000000400000004035
:101BB0000040004000400040004000400040004025
:101BC00000000040004000480050006000500050FD
:101BD00000480048000000000000004000400040B5
:101BE0000040004000400040004000400000000075
:101BF0000000000000000052006D0049004900494B
